:100000000C94A7080C94D2080C94D2080C94D20833
:100010000C94D2080C94D2080C94D2080C94D208F8
:100020000C94D2080C94D2080C94E4730C945E7275
:100030000C94D2080C94D2080C94D2080C94D208D8
:100040000C94D2080C9447300C94D2080C94D2082B
:100050000C94D2080C94D2080C9456130C94846D12
:100060000C94D2080C94D2080C94D2080C94D208A8
:100070000C94D2080C94D2080C94D2080C94D20898
:100080000C94D2080C94D2080C94D2080C94D20888
:100090000C94D2080C94D208084AD73B3BCE016E90
:1000A00084BCBFFDC12F3D6C74319ABD56833DDACF
:1000B0003D00C77F11BED9E4BB4C3E916BAAAABEDE
:1000C000000000803F05A84CCDB2D44EB93836A907
:1000D000020C50B9918688083CA6AAAA2ABE000044
:1000E00000803F4572726F723A0054656D706572A0
:1000F0006174757265206865617465642062656409
:10010000207377697463686564206F66662E204D7E
:10011000415854454D502074726967676572656433
:10012000202121003A20457874727564657220732D
:1001300077697463686564206F66662E204D494E4A
:1001400054454D502074726967676572656420215B
:10015000003A20457874727564657220737769740B
:1001600063686564206F66662E204D415854454D86
:100170005020747269676765726564203A292100AE
:10018000C001FA00F001F5003002F0007002EB004F
:10019000A002E600C002E1001003DC005003D7001B
:1001A000E003D2009004CD008004C800E005BE004A
:1001B0006006B9004007AA00F008A000700B960086
:1001C000F00D8C00E0108200E0137800F0176E0054
:1001D000D0196900701B6400401E5F0010205A0097
:1001E000F025500080294600D0303C00A032370076
:1001F0001035320020392D0020392800703A2300B4
:10020000A03B1E00A03C1900203D1600003F03004B
:10021000202D20496E76616C696420657874727552
:10022000646572206E756D626572202100202D203C
:10023000496E76616C696420657874727564657264
:10024000206E756D626572210020403A006F6B2050
:10025000543A00504944204175746F74756E65209E
:100260006661696C656420212C2054656D7065722F
:10027000617475726520746F206869676800204B2F
:10028000643A2000204B693A2000204B703A20004D
:10029000204E6F206F76657273686F6F7420002038
:1002A0004B643A2000204B693A2000204B703A20E2
:1002B0000020536F6D65206F76657273686F6F7481
:1002C0002000204B643A2000204B693A2000204B4C
:1002D000703A200020436C617369632050494420C8
:1002E000002054753A2000204B753A2000206D61A3
:1002F000783A2000206D696E3A200020643A200090
:1003000020626961733A20006563686F3A00207467
:100310006F6F206C6F6E6720657874727573696F8C
:100320006E2070726576656E7465640020636F6C14
:100330006420657874727573696F6E20707265766B
:10034000656E7465640024F404D9201BC40C5C0E33
:100350009804C4095F0265077101F405F900FB0404
:10036000B30048048700C103690058035500030324
:100370004500BE023A008402310053022A002902DD
:10038000250004022000E4011C00C8011900AF018F
:10039000170098011400840113007101100061011D
:1003A000100051010E0043010D0036010B002B011E
:1003B0000B0020010B00150109000C0109000301CD
:1003C0000800FB000800F3000800EB000700E40051
:1003D0000600DE000600D8000600D2000600CC00B1
:1003E0000500C7000500C2000500BD000400B900FB
:1003F0000400B5000400B1000400AD000400A90031
:100400000400A5000300A20003009F0004009B005D
:100410000300980003009500020093000300900081
:1004200003008D0002008B0003008800020086009C
:10043000020084000300810002007F0002007D00B2
:1004400002007B00020079000200770001007600C4
:1004500002007400020072000100710002006F00CF
:1004600002006D0001006C0002006A0001006900DA
:1004700002006700010066000100650001006400E1
:1004800002006200010061000100600001005F00E5
:1004900002005D0001005C0001005B0001005A00E9
:1004A00001005900010058000100570001005600EA
:1004B00001005500010054000100530000005300EA
:1004C00001005200010051000100500001004F00E6
:1004D00001004E0000004E0001004D0001004C00E4
:1004E00001004B0000004B0001004A0001004900E0
:1004F00001004800000048000100470001004600DC
:1005000000004600010045000000450001004400D5
:1005100001004300000043000100420000004200CF
:1005200001004100000041000100400001003F00C7
:1005300000003F0001003E0000003E0001003D00C1
:1005400000003D0001003C0000003C0000003C00B9
:1005500001003B0000003B0001003A0000003A00AF
:1005600001003900000039000100380000003800A7
:10057000000038000100370000003700010036009D
:100580000000360000003600010035000000350094
:100590000000350001003400000034000000340089
:1005A000010033000000330000003300010032007E
:1005B0000000320000003200010031000000310074
:1005C0000000310001003000000030000000300069
:1005D00001002F0000002F0000002F0000002F005E
:1005E00001002E0000002E0000002E0001002D0052
:1005F00000002D0000002D0000002D0001002C0047
:1006000000002C0000002C0000002C0001002B003A
:1006100000002B0000002B0000002B0001002A002E
:1006200000002A0000002A0000002A000100290022
:100630000000290000002900000029000000290016
:100640000100280000002800000028000000280009
:1006500000002800010027000000270000002700FC
:1006600000002700000027000100260000002600EF
:1006700000002600000026000000260001002500E2
:1006800000002500000025000000250000002500D6
:1006900000002500010024000000240000002400C8
:1006A00000002400000024000100230000002300BB
:1006B00000002300000023000000230000002300AE
:1006C00000002300010022000000220000002200A0
:1006D0000000220000002200000022000100210092
:1006E0000000210000002100000021000000210086
:1006F0000000210000002100010020000000200077
:100700000000200000002000000020000000200069
:10071000000020000000200001001F0000001F005A
:1007200000001F0000001F0000001F0000001F004D
:1007300000001F0001001E0000001E0000001E003F
:1007400000001E00000024F4D43050C38E20C2A24A
:100750004017828B7011127A910D816CD90AA861B1
:10076000E108C7586607615143061E4B5D05C14548
:10077000A7041A411104093D980371393103403629
:10078000DB0265339102D4305402802E1D02632CAB
:10079000EE01752AC501B028A001102781018F251F
:1007A00064012B244B01E0223401AC211F018D2078
:1007B0000D01801FFC00841EED00971DDF00B81C9A
:1007C000D200E61BC600201BBC00641AB200B2199E
:1007D000A8000A19A0006A189900D11791004017C3
:1007E0008B00B516840031167E00B31579003A15DA
:1007F0007300C7146F0058146A00EE136600881364
:10080000630025135E00C7125B006C1257001512BF
:100810005400C111510070114F0021114B00D6102E
:1008200049008D1047004610440002104200C00FDE
:100830004000800F3E00420F3C00060F3B00CB0EF5
:100840003800930E37005C0E3500270E3400F30D90
:100850003200C10D3100900D3000600D2E00320DC0
:100860002D00050D2C00D90C2B00AE0C2900850C99
:1008700029005C0C2700350C27000E0C2600E80B25
:100880002400C40B2400A00B23007D0B23005A0B73
:100890002100390B2100180B2000F80A1F00D90A8B
:1008A0001E00BB0A1E009D0A1D00800A1D00630A6F
:1008B0001C00470A1B002C0A1B00110A1A00F7092A
:1008C0001A00DD091900C4091900AB0919009209C1
:1008D00017007B091800630917004C091600360938
:1008E0001600200916000A091500F5081500E00891
:1008F0001400CC081400B8081400A40814009008D0
:1009000013007D0812006B081300580812004608F7
:100910001200340811002308110012081100010808
:100920001100F0071000E0071000D0071000C0070A
:100930001000B0070F00A107100091070E008307F9
:100940000F0074070F0065070E0057070E004907D8
:100950000E003B070D002E070E0020070D001307A9
:100960000D0006070D00F9060C00ED060D00E0066F
:100970000C00D4060C00C8060C00BC060C00B00627
:100980000C00A4060B0099060C008D060B008206D5
:100990000B0077060B006C060B0061060A00570679
:1009A0000B004C060A0042060A0038060A002E0612
:1009B0000A0024060A001A060A00100609000706A3
:1009C0000A00FD050900F4050900EB050900E20530
:1009D0000900D9050900D0050900C7050900BE05B1
:1009E0000900B5050800AD050800A50509009C052E
:1009F0000800940508008C050800840508007C05A3
:100A00000800740508006C050700650508005D0511
:100A10000700560508004E0507004705070040057A
:100A2000080038050700310507002A0507002305DF
:100A300007001C050600160507000F05070008053E
:100A4000060002050700FB040600F5040700EE049B
:100A50000600E8040600E2040700DB040600D504F3
:100A60000600CF040600C9040600C3040600BD0446
:100A70000600B7040600B1040500AC040600A60495
:100A80000600A00405009B040600950405009004E0
:100A900006008A04050085040500800406007A0427
:100AA000050075040500700405006B04050066046C
:100AB0000500610405005C040500570405005204AC
:100AC00005004D04050048040500430405003E04EC
:100AD00004003A04050035040500300404002C0429
:100AE000050027040400230405001E0404001A0462
:100AF000040016040500110404000D040400090498
:100B000005000404040000040400FC030400F803CE
:100B10000400F4030400F0030400EC030400E80301
:100B20000400E4030400E0030400DC030400D80331
:100B30000400D4030400D0030400CC030400C80361
:100B40000300C50303006563686F3A00205A3A004A
:100B500020593A0020583A00656E6473746F7073C0
:100B6000206869743A20004572726F723A005072C0
:100B7000696E7465722068616C7465642E206B699F
:100B80006C6C28292063616C6C6564202121006FE6
:100B90006B00526573656E643A006563686F3A0076
:100BA0002200556E6B6E6F776E20636F6D6D616E98
:100BB000643A22007A5F6D696E3A00795F6D696E02
:100BC0003A00785F6D696E3A005A3A00593A00204F
:100BD000436F756E7420583A00453A005A3A0059EE
:100BE0003A00583A004649524D574152455F4E41EE
:100BF0004D453A4D61726C696E2056313B20537001
:100C000072696E7465722F6772626C206D617368B1
:100C1000757020666F722067656E36204649524DAA
:100C2000574152455F55524C3A687474703A2F2FB1
:100C30007777772E6D656E64656C2D706172747355
:100C40002E636F6D2050524F544F434F4C5F5645AB
:100C50005253494F4E3A312E30204D414348494E70
:100C6000455F545950453A4D656E64656C20455852
:100C70005452554445525F434F554E543A310A0041
:100C800020423A0020453A00543A0020573A0020CA
:100C9000453A00543A0020403A0020423A006F6B37
:100CA00020543A00456E642066696C65206C697357
:100CB0007400426567696E2066696C65206C6973B3
:100CC0007400446F6E65207072696E74696E67207F
:100CD00066696C65006F6B004E6F204C696E652015
:100CE0004E756D626572207769746820636865630C
:100CF0006B73756D2C204C617374204C696E653A72
:100D0000004E6F20436865636B73756D207769745F
:100D100068206C696E65206E756D6265722C204C62
:100D2000617374204C696E653A00636865636B7328
:100D3000756D206D69736D617463682C204C6173EF
:100D400074204C696E653A004C696E65204E756D75
:100D5000626572206973206E6F74204C6173742019
:100D60004C696E65204E756D6265722B312C204C7E
:100D7000617374204C696E653A00446F6E65207330
:100D80006176696E672066696C652E006F6B002066
:100D900020506C616E6E657242756666657242794E
:100DA0007465733A20002046726565204D656D6F4D
:100DB00072793A20006572696B00207C204175745D
:100DC000686F723A2000323031322D30322D323598
:100DD00000204C61737420557064617465643A201E
:100DE00000312E302E3020524332004D61726C693A
:100DF0006E3A200020536F667477617265205265E9
:100E000073657400205761746368646F672052656E
:100E1000736574002042726F776E206F7574205274
:100E200065736574002045787465726E616C20523C
:100E30006573657400506F776572557000737461E7
:100E40007274002200656E717565696E67202200FC
:100E50007C3C3E5E2B3D3F2F5B5D3B2C2A225C00A1
:100E60006563686F3A0043616E6E6F7420656E74DF
:100E70006572207375626469723A004572726F72AE
:100E80003A006572726F722077726974696E6720BA
:100E9000746F2066696C65004E6F74205344207037
:100EA00072696E74696E67002F0053442070726916
:100EB0006E74696E67206279746520002E00446547
:100EC0006C6574696F6E206661696C65642C204680
:100ED000696C653A200046696C652064656C6574D0
:100EE00065643A002E006F70656E206661696C65FE
:100EF000642C2046696C653A200057726974696EEB
:100F00006720746F2066696C653A20002E006F7050
:100F1000656E206661696C65642C2046696C653A73
:100F200020002E006F70656E206661696C65642C10
:100F30002046696C653A200046696C652073656CD3
:100F40006563746564002053697A653A0046696C8C
:100F500065206F70656E65643A002E006F70656E77
:100F6000206661696C65642C2046696C653A2000D6
:100F7000776F726B446972206F70656E206661696D
:100F80006C656400776F726B446972206F70656E78
:100F9000206661696C65640053442063617264205B
:100FA0006F6B006F70656E526F6F74206661696C55
:100FB000656400766F6C756D652E696E6974206668
:100FC00061696C656400534420696E6974206661D0
:100FD000696C0001290229042908291029202940C7
:100FE000298029012C022C0126022604260826101D
:100FF00026202640268026402C802C012302230414
:1010000023082310232023402380230120022004CF
:101010002008201020202040208020102C202C018F
:101020002F022F042F082F102F202F402F802F7ECC
:10103000FE7EFD7EFB7EF77EEF7EDF7EBF7E7F0045
:10104000010000731012000200008510430003002D
:1010500000C8100401030904CC101802030904E6B7
:10106000101603030904FE100C0001C102018036B2
:101070000181361201000202000020C01683040024
:10108000010102030109024300020100C032090408
:1010900000000102020100052400100105240100E6
:1010A0000104240206052406000107058203080046
:1010B0004009040100020A00000007050302400085
:1010C00000070584024000000403090418035400CB
:1010D000650065006E0073007900640075006900AA
:1010E0006E006F0000001603550053004200200000
:1010F000530065007200690061006C0000000C0381
:10110000310032003300340035000000494E4649BA
:101110004E4954594E414ECDCCCC3D0AD7233C17B5
:10112000B7D13877CC2B329595E6241FB14F0A0002
:101130000020410000C84200401C4620BCBE4CCAF2
:101140001B0E5AAEC59D74000E393070093911243A
:101150001FBECFEFD0E2DEBFCDBF12E0A0E0B1E016
:10116000EAE9F3EF00E00BBF02C007900D92AE3D3D
:10117000B107D9F71BBE1DE0AEEDB2E001C01D9274
:10118000AD3BB107E1F711E1CCE4D1E104C0229716
:10119000FE010E947379C834D107C9F70E943672E4
:1011A0000C94C1790C940000A0E0B0E0EAEDF8E006
:1011B0000C949079EC015B016115710519F0FB014C
:1011C00091838083F9908F2D90E00E947779892B0D
:1011D000C9F7FDE2FF1621F4F990EE24E39405C06F
:1011E0002BE2F21609F4F990EE248E010150104022
:1011F000C8016CE071E143E050E062D2892BF9F460
:101200008E010E5F1F4FC8016FE071E145E050E0B5
:1012100057D2892B19F48E01095F1F4FA114B10415
:1012200019F0F50111830083E0FC04C070E090E048
:1012300080E813C070E090E080E86FEF07C1C8015C
:1012400064E171E143E050E03BD2892B69F4A114E1
:10125000B10429F470E090E080EC6FE7F7C02296CB
:10126000F501D183C083F6CF8824992440E050E073
:1012700060E070E0EF2DE053EA30A0F5F2E0EF2AF5
:101280008E2D90E09C0128703070E2FE06C0232B6A
:1012900079F50894811C911C2BC0232B19F008941C
:1012A00081089108DB01CA0112E0880F991FAA1F6B
:1012B000BB1F1A95D1F7480F591F6A1F7B1F440F98
:1012C000551F661F771F4E0F511D611D711D483937
:1012D00029E9520729E9620729E1720748F084E009
:1012E000E82A06C0EE3F31F4E3FC39C098E0E92A71
:1012F000F990C0CFE53311F0E53189F529912D3210
:1013000019F4E0E1EE2A05C02B3219F081E090E0FB
:1013100003C0299182E090E0E22FE053EA3018F018
:10132000C81BD90B1CC020E030E0FCE020383F0790
:101330005CF4C901880F991F880F991F280F391F66
:10134000220F331F2E0F311DE991E053EA3068F36D
:10135000E4FE03C0309521953F4F820E931ECE2CA4
:10136000DD24E1FE07C0A114B10421F02197F501AD
:10137000D183C083CB01BA010E94DC757B018C0153
:10138000F3E0CF22DD2423E0C216D10421F417FBC1
:10139000109517F9109557016801C801B70120E0B1
:1013A00030E040E050E00E943C75882309F44AC0D8
:1013B00097FE0DC02BE2E22E21E1F22E9094819453
:1013C00091089394C0E2D0E000E010E012C093E4F2
:1013D000E92E91E1F92EF6CFF7012591359145914E
:1013E0005491C601B5010E941C785B016C018C1AF6
:1013F0009D0A8C169D0684F7D595C7950F5F1F4FE4
:101400000630110529F08CEF9FEFE80EF91EF1CFA1
:10141000C501D6017C018D018C2D880F8D2D881F73
:101420008F3F51F0C601B50120E030E040E050E0D0
:101430000E943C75882331F482E290E09093BC0DC9
:101440008093BB0D7E2D9F2D802F612F272F392F4D
:10145000482F562FB901CA01CDB7DEB7ECE00C9486
:10146000AC792F923F925F926F927F928F929F9270
:10147000AF92BF92CF92DF92EF92FF920F931F93A2
:10148000CF93DF938C011B01EA016115710519F0FF
:10149000FB0191838083209749F0CE0102978397C7
:1014A00028F020E030E040E050E0F6C0F801A190E4
:1014B0008F018A2D90E00E947779892BB9F7FDE2A0
:1014C000AF1631F4F801A1908F015524539407C051
:1014D000FBE2AF1619F4F801A1908F015524209773
:1014E00019F0C031D105C1F4F0E3AF1679F4F80179
:1014F0008081883711F0883549F4F801A1800E5FAA
:101500001F4FF2E05F2AC0E1D0E006C0209721F42F
:1015100080E3A816E9F427C0C830D10531F1C930FD
:10152000D10524F4C230D10531F50CC0CA30D10543
:1015300089F0C031D105F9F4C12CD12CE12CB8E0EF
:10154000FB2E28C0C12CD12CE12CA0E4FA2E22C005
:10155000CAE0D0E0FCECCF2EFCECDF2EFCECEF2E52
:10156000FCE0FF2E17C0C8E0D0E0C12CD12CE12C4C
:10157000E0E1FE2E0FC09E01442737FD4095542F19
:1015800060E070E080E090E80E942079C901DA0113
:101590006C017D0120E030E040E050E060E03E0181
:1015A000882477FC8094982C70EDB72EBA0CE9E073
:1015B000EB1570F48A2D81548A3118F499ECB92E08
:1015C00006C08A2D81568A3150F589EAB82EBA0CA8
:1015D0008B2D90E08C179D0714F56F3FE1F0C2163C
:1015E000D306E406F506B0F0CA01B901A4019301DF
:1015F0000E94EE789B01AC012B0D311D411D511D48
:101600002130F0E03F07F0E04F07F0E85F0710F40B
:1016100061E001C06FEFF801A1908F01C5CF2114E7
:10162000310481F0662331F001501040F101118343
:10163000008308C051FE1AC002501040F10111830E
:10164000008314C067FF12C050FC05C02FEF3FEFAE
:101650004FEF5FE704C020E030E040E050E882E276
:1016600090E09093BC0D8093BB0D16C050FE08C057
:1016700050954095309521953F4F4F4F5F4F0CC08F
:1016800057FF0AC082E290E09093BC0D8093BB0D9F
:101690002FEF3FEF4FEF5FE7B901CA01DF91CF9125
:1016A0001F910F91FF90EF90DF90CF90BF90AF9080
:1016B0009F908F907F906F905F903F902F900895B4
:1016C000FB01DC014150504088F08D9181341CF0C9
:1016D0008B350CF4805E659161341CF06B350CF435
:1016E000605E861B611171F3990B0895881BFCCF16
:1016F000FB01DC0104C08D910190801921F441505F
:101700005040C8F7881B990B0895FB01DC0102C00B
:1017100001900D9241505040D8F70895FB01DC0133
:101720000D900020E9F7119701900D920020E1F74C
:101730000895FC018191861721F08823D9F7992714
:1017400008953197CF010895FB01DC0101900D92BE
:101750000020E1F70895FB01DC014150504030F0DA
:101760008D910190801919F40020B9F7881B990B0D
:101770000895FB01DC014150504048F001900D926A
:101780000020C9F701C01D9241505040E0F7089574
:10179000FB0151915523A9F0BF01DC014D91451783
:1017A0004111E1F759F4CD010190002049F04D912C
:1017B00040154111C9F3FB014111EFCF81E090E0E9
:1017C00001970895AEE0B0E0E8EEFBE00C94987964
:1017D0000D891E8986E08C831A8309838FEF9FE72A
:1017E0009E838D839E01275E3F4FCE0101966F89B8
:1017F000788DA9010AD02F813885020F131FF801B7
:1018000010822E96E4E00C94B479ABE0B0E0EBE00B
:10181000FCE00C948A793C012B015A01FC011782EF
:101820001682838181FD03C06FEF7FEFB9C19AE01B
:10183000892E1E010894211C311CF3012381F20121
:1018400023FD859123FF81912F01882309F4A5C1F0
:10185000853239F423FD859123FF81912F01853253
:1018600021F490E0B301B7D1E8CF982FFF24EE2404
:101870009924FFE1FF15D0F09B3269F09C3228F4E7
:10188000903259F0933291F40EC09D3249F090336A
:1018900069F441E024C052E0F52A84E0F82A28C027
:1018A00098E0F92A25C0E0E1FE2A22C0F7FC29C011
:1018B000892F80538A3070F4F6FE05C0989C902CD6
:1018C0001124980E15C0E89CE02C1124E80EF0E2DB
:1018D000FF2A0EC09E3229F4F6FC5FC140E4F42AD0
:1018E00007C09C3619F450E8F52A02C0983649F42E
:1018F000F20123FD959123FF91912F01992309F086
:10190000B8CF892F8554833018F08052833038F453
:1019100044E050E0A40EB51E5FE359830FC0933638
:1019200031F0933779F0933509F052C01FC0F501BB
:101930008081898342E050E0A40EB51E610101E080
:1019400010E011C0F501C080D180F6FC03C06FEF3C
:101950007FEF02C0692D70E042E050E0A40EB51E9A
:10196000C6012ED18C015FE7F52213C0F501C080BE
:10197000D180F6FC03C06FEF7FEF02C0692D70E0ED
:1019800042E050E0A40EB51EC6010FD18C0150E814
:10199000F52AF3FE06C018C080E290E0B3011BD127
:1019A000EA948E2D90E008171907B0F30DC0F601E8
:1019B000F7FC8591F7FE81916F0190E0B3010BD1A7
:1019C000E110EA94015010400115110581F7E2C0C1
:1019D000943611F0993661F5F7FE08C0F5012081C3
:1019E00031814281538184E090E00AC0F501808119
:1019F00091819C01442737FD4095542F82E090E06F
:101A0000A80EB91E9FE6F92257FF09C050954095D0
:101A1000309521953F4F4F4F5F4FE0E8FE2ACA01B6
:101A2000B901A1012AE030E002D1D82ED2183FC07E
:101A3000953729F41F2D1F7E2AE030E01DC01F2D91
:101A4000197F9F3661F0903720F4983509F0A5C0D2
:101A50000FC0903739F0983709F09FC004C028E0D4
:101A600030E00AC0106114FD146020E130E004C0D1
:101A700014FD166020E132E017FF08C0F501608117
:101A800071818281938144E050E008C0F50180813A
:101A90009181BC0180E090E042E050E0A40EB51ED0
:101AA000A101C5D0D82ED2188FE7F82EF122F6FE6C
:101AB0000BC05EEFF522D91438F4F4FE07C0F2FC37
:101AC00005C08FEEF82202C01D2D01C0192DF4FEB5
:101AD0000DC0FE01ED0DF11D8081803319F499EEEA
:101AE000F92208C01F5FF2FE05C003C08F2D867863
:101AF00009F01F5F0F2DF3FC13C0F0FE0EC01E1582
:101B000010F09D2C0AC09D2C9E0C911A1E2D05C014
:101B100080E290E0B3015FD01F5F1E15C8F304C0E0
:101B20001E1510F4E11A01C0EE2404FF0EC080E37C
:101B300090E0B30150D002FF1BC001FD03C088E755
:101B400090E00EC088E590E00BC0802F867881F091
:101B500001FF02C08BE201C080E2F7FC8DE290E061
:101B6000B30139D005C080E390E0B30134D09A943A
:101B7000D914C8F3DA94F101ED0DF11D808190E0E4
:101B8000B30129D0DD20B1F705C080E290E0B301B8
:101B900022D0EA94EE20C9F750CEF3016681778116
:101BA000CB012B96E2E10C94A679FC0105906150E3
:101BB00070400110D8F7809590958E0F9F1F089563
:101BC000FC016150704001900110D8F7809590950C
:101BD0008E0F9F1F08950F931F93CF93DF938C0158
:101BE000EB018B8181FF1BC082FF0DC02E813F81E5
:101BF0008C819D812817390764F4E881F98101936C
:101C0000F983E88306C0E885F985802F0995892B3B
:101C100031F48E819F8101969F838E8302C00FEFE6
:101C20001FEFC801DF91CF911F910F910895FA0125
:101C3000AA27283051F1203181F1E8946F936E7F0B
:101C40006E5F7F4F8F4F9F4FAF4FB1E03ED0B4E0FC
:101C50003CD0670F781F891F9A1FA11D680F791F3D
:101C60008A1F911DA11D6A0F711D811D911DA11D4E
:101C700020D009F468943F912AE0269F112430195E
:101C8000305D3193DEF6CF010895462F4770405DF9
:101C90004193B3E00FD0C9F7F6CF462F4F70405DA8
:101CA0004A3318F0495D31FD4052419302D0A9F703
:101CB000EACFB4E0A6959795879577956795BA95FD
:101CC000C9F700976105710508959B01AC010A2EC3
:101CD00006945795479537952795BA95C9F7620F9A
:101CE000731F841F951FA01D08952F923F924F923E
:101CF0005F926F927F928F929F92AF92BF92CF929C
:101D0000DF92EF92FF920F931F93DF93CF93CDB7A4
:101D1000DEB7CD55D0400FB6F894DEBF0FBECDBFB5
:101D20002F969FAF8EAF2F9761967FAF6EAF619763
:101D30002A0162962FAF629763960FAF63976496FE
:101D4000EFAE64976896ACAEBDAECEAEDFAE689730
:101D5000E22EFF24EE0CFF1CEE0CFF1C9A012E0D50
:101D60003F1D2D963FAF2EAF2D97D9016D907D90E1
:101D70008D909C90FC01EE0DFF1DC401B3012081EC
:101D80003181428153810E94637469AF7AAF8BAF16
:101D90009CAF10E0000F111F000F111FF201E00FA8
:101DA000F11F2B96FFAFEEAF2B97A080B180C280C2
:101DB000D3802F96EEADFFAD2F97E00FF11FC60138
:101DC000B50120813181428153810E9463746DABE2
:101DD0007EAB8FAB98AF64962FAD6497E22FF0E0A7
:101DE000EE0FFF1FEE0FFF1F2F96AEADBFAD2F976B
:101DF000AE0FBF1F4D915D916D917C9129964CAFB7
:101E00005DAF6EAF7FAF299761966EAD7FAD619785
:101E1000E60FF71F608171818281938129962CAD35
:101E20003DAD4EAD5FAD29970E94627469AB7AAB50
:101E30008BAB9CAB6196AEADBFAD61971C968D919F
:101E40009D910D90BC91A02D25968CAF9DAFAEAF0E
:101E5000BFAF25972F96AEADBFAD2F971C962D9196
:101E60003D914D915C911F9721962CAF3DAF4EAFA8
:101E70005FAF2197A401930150582DA73EA74FA70C
:101E800058ABB601A501705849A75AA76BA77CA704
:101E900061966EAD7FAD6197E60EF71ED7016D912D
:101EA0007D918D919C9129AD3AAD4BAD5CAD0E9479
:101EB00062743B014C016196EEADFFAD61970E0F70
:101EC0001F1FD8016D917D918D919C912DA93EA9E7
:101ED0004FA958AD0E9462745B016C016DA57EA58F
:101EE0008FA598A9A60195010E941C787B018C0101
:101EF00069A57AA58BA59CA5A40193010E941C78D5
:101F00009B01AC01C801B7010E9462741B012C0146
:101F10006DA57EA58FA598A9A40193010E941C78A8
:101F20007B018C0169A57AA58BA59CA5A6019501CD
:101F30000E941C789B01AC01C801B7010E94637428
:101F40009B01AC01C201B1010E94D6745B016C011E
:101F500020E030E040E050E00E943C75882354F4DB
:101F6000C601B5012BED3FE049EC50E40E946374DB
:101F70005B016C01E7968FADE797882351F0C601AE
:101F8000B5012BED3FE049EC50E40E9462745B0127
:101F90006C01C601B501E6962CAD3DAD4EAD5FAD11
:101FA000E6970E941C7829A93AA94BA95CA95F77FA
:101FB0000E9457777B018C012FE632E143E85AE318
:101FC0000E943C7587FDE5C1C801B7010E941976E2
:101FD0000E94B07578A76FA380E090E00E94DC7546
:101FE0007B018C01C601B501A80197010E944375D0
:101FF0006BA37CA38DA39EA369A97AA98BA99CA995
:10200000A80197010E9443756F8F78A389A39AA3B3
:1020100025966CAD7DAD8EAD9FAD259721962CADEF
:102020003DAD4EAD5FAD21970E946274A80197014E
:102030000E9443756B8F7C8F8D8F9E8F6BA17CA1CF
:102040008DA19EA120E030E040E05FEB0E941C7873
:102050002BA13CA14DA15EA10E941C7820E030E0A4
:1020600040E85FE30E9463746F8B788F898F9A8F4B
:1020700064962FAD6497E22FF0E0EE0FFF1FEE0F96
:10208000FF1F9E012F5F3F4FE20FF31F29964CADBC
:102090005DAD6EAD7FAD29974083518362837383BD
:1020A0002F96AEADBFAD2F971C964D915D916D9162
:1020B0007C911F974D875E876F87788B41E050E05A
:1020C0005A8B498B662462967FAD6297672F70E0CA
:1020D000660F771F660F771FC901860F971F6A96D5
:1020E0009FAF8EAF6A976396BFAD6397AB2FB0E09B
:1020F000AA0FBB1FAA0FBB1F21E030E02C0F3D1F12
:102100002A0F3B1F6C963FAF2EAF6C976E96FFAFBA
:10211000EEAF6E9716C138E136150CF446C06DA5CA
:102120007EA58FA598A92BA13CA14DA15EA10E94DF
:102130001C787B018C0169A57AA58BA59CA52F89AC
:10214000388D498D5A8D0E941C789B01AC01C801C5
:10215000B7010E9463747B018C016DA57EA58FA5DC
:1021600098A92F89388D498D5A8D0E941C785B0162
:102170006C0169A57AA58BA59CA52BA13CA14DA1BD
:102180005EA10E941C789B01AC01C601B5010E94B2
:1021900062746DA77EA78FA798AB6394C701D8011F
:1021A00089A79AA7ABA7BCA765C049895A89BA0174
:1021B00080E090E00E94DC752BA13CA14DA15EA1C6
:1021C0000E941C787B018C01C8010E9440756B8BBA
:1021D0007C8B8D8B9E8BB701C8010E947F783B0161
:1021E0004C012D96AEADBFAD2D97ED90FD900D91AC
:1021F0001C9117FB109517F910952B96EEADFFADBE
:102200002B972080318042805380C801B7012B89F1
:102210003C894D895E890E941C785B016C01C2017A
:10222000B101A40193010E941C789B01AC01C6017D
:10223000B5010E9463746DA77EA78FA798ABC801F4
:10224000B701A40193010E941C787B018C01C2019B
:10225000B1012B893C894D895E890E941C789B01C4
:10226000AC01C801B7010E94627469A77AA78BA765
:102270009CA7662469AD7AAD8BAD9CAD2DA53EA51E
:102280004FA558A90E9463746A96AEADBFAD6A9718
:102290006D937D938D939C9313976DA97EA98FA9C0
:1022A00098AD29A53AA54BA55CA50E9463746C96D0
:1022B000EEADFFAD6C9760837183828393836E96DE
:1022C000AEADBFAD6E976D917D918D919C912F8D2F
:1022D00038A149A15AA10E9463746E96EEADFFAD7C
:1022E0006E9760837183828393836D857E858F85EE
:1022F00098892B8D3C8D4D8D5E8D0E9463746D870A
:102300007E878F87988BCE010196BE016B5F7F4FD2
:10231000AE01475F5F4F9E01235F3F4F6896ECAC75
:10232000FDAC0EAD1FAD6897F7E7CF2ED12CCC0ECC
:10233000DD1E0E94002329893A892F5F3F4F3A8B87
:10234000298B49895A896FA178A54617570708F440
:10235000E2CE61964EAD5FAD6197485F5F4F61968B
:102360002EAD3FAD6197245F3F4F61968EAD9FAD1F
:102370006197DC011496BD016896ECACFDAC0EAD26
:102380001FAD6897E7E7CE2ED12CCC0EDD1E0E9444
:102390000023C35ADF4F0FB6F894DEBF0FBECDBF88
:1023A000CF91DF911F910F91FF90EF90DF90CF9031
:1023B000BF90AF909F908F907F906F905F904F9065
:1023C0003F902F900895DF93CF930F92CDB7DEB754
:1023D000FC016983A081B18112962D913C911397E4
:1023E000BE016F5F7F4F41E050E0F90109950F900A
:1023F000CF91DF91089560E070E08FE793E4209142
:1024000018023091190240911A0250911B020E9449
:1024100043756093050370930603809307039093BD
:1024200008030895FC01E651FD4F808190E0089576
:102430000F931F93DC0141E050E0BA01660F771F54
:10244000660F771F6E5F7F4FFB01E058FE4F85914F
:1024500094918A179B070CF033C09A0121503040A9
:10246000220F331F220F331FC90180589E4FFC01DA
:10247000059114912E573E4FF90125913491FA019F
:10248000EE0FFF1FEE0FFF1FE058FE4F8591949156
:10249000FB01E058FE4F65917491801B910BA21BCC
:1024A000B30B621B730B9C012A9FC0012B9F900DE5
:1024B0003A9F900D11240E940D79600F711F11C079
:1024C000842F8F5F4F5F5F4F4432510509F0B5CFC6
:1024D000843219F060E070E004C0ECE0F2E0659155
:1024E000749120EF3FE3261B370BC9011F910F9119
:1024F00008952F923F924F925F926F927F928F92A8
:102500009F92AF92BF92CF92DF92EF92FF920F9382
:102510001F93CF93DF93C0EFDFE3C81BD90B21E0FC
:1025200030E0A901440F551F440F551FFA01E05830
:10253000FE4F85919491C817D9070CF059C0B90185
:1025400061507040660F771F660F771FCB018E5763
:102550009E4FFC010591149160587E4FFB01C59080
:10256000D490FA01EE57FE4FE590F490FA01E0584E
:10257000FE4FA590B490B801882777FD8095982FDD
:102580000E94DE751B012C01CC19DD09BE018827D4
:1025900077FD8095982F0E94DE753B014C01E01A73
:1025A000F10A0027F7FC0095102FC801B7010E941F
:1025B000DE759B01AC01C401B3010E941C787B0154
:1025C0008C01AC18BD08CC24B7FCC094DC2CC6012F
:1025D000B5010E94DE759B01AC01C801B7010E94E4
:1025E00043759B01AC01C201B1010E94637419C023
:1025F000822F8F5F2F5F3F4F2432310509F091CF3B
:10260000843229F0E0E070E080E060E00CC0EEE0B1
:10261000F2E065917491882777FD8095982F0E944C
:10262000DE75E62F692F2E2F372F482F562FB90131
:10263000CA01DF91CF911F910F91FF90EF90DF9032
:10264000CF90BF90AF909F908F907F906F905F9052
:102650004F903F902F9008950895CF93DF93449823
:1026600080919000877F80939000E3EEF0E064918A
:10267000EF0106C08DEA9DE0A6DE2196FE01649181
:102680006623C1F7EAEEF0E06491EF0106C08DEA3F
:102690009DE099DE2196FE0164916623C1F78DEAE3
:1026A0009DE06AE090DEDF91CF9108951F920F9236
:1026B0000FB60F920BB60F9211242F933F934F93A7
:1026C0005F936F937F938F939F93AF93BF93EF939A
:1026D000FF9390912802992331F48091EA0280932C
:1026E000EE028111459A8091EE02981708F0459804
:1026F0009F5F9F77909328028091EF02833009F4C7
:1027000048C0843028F48130E1F08230C0F50DC03B
:10271000853009F45CC0853008F457C0863009F470
:1027200058C0873009F05EC056C010927B0081E42B
:1027300080937C0080917A00806480937A0081E0AD
:102740001BC08091780090917900A0E0B0E02091CA
:10275000FC023091FD024091FE025091FF02280FD1
:10276000391F4A1F5B1F2093FC023093FD024093E8
:10277000FE025093FF0282E08093EF0233C080E4B8
:1027800080937C0080917A00806480937A0083E05B
:10279000F3CF8091780090917900A0E0B0E0209193
:1027A000F0023091F1024091F2025091F302280FB1
:1027B000391F4A1F5B1F2093F0023093F1024093B0
:1027C000F2025093F30284E0D7CF85E0D5CF86E0C4
:1027D000D3CF87E0D1CF1092EF02809100038F5FBB
:1027E0008093000380910003803108F45DC0409124
:1027F000FC025091FD025093E3024093E2022FEF5E
:102800003FE38091F0029091F102281B390B309345
:10281000E5022093E40281E08093EB021092000332
:102820001092FC021092FD021092FE021092FF0222
:102830001092F8021092F9021092FA021092FB0222
:102840001092F4021092F5021092F6021092F70222
:102850001092F0021092F1021092F2021092F30222
:1028600080912402909125024817590724F0109274
:10287000DF021092DE028091EC029091ED0284174B
:10288000950724F01092DF021092DE02809126025A
:1028900090912702281739073CF01092E10210921C
:1028A000E002DBDE0E941339FF91EF91BF91AF91FF
:1028B0009F918F917F916F915F914F913F912F9158
:1028C0000F900BBE0F900FBE0F901F9018952F9278
:1028D0003F924F925F926F927F928F929F92AF92B0
:1028E000BF92CF92DF92EF92FF920F931F93DF93ED
:1028F000CF9300D0CDB7DEB76C01162F662371F1F0
:10290000E3EEF0E064914F0108C08DEA9DE05BDDED
:102910000894811C911CF40164916623B1F7412F46
:1029200050E0662757FD6095762F8DEA9DE00E9466
:102930007171E0E1F2E064914F0108C08DEA9DE021
:1029400042DD0894811C911CF40164916623B1F767
:102950008DEA9DE06AE037DD0E941339A12FB0E0D7
:10296000AA0FBB1FFD01EC5AFD4F208131812115BB
:10297000310509F497C0E0EF8E2EEFE39E2E8C1800
:102980009D08AA5ABD4F4D915C9161E06CC08D01CC
:10299000000F111F000F111FF901E00FF11F8591AA
:1029A0009491881699060CF05DC0CD010197880FAF
:1029B000991F880F991FFC013296E20FF31FC590F3
:1029C000D490820F931FFC01859194919A838983FF
:1029D000F8013296E20FF31FE590F490F901E00F51
:1029E000F11FA590B490B601882777FD8095982FA8
:1029F0000E94DE751B012C01B401E981FA816E1B76
:102A00007F0B882777FD8095982F0E94DE753B010C
:102A10004C01EC18FD080027F7FC0095102FC801A9
:102A2000B7010E94DE759B01AC01C401B3010E9495
:102A30001C787B018C0189819A81A81AB90ACC245F
:102A4000B7FCC094DC2CC601B5010E94DE759B0169
:102A5000AC01C801B7010E9443759B01AC01C201E2
:102A6000B10137C06F5FA62FB0E0A417B5070CF413
:102A70008ECFA417B50729F0E0E070E080E060E0B9
:102A80002CC0FA01EE0FFF1FEE0FFF1F3297E20F6F
:102A9000F31F65917491882777FD8095982F0E9488
:102AA000DE7519C0B601882777FD8095982F0E94A2
:102AB000DE7520E030E04AEF5EE30E941C7820E003
:102AC00030E040E85DE30E941C7820E030E040E028
:102AD00050E00E946374E62F692F2E2F372F482F66
:102AE000562FB901CA010F900F90CF91DF911F911E
:102AF0000F91FF90EF90DF90CF90BF90AF909F909D
:102B00008F907F906F905F904F903F902F9008959F
:102B10002F923F924F925F926F927F928F929F92ED
:102B2000AF92BF92CF92DF92EF92FF920F931F93DB
:102B30008091EB02882309F490C18FB7F89410922A
:102B4000EB028FBF8091E2029091E30260E0BFDE72
:102B50003B014C016091E6027091E7028091E8022E
:102B60009091E902A40193010E9462747B018C019F
:102B700060930B0370930C0380930D0390930E03EB
:102B800020E030E040E251E40E944A77181624F435
:102B900081E080930F03EFC0C801B70120E030E06F
:102BA00040E251EC0E943C75882324F481E080933C
:102BB0000F03CCC080910F03882371F080E090E078
:102BC000A0E0B0E08093100390931103A093120350
:102BD000B093130310920F03C801B70120911402A0
:102BE0003091150240911602509117020E941C78F4
:102BF0001B012C016093140370931503809316033B
:102C000090931703C801B70120911003309111036D
:102C100040911203509113030E9463745B016C0195
:102C2000E0900103F090020300910303109104036C
:102C3000A80197010E943C7587FD12C0E090050332
:102C4000F09006030091070310910803C601B50137
:102C5000A80197010E944A77181614F086017501A1
:102C6000E0921003F09211030093120310931303E8
:102C7000C801B701209118023091190240911A023F
:102C800050911B020E941C785B016C016093180339
:102C90007093190380931A0390931B03C401B3012B
:102CA00020911C0330911D0340911E0350911F037E
:102CB0000E94627420911C0230911D0240911E02FC
:102CC00050911F020E941C7820ED3CEC4CE45DE327
:102CD0000E941C787B018C0160912003709121037C
:102CE000809122039091230323E333E343E75FE3DF
:102CF0000E941C789B01AC01C801B7010E9463745B
:102D00007B018C0160932003709321038093220345
:102D10009093230360921C0370921D0380921E0304
:102D200090921F03C201B101A60195010E94637434
:102D3000A80197010E9462747B018C0120E030E0C1
:102D400040E050E00E943C7588235CF40F2EF0E0D8
:102D5000EF2EF0E0FF2EF0E00F2FF0E01F2FF02D10
:102D600014C0C801B70120E030E04FE753E40E94EF
:102D70004A77181654F40F2EF0E0EF2EF0E0FF2EF5
:102D8000FFE70F2FF3E41F2FF02D2091E202309187
:102D9000E3028091EC029091ED028217930784F494
:102DA0008091240290912502281739074CF4C8011C
:102DB000B7010E94AB75759567956093EA0202C0F2
:102DC0001092EA020FB6F8948091A80D9091A90D87
:102DD000A091AA0DB091AB0D0FBE209124033091AC
:102DE00025034091260350912703821B930BA40BCC
:102DF000B50B88589341A040B04078F10FB6F894D5
:102E00008091A80D9091A90DA091AA0DB091AB0D44
:102E10000FBE8093240390932503A0932603B093C1
:102E200027032091E4023091E502809109039091FB
:102E30000A038217930784F4809126029091270257
:102E4000281739074CF48091E0029091E10228178D
:102E5000390714F4449A01C044981F910F91FF90D0
:102E6000EF90DF90CF90BF90AF909F908F907F902A
:102E70006F905F904F903F902F900895EF92FF9248
:102E80000F931F93CF93DF937C01062F662351F19D
:102E9000E3EEF0E06491EF0106C08DEA9DE093DA85
:102EA0002196FE0164916623C1F7402F50E066270A
:102EB00057FD6095762F8DEA9DE00E947171EDE2DD
:102EC000F2E06491EF0106C08DEA9DE07CDA219684
:102ED000FE0164916623C1F78DEA9DE06AE073DA32
:102EE0000E941339A02FB0E0AA0FBB1FFD01EC5ABE
:102EF000FD4FC081D181209709F468C0AA5ABD4F07
:102F00004D915C9121E047C0BD01660F771F660FB0
:102F1000771F6E5F7F4FFE01E60FF71F859194913B
:102F20008E159F050CF036C09D0121503040220FB8
:102F3000331F220F331FCE01820F931FFC01059117
:102F400014912E5F3F4F2C0F3D1FF90125913491B5
:102F5000FD01EE0FFF1FEE0FFF1FEC0FFD1F859110
:102F60009491FE01E60FF71F65917491801B910B00
:102F7000E21AF30A621B730B9C012E9DC0012F9D68
:102F8000900D3E9D900D11240E940D79CB01800F74
:102F9000911F17C02F5FA22FB0E0A417B5070CF444
:102FA000B3CFA417B50719F080E090E00AC0FA018A
:102FB0003197EE0FFF1FEE0FFF1FEC0FFD1F8591E6
:102FC000949160EF7FE3681B790B15C0B7018827E8
:102FD00077FD8095982F0E94DE752FE632E143E061
:102FE00050E40E941C7820E030E040E851E40E9468
:102FF0001C780E94AB75CB01DF91CF911F910F918F
:10300000FF90EF90089580E090E060E037DF9093CC
:10301000DF028093DE0280E090E0A0E0B0E08093E9
:10302000E6029093E702A093E802B093E90280E001
:1030300090E0FED91092DF021092DE021092EA02B6
:103040004598E0E9F0E080818F7D80831092E10275
:103050001092E00244988081877F8083089580E009
:1030600090E0A0E0B0E08093010390930203A0936E
:103070000303B093040360E070E08FE793E42091D2
:1030800018023091190240911A0250911B020E94BD
:103090004375609305037093060380930703909331
:1030A00008033D9A3C9A3E9A87ED80937A00EEE7BA
:1030B000F0E01082808182608083808181608083E3
:1030C00080E888BDEEE6F0E08081846080836AEF6E
:1030D00070E080E090E00E94C46D85E090E060E0E8
:1030E000CDDE9093ED028093EC028AEF90E060E0F9
:1030F000C5DE909325028093240285E090E098D964
:1031000090930A038093090386E990E091D9909304
:1031100027028093260208952F923F924F925F924A
:103120006F927F928F929F92AF92BF92CF92DF92D7
:10313000EF92FF920F931F93DF93CF93CDB7DEB73C
:10314000E4970FB6F894DEBF0FBECDBF6F8F78A3A4
:1031500089A39AA38FE78093EA020FB6F89420918F
:10316000A80D3091A90D4091AA0D5091AB0D0FBE45
:103170002D8B3E8B4F8B588FE091AD0DF091AE0DA6
:103180000280F381E02D8DEA9DE060E071E042E194
:1031900050E009958DEA9DE06AE015D98D899E89F8
:1031A000AF89B88D898B9A8BAB8BBC8B8D879E87B3
:1031B000AF87B88B1A8E198E11E05FE7652E712CE0
:1031C000812C912C4FE7242E312C412C512CE0E006
:1031D000F3E094919BA3EBEFF2E0A491ACA3E4EFB6
:1031E000F2E0B491BDA3EDEEF2E024912EA3E7EE60
:1031F000F2E034913FA3E1EEF2E0449148A7E4ED20
:10320000F2E0549159A7EEECF2E084918AA7E8EC41
:10321000F2E094919BA7E2ECF2E0A491ACA7E1EB81
:10322000F2E0B491BDA7EBEAF2E024912EA78091E1
:10323000EB02882309F4D2C38FB7F8941092EB0203
:103240008FBF8091E2029091E30260E040DB6FA7C4
:1032500078AB89AB9AAB69817A818B819C812FA5F0
:1032600038A949A95AA90E944A77181644F08FA58F
:1032700098A9A9A9BAA989839A83AB83BC83C601FB
:10328000B5012FA538A949A95AA90E943C7587FD07
:1032900006C08FA598A9A9A9BAA95C016D0111233F
:1032A00009F455C06FA578A989A99AA92F8D38A1CD
:1032B00049A15AA10E944A7718160CF08FC30FB685
:1032C000F8948091A80D9091A90DA091AA0DB091AC
:1032D000AB0D0FBE2D853E854F855889821B930B04
:1032E000A40BB50B89589341A040B04008F476C3B5
:1032F000D401C30182199309A409B509B595A7950D
:10330000979587958093EA020FB6F8948091A80D5F
:103310009091A90DA091AA0DB091AB0D0FBE898B14
:103320009A8BAB8BBC8B2D853E854F855889821B34
:10333000930BA40BB50B89879A87AB87BC878F8DBE
:1033400098A1A9A1BAA189839A83AB83BC836FA5F5
:1033500078A989A99AA92F8D38A149A15AA10E94BB
:103360003C7588230CF039C30FB6F8948091A80DF2
:103370009091A90DA091AA0DB091AB0D0FBE298916
:103380003A894B895C89821B930BA40BB50B895836
:103390009341A040B04008F420C30FB6F894809148
:1033A000A80D9091A90DA091AA0DB091AB0D0FBEE3
:1033B0008D879E87AF87B88BA98DBA8DAB2B09F40B
:1033C000F4C28D859E85AF85B88929893A894B8954
:1033D0005C89821B930BA40BB50B29853A854B8521
:1033E0005C85280F391F4A1F5B1F2B8F3C8F4D8F29
:1033F0005E8F29853A854B855C85281B390B4A0BE6
:103400005B0BCA01B901A20191010E94EE782B8DDC
:103410003C8D4D8D5E8D0E944279260D371D481DD5
:10342000591D24313105410551055CF424E1222E5A
:10343000312C412C512C94E1692E712C812C912C32
:103440001FC039014A013CEE6316710481049104E6
:103450002CF08BEE682E712C812C912C40E8641698
:103460007104810491041CF41301240109C00EEFBE
:10347000202E312C412C512C261837084808590889
:103480006BA100E013E008C08DEA9DE00E94E3110B
:103490000F5F1F4FF80164916623B1F78DEA9DE03D
:1034A000B401A3010E9471716CA10BEF12E008C07E
:1034B0008DEA9DE00E94E3110F5F1F4FF8016491B8
:1034C0006623B1F78DEA9DE0B201A1010E947171FE
:1034D0006DA104EF12E008C08DEA9DE00E94E311A7
:1034E0000F5F1F4FF80164916623B1F78DEA9DE0ED
:1034F000B601A50122E00E9482716EA10DEE12E0DC
:1035000008C08DEA9DE00E94E3110F5F1F4FF80194
:1035100064916623B1F78DEA9DE049815A816B8100
:103520007C8122E00E9482718DEA9DE06AE00E9427
:10353000E311298D3A8D233031050CF436C2C201D6
:10354000B1010E94DE7520E030E040E850E40E94C6
:103550001C787B018C0169817A818B819C81A60119
:1035600095010E94627420ED3FE049E450E40E941E
:103570001C7820E030E040E05FE30E941C789B0173
:10358000AC01C801B7010E9443756D837E838F83B0
:1035900098876B8D7C8D8D8D9E8D0E94DE7520E0D1
:1035A00030E04AE754E40E9443755B016C016FA16F
:1035B00007EE12E008C08DEA9DE00E94E3110F5F64
:1035C0001F4FF80164916623B1F78DEA9DE04D81AC
:1035D0005E816F81788522E00E94827168A501EE8C
:1035E00012E008C08DEA9DE00E94E3110F5F1F4FBB
:1035F000F80164916623B1F78DEA9DE0B601A5015B
:1036000022E00E9482718DEA9DE06AE00E94E3114F
:103610006D817E818F8198852AE939E949E15FE3EF
:103620000E941C787B018C0169A524ED32E03CAB43
:103630002BAB0CC08DEA9DE00E94E3114BA95CA965
:103640004F5F5F4F5CAB4BABFA016491662391F720
:103650008DEA9DE06AE00E94E3116AA52EEC32E05B
:103660003CAB2BAB0CC08DEA9DE00E94E3114BA953
:103670005CA94F5F5F4F5CAB4BABFA016491662373
:1036800091F78DEA9DE0B801A70122E00E948271C6
:103690008DEA9DE06AE00E94E3116BA528EC32E020
:1036A0003CAB2BAB0CC08DEA9DE00E94E3114BA913
:1036B0005CA94F5F5F4F5CAB4BABFA016491662333
:1036C00091F7C801B701A80197010E946374A60190
:1036D00095010E944375AB01BC018DEA9DE022E09B
:1036E0000E9482718DEA9DE06AE00E94E3116CA560
:1036F00022EC32E03CAB2BAB0CC08DEA9DE00E948B
:10370000E3114BA95CA94F5F5F4F5CAB4BABFA0178
:103710006491662391F7C801B701A60195010E9443
:103720001C7820E030E040E05EE30E941C78AB01B2
:10373000BC018DEA9DE022E00E9482718DEA9DE04D
:103740006AE00E94E3116D817E818F81988523EC70
:1037500035EF48EA5EE30E941C787B018C016DA581
:1037600021EB32E03CAB2BAB0CC08DEA9DE00E941C
:10377000E3114BA95CA94F5F5F4F5CAB4BABFA0108
:103780006491662391F78DEA9DE06AE00E94E3115F
:103790006EA52BEA32E03CAB2BAB0CC08DEA9DE072
:1037A0000E94E3114BA95CA94F5F5F4F5CAB4BAB31
:1037B000FA016491662391F78DEA9DE0B801A701B3
:1037C00022E00E9482718DEA9DE06AE00E94E3118E
:1037D000E5EAF2E06491FCABEBAB0CC08DEA9DE056
:1037E0000E94E3112BA93CA92F5F3F4F3CAB2BABB1
:1037F000F9016491662391F7C801B701A60195010B
:103800000E944375AB01BC018DEA9DE022E00E945D
:1038100082718DEA9DE06AE00E94E311EFE9F2E037
:103820006491FCABEBAB0CC08DEA9DE00E94E31110
:103830002BA93CA92F5F3F4F3CAB2BABF901649107
:10384000662391F7C801B701A60195010E941C7873
:1038500020E030E040E450E40E944375AB01BC013D
:103860008DEA9DE022E00E9482718DEA9DE06AE08F
:103870000E94E3116D817E818F8198852DEC3CEC57
:103880004CE45EE30E941C787B018C01E0E9F2E0ED
:103890006491FCABEBAB0CC08DEA9DE00E94E311A0
:1038A0002BA93CA92F5F3F4F3CAB2BABF901649197
:1038B000662391F78DEA9DE06AE00E94E311EAE851
:1038C000F2E06491FCABEBAB0CC08DEA9DE00E9492
:1038D000E3112BA93CA92F5F3F4F3CAB2BABF90168
:1038E0006491662391F78DEA9DE0B801A70122E07B
:1038F0000E9482718DEA9DE06AE00E94E311E4E893
:10390000F2E06491FCABEBAB0CC08DEA9DE00E9451
:10391000E3112BA93CA92F5F3F4F3CAB2BABF90127
:103920006491662391F7C801B701A80197010E942D
:103930006374A60195010E944375AB01BC018DEA39
:103940009DE022E00E9482718DEA9DE06AE00E9483
:10395000E311EEE7F2E06491FCABEBAB0CC08DEA57
:103960009DE00E94E3112BA93CA92F5F3F4F3CAB88
:103970002BABF9016491662391F7C801B701A60149
:1039800095010E941C7820E030E040E450E40E9461
:103990004375AB01BC018DEA9DE022E00E9482717B
:1039A0008DEA9DE06AE00E94E311D201C101860D1B
:1039B000971DA81DB91DB595A795979587958093D7
:1039C000EA02298D3A8D2F5F3F4F3A8F298FAF8CB6
:1039D000B8A0C9A0DAA011E001C010E06F8D78A1F5
:1039E00089A19AA120E030E040EA51E40E9463748A
:1039F0009B01AC016FA578A989A99AA90E944A7771
:103A000018166CF5E3E5F2E064918F0108C08DEAC9
:103A10009DE00E94E3110F5F1F4FF8016491662340
:103A2000B1F78DEA9DE06AE00E94E311E4960FB6DB
:103A3000F894DEBF0FBECDBFCF91DF911F910F91E4
:103A4000FF90EF90DF90CF90BF90AF909F908F90BE
:103A50007F906F905F904F903F902F9008950FB69A
:103A6000F8948091A80D9091A90DA091AA0DB09104
:103A7000AB0D0FBE2D893E894F89588D821B930B4C
:103A8000A40BB50B815D9740A040B04008F4CFCBAC
:103A90000FB6F8948091A80D9091A90DA091AA0D50
:103AA000B091AB0D0FBE8D8B9E8BAF8BB88FEDE4BD
:103AB000F2E064917F0109C08DEA9DE00E94E3116C
:103AC0000894E11CF11CF70164916623A9F7809129
:103AD000E2029091E3020E946714AB01BC018DEAFF
:103AE0009DE022E00E948271E9E4F2E064917F01AE
:103AF00009C08DEA9DE00E94E3110894E11CF11CCD
:103B0000F70164916623A9F74091EA0250E0662725
:103B100057FD6095762F8DEA9DE00E9471718DEAC8
:103B20009DE06AE00E94E31182CB90916908809148
:103B30006808981781F140916908242F30E08DE4DE
:103B400090E0289FF001299FF00D389FF00D11247F
:103B5000E052FC4F308120E06DE470E016C0842F0D
:103B600090E0869FF001879FF00D969FF00D112445
:103B7000E052FC4F80819181A281B3810097A10521
:103B8000B10509F02F5F4F5F4F70809168084817AB
:103B900031F7E32F11C08091C809882359F03E9A6C
:103BA00090E09093990080939800809190008068B5
:103BB0008093900020E0E0E08091C809882369F4B8
:103BC0002223C9F43E9A1092990010929800809195
:103BD00090008068809390000895EE2361F03E9AF3
:103BE0008E2F90E0909399008093980080919000A0
:103BF000806880939000089580936A080895FC017E
:103C000060817181828193812091480330914903C1
:103C100040914A0350914B030E941C780E94EC771C
:103C20006093940370939503809396039093970306
:103C300084E993E00C94DA2FAF92BF92CF92DF9297
:103C4000EF92FF920F931F93FC017B016A015901D0
:103C5000608171818281938120913C0330913D0389
:103C600040913E0350913F030E941C780E94EC77E4
:103C700008E813E0609388037093890380938A03B4
:103C800090938B03F70160817181828193812091F0
:103C900040033091410340914203509143030E94FD
:103CA0001C780E94EC7760938C0370938D03809353
:103CB0008E0390938F03F6016081718182819381DD
:103CC00020914403309145034091460350914703AE
:103CD0000E941C780E94EC7728E0E22EF12CE00E86
:103CE000F11E6093900370939103809392039093DD
:103CF0009303F50160817181828193812091480352
:103D00003091490340914A0350914B030E941C7823
:103D10000E94EC779801245F3F4F60939403709367
:103D200095038093960390939703C8010C5F1F4FF0
:103D3000B801A7010E94A02F80E090E0A0E0B0E0D1
:103D400080936B0890936C08A0936D08B0936E08F5
:103D500080936F0890937008A0937108B0937208D5
:103D60008093730890937408A0937508B0937608B5
:103D70008093770890937808A0937908B0937A0895
:103D800080937B0890937C08A0937D08B0937E0875
:103D90001F910F91FF90EF90DF90CF90BF90AF9069
:103DA00008958F929F92AF92BF92CF92DF92EF923F
:103DB000FF920F931F93CF93DF93EC016B0100975A
:103DC00009F45CC08FA9882309F058C0EEA0FFA0B9
:103DD00008A519A5FB01B6A0A7A090A481A4C801BD
:103DE000B7012B2D3A2D492D582D0E943C75882363
:103DF0000CF044C0C801B701A80197010E941C78CB
:103E00007B018C016AA97BA98CA99DA9905820E00F
:103E100030E040E050EC0E941C782EA53FA548A958
:103E200059A90E941C789B01AC01C801B7010E94EE
:103E300063740E9489787B018C016B2D7A2D892D0A
:103E4000982D9701A8010E943C75882324F4EB2C3F
:103E5000FA2C092D182D6B2D7A2D892D982D97016F
:103E6000A8010E943C75882349F0C701D801F601DA
:103E700086A397A3A0A7B1A781E086ABDF91CF91DE
:103E80001F910F91FF90EF90DF90CF90BF90AF9078
:103E90009F908F900895EF92FF920F931F93CF936F
:103EA000DF93F090690800E010E020E030E04DE49E
:103EB000E42E11C0FE9CE0011124C856DC4FC9015C
:103EC000B801AE016EDF8F2D8F5F803109F480E085
:103ED000F82E98018E0180916808F81659F7C901EB
:103EE000B80140E050E05DDFDF91CF911F910F916D
:103EF000FF90EF900895AF92BF92CF92DF92EF9232
:103F0000FF920F931F93CF93DF93EB018A0161150B
:103F1000710509F466C04115510509F462C0DAA4BF
:103F2000CBA4BCA4ADA46EA17FA188A599A52D2D7D
:103F30003C2D4B2D5A2D0E943C75882309F451C00D
:103F40008FA9882309F043C0F801E6A0F7A000A5D7
:103F500011A56D2D7C2D8B2D9A2DA80197010E9406
:103F60004A771816A4F5C801B701A80197010E9465
:103F70001C787B018C016AA97BA98CA99DA990580A
:103F800020E030E040E050EC0E941C782EA53FA5D8
:103F900048A959A90E941C789B01AC01C801B7012E
:103FA0000E9463740E9489787B018C016D2D7C2DA9
:103FB0008B2D9A2D9701A8010E943C75882324F42B
:103FC000ED2CFC2C0B2D1A2DC701D80104C08D2D12
:103FD0009C2DAB2DBA2D8EA39FA3A8A7B9A781E0D6
:103FE0008EABDF91CF911F910F91FF90EF90DF90FB
:103FF000CF90BF90AF900895CF92DF92FF920F9332
:10400000DF93CF9300D0CDB7DEB780916808809161
:1040100068082091690890E04096821B91098F7092
:10402000907004970CF10091680803500F70CC2435
:10403000DD2440E050E06DE4F62E12C0802F002316
:1040400009F480E1082F01500F9DC001112488560A
:104050009C4F9A838983B6014EDFA601C980DA801E
:1040600080916908081751F70F900F90CF91DF9159
:104070000F91FF90DF90CF900895109268081092F2
:10408000690880E1E8E8F3E0DF011D928A95E9F72D
:1040900080E090E0A0E0B0E080936F08909370081B
:1040A000A0937108B093720880937308909374087A
:1040B000A0937508B093760880937708909378085A
:1040C000A0937908B0937A0880937B0890937C083A
:1040D000A0937D08B0937E0880936B0890936C0842
:1040E000A0936D08B0936E0808952F923F924F925F
:1040F0005F926F927F928F929F92AF92BF92CF9278
:10410000DF92EF92FF920F931F93DF93CF93CDB780
:10411000DEB766970FB6F894DEBF0FBECDBF9E8B9D
:104120008D8B6A017B0148015901DC01D8966D91A4
:104130007D918D919C91DB970E94DC75698B7A8BC8
:104140008B8B9C8BA70196010E941C780E9429757D
:104150000E94B0756D837E838F83988769897A8981
:104160008B899C89A50194010E941C780E94297565
:104170000E94B07569837A838B839C832D813E81F5
:104180004F815885283731054105510540F448E7EE
:1041900050E060E070E04D835E836F8378876981D3
:1041A0007A818B819C81683771058105910540F486
:1041B00088E790E0A0E0B0E089839A83AB83BC837A
:1041C000AD89BE89AC5BBF4FAD90BD90CD90DC900A
:1041D0001397A454B040BE8BAD8BDC966D917D914E
:1041E0008D919C91DF970E94DC756D877E878F870C
:1041F000988BC601B5010E94DE751B012C0120E0E1
:1042000030E040E050E00E943C75882321F4E0E07B
:1042100070E060E028C069897A898B899C899B015C
:10422000AC010E941C787B018C016D857E858F8599
:1042300098899B01AC010E941C789B01AC01C801CC
:10424000B7010E9462747B018C01C201B101A2011D
:1042500091010E9463749B01AC01C801B7010E94E7
:104260004375E62F692F2E2F372F482F562FB90170
:10427000CA010E9429750E94AB753B014C01ED8972
:10428000FE89E05CFF4F60817181828193810E9491
:10429000DC7569877A878B879C8766277727CB01B0
:1042A0006A197B098C099D090E94DE755B016C010E
:1042B00020E030E040E050E00E943C75882321F48B
:1042C000E0E070E060E028C069857A858B859C8598
:1042D0009B01AC010E941C787B018C0169897A8961
:1042E0008B899C899B01AC010E941C789B01AC01CD
:1042F000C801B7010E9462747B018C01C601B5013F
:10430000A60195010E9463749B01AC01C801B7012D
:104310000E944375E62F692F2E2F372F482F562FD7
:10432000B901CA010E941976ED89FE89A088B18879
:10433000C288D38886017501E618F70808091909AB
:104340000E94AB75A8019701261B370B480B590B30
:1043500057FF71C0C201B10120E030E040E050E001
:104360000E943C75882321F4E0E070E060E044C0E6
:10437000C201B101A20191010E9463747B018C0111
:10438000C601B5010E94DC759B01AC01C801B701F3
:104390000E941C787B018C016D857E858F859889B4
:1043A0009B01AC010E941C789B01AC01C801B701C4
:1043B0000E9462747B018C0169857A858B859C855E
:1043C0009B01AC010E941C789B01AC01C801B701A4
:1043D0000E9463747B018C01C201B10120E030E0D6
:1043E00040E850E40E941C789B01AC01C801B70171
:1043F0000E944375E62F692F2E2F372F482F562FF7
:10440000B901CA010E9429750E94AB75AC01CB01AC
:10441000DA013C014D0197FE03C066247724430175
:104420006A147B048C049D0410F03501460120E0E1
:1044300030E040E050E09FB7F8946D897E89645B7E
:104440007F4FDB018C91AC54B040BE8BAD8B882389
:1044500021F5FD01648A758A868A978A260D371DA3
:10446000481D591D58962D933D934D935C935B9732
:104470002D813E814F815885DC962D933D934D9340
:104480005C93DF97A05CBF4F29813A814B815C81AF
:104490002D933D934D935C9313979FBF66960FB6F4
:1044A000F894DEBF0FBECDBFCF91DF911F910F916A
:1044B000FF90EF90DF90CF90BF90AF909F908F9044
:1044C0007F906F905F904F903F902F9008954F9204
:1044D0005F927F928F929F92AF92BF92CF92DF9224
:1044E000EF92FF920F931F93CF93DF937090690821
:1044F000C0E0D0E07DE4472E512C45C02097A9F1C3
:104500008EA9882361F4849CF001859CF00D949C15
:10451000F00D1124E856FC4F86A9882331F1EAA05A
:10452000FBA00CA11DA16EA17FA188A599A5A80142
:1045300097010E9443755B016C01849CF001859C8E
:10454000F00D949CF00D1124E856FC4F66A177A164
:1045500080A591A5A80197010E9443758B019C013C
:10456000CE01B601A501C1DD1EAA739480E17816C3
:1045700009F47724849CE001859CD00D949CD00D97
:104580001124C856DC4F872C992487FC9094809185
:10459000680890E08816990609F0B0CF2097E9F0F6
:1045A000EAA0FBA00CA11DA16EA17FA188A599A5E1
:1045B000A80197010E9443755B016C0160E070E007
:1045C00080E090E4A80197010E9443758B019C0153
:1045D000CE01B601A50189DD1EAADF91CF911F9101
:1045E0000F91FF90EF90DF90CF90BF90AF909F9092
:1045F0008F907F905F904F900895FEDC4CDC67CFEA
:104600002F923F924F925F926F927F928F929F92E2
:10461000AF92BF92CF92DF92EF92FF920F931F93D0
:10462000DF93CF93CDB7DEB7C558D0400FB6F8941F
:10463000DEBF0FBECDBF5C014B013A012901CE5751
:10464000DF4FE882C258D040CD57DF4FF882C358C1
:10465000D040CC57DF4F0883C458D040CB57DF4FF2
:104660001883C558D040E296DFAECEAEE297809177
:1046700068088F5F803109F480E0282F332727FDF9
:10468000309539AB28AB05C00E94881581E00E94A7
:1046900040398091690890E048A959A98417950785
:1046A00099F3D5016D917D918D919C9120913C0361
:1046B00030913D0340913E0350913F030E941C788E
:1046C0000E94EC77E0966CAF7DAF8EAF9FAFE09726
:1046D000F401608171818281938120914003309146
:1046E000410340914203509143030E941C780E9471
:1046F000EC77AC966CAF7DAF8EAF9FAFAC97D3012C
:104700006D917D918D919C91209144033091450351
:1047100040914603509147030E941C780E94EC7719
:10472000A8966CAF7DAF8EAF9FAFA897F201608166
:104730007181828193812091480330914903409196
:104740004A0350914B030E941C780E94EC77A49678
:104750006CAF7DAF8EAF9FAFA49780919403909183
:104760009503A0919603B0919703A4962CAD3DAD0F
:104770004EAD5FADA497281739074A075B0709F4C8
:104780005FC06091C709E62FF0E0EE0FFF1FEE510A
:10479000FD4F808191810E94671420E030E04AE261
:1047A00053E40E943C7588230CF04AC080916A084B
:1047B000882309F045C0A4964CAD5DAD6EAD7FADCC
:1047C000A49740939403509395036093960370933A
:1047D0009703E8E0F3E084918F017E010894E11CE7
:1047E000F11C0CC089838DEA9DE0B70141E050E0E7
:1047F0000E94196F0F5F1F4FF8018491882391F772
:10480000ECE2F3E084918F017E010894E11CF11C3D
:104810000CC089838DEA9DE0B70141E050E00E9421
:10482000196F0F5F1F4FF8018491882391F78AE079
:1048300089838DEA9DE0B70141E050E00E94196F45
:104840008091940390919503A0919603B091970362
:10485000A4962CAD3DAD4EAD5FADA497281B390B92
:104860004A0B5B0BCA01B90157FF07C090958095B1
:10487000709561957F4F8F4F9F4F0E94DE757B0132
:104880008C01609148037091490380914A03909193
:104890004B0320E030E04DEC53E40E941C789B0178
:1048A000AC01C801B7010E944A7718160CF045C048
:1048B000A4964CAD5DAD6EAD7FADA49740939403CF
:1048C000509395036093960370939703E8E0F3E0A9
:1048D00084918F017E010894E11CF11C0CC0898336
:1048E0008DEA9DE0B70141E050E00E94196F0F5F33
:1048F0001F4FF8018491882391F7EEE0F3E0849153
:104900008F017E010894E11CF11C0CC089838DEAA3
:104910009DE0B70141E050E00E94196F0F5F1F4F0B
:10492000F8018491882391F78AE089838DEA9DE0DC
:10493000B70141E050E00E94196F80916808282F6C
:1049400030E0A0963FAF2EAFA0978DE490E0289F77
:10495000F001299FF00D389FF00D1124E856FC4F0F
:10496000E45BFF4F1082EC54F0404091880350917B
:10497000890360918A0370918B036E964CAF5DAF93
:104980006EAF7FAF6E97E0968CAD9DADAEADBFAD17
:10499000E097841B950BA60BB70B6A968CAF9DAF67
:1049A000AEAFBFAF6A9780839183A283B383B7FF13
:1049B0000BC0B095A095909581959F4FAF4FBF4F7D
:1049C00080839183A283B38320918C0330918D03E4
:1049D00040918E0350918F0366962CAF3DAF4EAF42
:1049E0005FAF6697AC966CAD7DAD8EAD9FADAC976D
:1049F000621B730B840B950B62966CAF7DAF8EAF11
:104A00009FAF62978DE490E0A096AEADBFADA0974A
:104A1000A89FF001A99FF00DB89FF00D1124E85652
:104A2000FC4F62962CAD3DAD4EAD5FAD62972483D9
:104A300035834683578357FF0DC0DA01C901B0950E
:104A4000A095909581959F4FAF4FBF4F84839583DD
:104A5000A683B78340919003509191036091920394
:104A6000709193032E964CAF5DAF6EAF7FAF2E97D4
:104A7000A8968CAD9DADAEADBFADA897841B950B30
:104A8000A60BB70B2A968CAF9DAFAEAFBFAF2A97E0
:104A90008DE490E0A096AEADBFADA097A89FF001C9
:104AA000A99FF00DB89FF00D1124E856FC4F2A96EF
:104AB0002CAD3DAD4EAD5FAD2A9720873187428743
:104AC000538757FF0DC0DA01C901B095A0959095A5
:104AD00081959F4FAF4FBF4F80879187A287B38744
:104AE0002090940330909503409096035090970344
:104AF000A4964CAD5DAD6EAD7FADA4974219530940
:104B0000640975094AA75BA76CA77DA7E0914002DD
:104B1000F0914102CB01BA0197FF07C090958095B3
:104B2000709561957F4F8F4F9F4F9F01442737FDB1
:104B30004095542F0E94EE7824E630E040E050E0AB
:104B40000E9442798DE490E0A0966EAD7FADA09773
:104B5000689FF001699FF00D789FF00D1124E856D1
:104B6000FC4FDF011C96248711963C9311971296F7
:104B70004C93129713965C9360807180828093802F
:104B8000A480B580C680D780E084F1840285138537
:104B9000C901DA018E159F05A007B10714F4D801E9
:104BA000C7018A159B05AC05BD0514F4D601C501E6
:104BB0009C01AD0186159705A805B90514F4A4015B
:104BC00093018DE490E0A096AEADBFADA097A89FF5
:104BD000B001A99F700DB89F700D112468567C4FCD
:104BE000FB01208B318B428B538B263031054105E5
:104BF000510510F40C942F2FE85BFF4F8091C809EA
:104C000090E0A0E0B0E080839183A283B383DB01D6
:104C100090961C92E0962CAD3DAD4EAD5FADE09709
:104C20006E968CAD9DADAEADBFAD6E9728173907B2
:104C30004A075B0724F481E0DB0190968C93AC96E5
:104C40002CAD3DAD4EAD5FADAC9766966CAD7DAD18
:104C50008EAD9FAD6697261737074807590794F41E
:104C60008DE490E0A096AEADBFADA097A89FF001F7
:104C7000A99FF00DB89FF00D1124E856FC4F80A1BC
:104C8000826080A3A8962CAD3DAD4EAD5FADA897D8
:104C90002E966CAD7DAD8EAD9FAD2E972617370746
:104CA0004807590794F48DE490E0A096AEADBFADEF
:104CB000A097A89FF001A99FF00DB89FF00D1124B7
:104CC000E856FC4F80A1846080A3A4962CAD3DAD36
:104CD0004EAD5FADA497221533054405550594F4F8
:104CE0008DE490E0A0964EAD5FADA097489FF00197
:104CF000499FF00D589FF00D1124E856FC4F80A1FC
:104D0000886080A38DE490E0A0966EAD7FADA09703
:104D1000689FF001699FF00D789FF00D1124E8560F
:104D2000FC4FE296AEADBFADE2978C9181A320819E
:104D300031814281538126962CAF3DAF4EAF5FAF9C
:104D40002697211531054105510509F077988DE425
:104D500090E0A0964EAD5FADA097489FF001499FAF
:104D6000F00D589FF00D1124E856FC4F64817581B9
:104D70008681978122966CAF7DAF8EAF9FAF2297D1
:104D8000611571058105910509F076988DE490E033
:104D9000A096AEADBFADA097A89FF001A99FF00D62
:104DA000B89FF00D1124E856FC4F60847184828412
:104DB0009384611471048104910409F047988DE48F
:104DC00090E0A0962EAD3FADA097289FF001299FBF
:104DD000F00D389FF00D1124E856FC4F8485958521
:104DE000A685B7850097A105B10551F0439820909D
:104DF0005C0330905D0340905E0350905F0308C0F9
:104E000020907403309075034090760350907703A0
:104E1000CE57DF4F6881C258D040CD57DF4F7881E1
:104E2000C358D040CC57DF4F8881C458D040CB57AF
:104E3000DF4F9881C558D040A20191010E943C7576
:104E400087FD16C0CE57DF4F8881C258D040CD575E
:104E5000DF4F9881C358D040CC57DF4FA881C4584A
:104E6000D040CB57DF4FB881C558D0401C012D0131
:104E70008091680890916908482F50E0405F5F4F2B
:104E8000491B51094F7050705FA74EA7BA01882780
:104E900077FD8095982F0E94DE757B018C0120E0C4
:104EA00030E040E051E40E943C7588239CF46EA5FC
:104EB0007FA56230710574F0C201B101A8019701AC
:104EC0000E941C7820E030E040E05EE30E941C7805
:104ED0001B012C016A966CAD7DAD8EAD9FAD6A97BE
:104EE0000E94DE7520913C0330913D0340913E03CA
:104EF00050913F030E944375EB966FAFEB97EC9692
:104F00007FAFEC97ED968FAFED97EE969FAFEE9754
:104F1000AC01CB01DA018A839B83AC83BD836296AB
:104F20006CAD7DAD8EAD9FAD62970E94DE75209118
:104F300040033091410340914203509143030E944A
:104F40004375E7966FAFE797E8967FAFE897E996E6
:104F50008FAFE997EA969FAFEA97AC01CB01DA01F0
:104F60008E839F83A887B9872A966CAD7DAD8EAD61
:104F70009FAD2A970E94DE7520914403309145032E
:104F800040914603509147030E944375E3966FAFEB
:104F9000E397E4967FAFE497E5968FAFE597E696C3
:104FA0009FAFE697AC01CB01DA018A879B87AC877C
:104FB000BD87E0904002F09041026AA57BA58CA5D8
:104FC0009DA50E94DE7520914803309149034091D0
:104FD0004A0350914B030E9443755B016C0100270B
:104FE000F7FC0095102FC801B7010E94DE759B01E8
:104FF000AC01C601B5010E941C7820E030E048EC0D
:1050000052E40E9443757B018C016E877F87888BF9
:10501000998B26968CAD9DADAEADBFAD2697009712
:10502000A105B10591F522962CAD3DAD4EAD5FAD1C
:105030002297211531054105510539F56114710497
:105040008104910411F5C801B70120E030E040E08F
:1050500050E00E944A77181624F017FB109517F9B4
:1050600010958DE490E0A0964EAD5FADA097489F5F
:10507000F001499FF00D589FF00D1124E856FC4FA8
:10508000E6A6F7A600AB11AB55C0EB962FADEB979C
:10509000EC963FADEC97ED964FADED97EE965FAD8C
:1050A000EE97B901CA010E94D3783B014C01E79603
:1050B0002FADE797E8963FADE897E9964FADE997B2
:1050C000EA965FADEA97B901CA010E94D3785B0105
:1050D0006C01E3962FADE397E4963FADE497E59638
:1050E0004FADE597E6965FADE697B901CA010E941C
:1050F000D3787B018C01C401B301A60195010E9404
:105100006374A80197010E9463740E9489782DE45A
:1051100030E0A096AEADBFADA097A29FF001A39FD7
:10512000F00DB29FF00D1124E856FC4F66A777A74B
:1051300080AB91AB8DE490E0A096EEADFFADA09773
:10514000E89F6001E99FD00CF89FD00C112428E95A
:1051500033E0C20ED31ED6019E96ED90FD900D91C8
:105160001C91D19760E070E080E89FE3A80197016F
:105170000E9443759B01AC01C201B1010E941C78E1
:105180004B015C01C801B701A50194010E941C7884
:10519000F60162A373A384A395A3608971898289B0
:1051A00093890E94DC75A50194010E941C780E94DD
:1051B00029750E94B075D601D8966D937D938D9315
:1051C0009C93DB97EE24FF2442E1642E712C6C0E3D
:1051D0007D1E32E0C32ED12CCC0EDD1E83010E0DC0
:1051E0001F1DF601EE0DFF1D60817181828193818B
:1051F000A50194010E941C78F80160837183828369
:10520000938324E030E0E20EF31E30E1E316F10474
:1052100029F70F2EF0E06F2EF0E07F2EF0E88F2EB2
:10522000FFE39F2EF02D4424552422E1222E312C21
:105230002C0E3D1EF101E40DF51DE080F180028190
:105240001381C801B70120E030E040E050E00E9447
:105250004A7718161CF4C801B70103C0C801B7018A
:105260009058F201E45DFC4FA080B180C280D380F1
:10527000A60195010E944A77181694F5C801B70156
:1052800020E030E040E050E00E944A7718161CF41D
:10529000A801970103C0A80197015058C601B501A4
:1052A0000E9443759B01AC01C401B3010E943C758F
:1052B00087FD16C0C801B70120E030E040E050E0B3
:1052C0000E944A77181624F017FB109517F91095CD
:1052D000C601B501A80197010E9443753B014C012D
:1052E00044E050E0440E551E50E14516510409F0CB
:1052F000A1CFC401B30120E030E040E85FE30E94A9
:105300003C7588230CF0B2C04424552492E1292E28
:10531000312C2C0E3D1EF101E40DF51DE080F180D5
:1053200002811381C801B70120E030E040E050E085
:105330000E944A7718161CF4C801B70103C0C801BF
:10534000B7019058F201E45DFC4FA080B180C280AB
:10535000D380A60195010E944A77181694F5C801DA
:10536000B70120E030E040E050E00E944A77181694
:105370001CF4A801970103C0A80197015058C60169
:10538000B5010E9443759B01AC01C401B3010E94A9
:105390003C7587FD16C0C801B70120E030E040E051
:1053A00050E00E944A77181624F017FB109517F961
:1053B0001095C601B501A80197010E9443753B01F4
:1053C0004C0164E070E0460E571E70E14716510430
:1053D00009F0A1CF8E010E5E1F4F82E2E82EF12C64
:1053E000EC0EFD1ED8016D917D918D919C91A401D3
:1053F00093010E941C78F8016193719381939193BA
:105400008F01EE15FF0571F78DE490E0A0962EADAB
:105410003FADA097289F8001299F100D389F100D48
:10542000112408561C4FD80192966D917D918D9153
:105430009C919597A40193010E941C78F80162A3A6
:1054400073A384A395A360AD71AD82AD93AD0E94AB
:10545000DC75A40193010E941C780E94B075D801EC
:10546000D8966D937D938D939C93DB978DE490E01C
:10547000A096EEADFFADA097E89F8001E99F100DCB
:10548000F89F100D112408561C4FD80150966D91AD
:105490007D918D919C9153970E94DC75F80126A512
:1054A00037A540A951A90E9443751B012C01F801A1
:1054B00080819181A281B3810097A105B10549F551
:1054C00084819581A681B7810097A105B10509F571
:1054D00080859185A285B3850097A105B105C9F4A2
:1054E000C201B101209164033091650340916603CC
:1054F000509167030E941C780E9429750C5B1F4F16
:105500000E94B075D8016D937D938D939C931397F2
:1055100071C1C201B10120916003309161034091DA
:105520006203509163030E941C780E9429750E94B7
:10553000B0752DE430E0A096EEADFFADA097E29FF0
:105540006001E39FD00CF29FD00C112428E933E0D6
:10555000C20ED31EB4E46B2E712C6C0C7D1CD301D7
:105560006D937D938D939C93139780907803909087
:105570007903A0907A03B0907B030E94DC757B01D5
:105580008C01F60160817181828193810E94DE75B8
:105590009B01AC01C801B7010E941C787B018C0102
:1055A000D60150966D917D918D919C9153970E945B
:1055B000DC759B01AC01C801B7010E9443757B01FA
:1055C0008C01C501B4010E94DC759B01AC01C801CE
:1055D000B7010E944A7718162CF4F3018082918259
:1055E000A282B38280907C0390907D03A0907E0382
:1055F000B0907F038DE490E0A0962EAD3FADA097D4
:10560000289F6001299FD00C389FD00C112448E9B5
:1056100053E0C40ED51EA4E46A2E712C6C0C7D1CC4
:10562000D3016D917D918D919C910E94DC757B01E0
:105630008C01F60164817581868197810E94DE75F7
:105640009B01AC01C801B7010E941C787B018C0151
:10565000D60150966D917D918D919C9153970E94AA
:10566000DC759B01AC01C801B7010E9443757B0149
:105670008C01C501B4010E94DC759B01AC01C8011D
:10568000B7010E944A7718162CF4F30180829182A8
:10569000A282B3828090840390908503A0908603B9
:1056A000B09087038DE490E0A0962EAD3FADA0971B
:1056B000289F6001299FD00C389FD00C112448E905
:1056C00053E0C40ED51EF4E46F2E712C6C0C7D1CBF
:1056D000D3016D917D918D919C910E94DC757B0130
:1056E0008C01F60164857585868597850E94DE7537
:1056F0009B01AC01C801B7010E941C787B018C01A1
:10570000D60150966D917D918D919C9153970E94F9
:10571000DC759B01AC01C801B7010E9443757B0198
:105720008C01C501B4010E94DC759B01AC01C8016C
:10573000B7010E944A7718162CF4F30180829182F7
:10574000A282B3828090800390908103A090820314
:10575000B09083038DE490E0A0962EAD3FADA0976E
:10576000289F6001299FD00C389FD00C112448E954
:1057700053E0C40ED51EE4E46E2E712C6C0C7D1C1F
:10578000D3016D917D918D919C910E94DC757B017F
:105790008C01F60160857185828593850E94DE7596
:1057A0009B01AC01C801B7010E941C787B018C01F0
:1057B000D60150966D917D918D919C9153970E9449
:1057C000DC759B01AC01C801B7010E9443757B01E8
:1057D0008C01C501B4010E94DC759B01AC01C801BC
:1057E000B7010E944A7718162CF4F3018082918247
:1057F000A282B3828DE490E0A0962EAD3FADA0973B
:10580000289F6001299FD00C389FD00C112448E9B3
:1058100053E0C40ED51EF601EC5BFF4F6081718131
:10582000828193810E94DC757B018C01A201910130
:105830000E944375D601D2966D937D938D939C9370
:10584000D597C801B7012DEB37E346E051E40E943C
:105850001C780E94AB75F601648F758F868F978FC9
:10586000209168033091690340916A0350916B0362
:105870002AAF3BAF4CAF5DAF4A8D5B8D6C8D7D8D9C
:105880004EA35FA368A779A7CB01BA0120E030E05F
:1058900040E050E00E944A7718162CF4EEA0FFA0DA
:1058A00008A519A508C0EEA0FFA008A519A517FB1B
:1058B000109517F9109560916C0370916D038091AC
:1058C0006E0390916F036EAB7FAB88AF99AF20E012
:1058D00030E040E05FE30E941C785B016C01C8018E
:1058E000B701A60195010E944A77181664F06AADC7
:1058F0007BAD8CAD9DAD20E030E040E05FE30E94E9
:105900001C785B016C018DE490E0A096AEADBFAD5C
:10591000A097A89FF001A99FF00DB89FF00D11244A
:10592000E856FC4FB2A1EF96BFAFEF9723A1C15845
:10593000DF4F2883CF57D04034A1C058DF4F388382
:10594000C058D04045A1CF57DF4F4883C158D04001
:10595000C601B5012B2FC158DF4F3881CF57D0403A
:10596000C058DF4F4881C058D040CF57DF4F5881D3
:10597000C158D0400E943C7587FD14C0EF968FAD92
:10598000EF97C158DF4F9881CF57D040C058DF4FB5
:10599000A881C058D040CF57DF4FB881C158D04000
:1059A0005C016D016E8D7F8D88A199A16AA37BA397
:1059B0008CA39DA320E030E040E050E00E944A77B5
:1059C00018162CF4EAA0FBA00CA11DA108C0EAA0A7
:1059D000FBA00CA11DA117FB109517F91095809144
:1059E000700390917103A0917203B09173038AAB1D
:1059F0009BABACABBDABBC01CD0120E030E040E0E7
:105A00005FE30E941C783B014C01C801B701A4016F
:105A100093010E944A77181644F4C601B501A40107
:105A200093010E943C75882314F435014601AEA50C
:105A3000BFA512970CF40FC160916B0870916C08B0
:105A400080916D0890916E0820E030E040E050E0D9
:105A50000E944A7718160CF0FEC0A0906F08B09014
:105A60007008C0907108D09072086A897B898C890F
:105A70009D89A60195010E9462749B01AC010E9460
:105A80001C787B018C012090730830907408409042
:105A90007508509076086E897F89888D998DA2014E
:105AA00091010E9462749B01AC010E941C789B01D1
:105AB000AC01C801B7010E9463740E9489787B0120
:105AC0008C01C601B50120E030E040E050E00E94CA
:105AD0003C75882351F4C201B10120E030E040E080
:105AE00050E00E943C758823A1F0EF968FADEF97B0
:105AF000C158DF4F9881CF57D040C058DF4FA881A1
:105B0000C058D040CF57DF4FB881C158D0403C017A
:105B10004D01C801B7012AAD3BAD4CAD5DAD0E9452
:105B20004A77181684F46AAD7BAD8CAD9DADA801A3
:105B300097010E9443759B01AC01C401B3010E940F
:105B40001C783B014C016EA17FA188A599A52091ED
:105B50007708309178084091790850917A080E942E
:105B600062747B018C0120E030E040E050E00E9454
:105B70004A7718161CF4C801B70103C0C801B70161
:105B800090582EA93FA948AD59AD0E944A771816E2
:105B9000F4F4C801B70120E030E040E050E00E949A
:105BA0004A77181624F017FB109517F910956EA96F
:105BB0007FA988AD99ADA80197010E9443759B010B
:105BC000AC01C401B3010E941C783B014C016AA1E5
:105BD0007BA18CA19DA120917B0830917C084091F4
:105BE0007D0850917E080E9462747B018C0120E048
:105BF00030E040E050E00E944A7718161CF4C801DB
:105C0000B70103C0C801B70190582AA93BA94CA904
:105C10005DA90E944A771816F4F4C801B70120E084
:105C200030E040E050E00E944A77181624F017FB5D
:105C3000109517F910956AA97BA98CA99DA9A801AF
:105C400097010E9443759B01AC01C401B3010E94FE
:105C50001C783B014C018DE490E0A096EEADFFADC9
:105C6000A097E89F8001E99F100DF89F100D112467
:105C700008561C4FD8019A966D927D928D929C92F7
:105C80009D97D2966D917D918D919C91D5979058CD
:105C900020E030E040E050EC0E941C78F80126A59E
:105CA00037A540A951A90E941C7820E030E040E8C7
:105CB00050E40E9463740E948978F62EE72ED82E55
:105CC000C92EC401B3012F2D3E2D4D2D5C2D0E94F8
:105CD0003C7587FD06C08F2D9E2DAD2DBC2D3C0142
:105CE0004D018DE490E0A0962EAD3FADA097289F8A
:105CF0008001299F100D389F100D112408561C4F4C
:105D0000D80196966D927D928D929C9299979296DB
:105D10006D917D918D919C9195972F2D3E2D4D2DBF
:105D20005C2D0E943C75181624F081E0F80187ABC9
:105D300003C0D801D7961C928DE490E0A0962EADBA
:105D40003FADA097289FF001299FF00D389FF00DDF
:105D50001124E856FC4F81E086ABAFE6B8E0FE01C7
:105D6000729680E101900D928150E1F78DE490E010
:105D7000A0964EAD5FADA097489F6001499FD00CA3
:105D8000589FD00C112468E973E0C60ED71ED601C7
:105D90009296ED90FD900D911C919597E0926B0875
:105DA000F0926C0800936D0810936E0896966D91B2
:105DB0007D918D919C919997A80197010E944375BF
:105DC0004B015C0160E070E080E090E4A801970185
:105DD0000E9443758B019C01C601B501A4010E947C
:105DE0007520B8A9B0936808A4962CAD3DAD4EAD12
:105DF0005FADA4972093940330939503409396034B
:105E000050939703A8964CAD5DAD6EAD7FADA8974E
:105E10004093900350939103609392037093930384
:105E2000AC966CAD7DAD8EAD9FADAC9760938C03A1
:105E300070938D0380938E0390938F03E0968CADC7
:105E40009DADAEADBFADE09780938803909389037D
:105E5000A0938A03B0938B030E94FD2224D0CB57DA
:105E6000DF4F0FB6F894DEBF0FBECDBFCF91DF91ED
:105E70001F910F91FF90EF90DF90CF90BF90AF9068
:105E80009F908F907F906F905F904F903F902F905A
:105E900008951092B3081092B5081092B7080895AB
:105EA00080932D020895EFE6F0E080818260808388
:105EB0000895099A0B9A0D9A0F9A6F9A779A6E9A8B
:105EC000769A3F9A479A3B9A439A6B98739A20988E
:105ED000289A6C98749A089A779A0A9A769A0C9AE1
:105EE000479A0E9A439AA1E8B0E08C918F7E8C93EA
:105EF0008C9188608C93E0E8F0E080818D7F8083D6
:105F000080818E7F808380818F73808380818F7C6E
:105F100080838C91887F82608C9380E090E4909362
:105F20008900809388001092850010928400EFE62B
:105F3000F0E080818260808310922D027894089531
:105F40001F93FC011FB7F89480819181A281B381D6
:105F500080938D0890938E08A0938F08B09390083B
:105F6000FB0180819181A281B381809391089093FC
:105F70009208A0939308B0939408FA0180819181CC
:105F8000A281B3818093950890939608A093970877
:105F9000B0939808F90180819181A281B3818093A7
:105FA000990890939A08A0939B08B0939C081FBFF0
:105FB0001F910895FC012FB7F89480819181A281EF
:105FC000B3818093990890939A08A0939B08B0930B
:105FD0009C082FBF0895E82F8FB7F894F0E0EE0FDC
:105FE000FF1FEE0FFF1FE357F74F208131814281E2
:105FF00053818FBFB901CA01089580916F008D7FD1
:1060000080936F0006C0809169088F5F8F708093C6
:1060100069089091680880916908981751F4109266
:10602000800810927F0880916F00826080936F00DB
:1060300008959091680880916908981751F3E3CF0B
:106040009091680880916908981731F00E9488152E
:1060500081E00E944039F4CF0895F2DF779A769A72
:10606000479A439A0895CF93DF93DB010D90002068
:10607000E9F71197A61BB70BEC01E881F9810280C3
:10608000F381E02DAD010995DF91CF9108951F9225
:106090000F920FB60F920BB60F921124AF92BF92D0
:1060A000CF92DF92EF92FF920F931F932F933F9324
:1060B0004F935F936F937F938F939F93AF93BF9310
:1060C000CF93DF93EF93FF9380917F0890918008A7
:1060D000892B09F089C19091680880916908981707
:1060E00019F4E0E0F0E014C08091690890E02DE43C
:1060F00030E0829FF001839FF00D929FF00D1124FC
:10610000E856FC4FE45BFF4F81E08083EC54F040A5
:10611000F0938008E0937F08309709F45FC11092F4
:10612000BF081092C0081092C1081092C20844AD76
:1061300055AD5093BE084093BD082CE94134520739
:1061400018F040E45CE904C03EE44132530730F00B
:10615000569547955695479584E007C067E24131CB
:10616000560730F05695479582E08093B80808C0EE
:1061700081E08093B8084032510510F440E250E0CD
:106180008A010052104078E000301707E8F0412FF4
:1061900050E0440F551F440F551F4A5B5C4F9A0156
:1061A0002E5F3F4FF901859194919C01AA27039F8F
:1061B000C001029F810D9A1F06948A1F9A1F112405
:1061C000FA01459154911EC0C801969587958C7F20
:1061D0008A5B984FFC0145915491FC0132962591C0
:1061E0003491802F90E087709070BC01269FC00191
:1061F000279F900D369F900D1124F3E0969587957B
:10620000FA95E1F7481B590B44365105A0F48DEA85
:106210009DE063E171E027DFA80160E070E08DEAB6
:106220009DE02AE000E00E94E6708DEA9DE00E9479
:10623000CA7044E650E0CA01A0E0B0E08093B9081B
:106240009093BA08A093BB08B093BC085093890000
:1062500040938800E0917F08F091800840AD51ADF7
:106260007CE94134570718F040E45CE904C08EE44F
:106270004132580730F0569547955695479584E03A
:1062800007C097E24131590730F05695479582E0B3
:106290008093B80808C081E08093B8084032510567
:1062A00010F440E250E08A0100521040E8E0003073
:1062B0001E07E8F0412F50E0440F551F440F551FB3
:1062C0004A5B5C4F9A012E5F3F4FF9018591949193
:1062D0009C01AA27039FC001029F810D9A1F06946B
:1062E0008A1F9A1F1124FA01459154911EC0C801BA
:1062F000969587958C7F8A5B984FFC0145915491C8
:10630000FC01329625913491802F90E08770907037
:10631000BC01269FC001279F900D369F900D112430
:1063200033E0969587953A95E1F7481B590B44362B
:106330005105A0F48DEA9DE063E171E094DEA801CF
:1063400060E070E08DEA9DE02AE000E00E94E670E7
:106350008DEA9DE00E94CA7044E650E05093C40864
:106360004093C308E0917F08F0918008808991896B
:10637000A289B389B695A79597958795B095A0956D
:10638000909581959F4FAF4FBF4F80939D089093FD
:106390009E08A0939F08B093A0088093A1089093B3
:1063A000A208A093A308B093A4088093A508909393
:1063B000A608A093A708B093A8088093A908909373
:1063C000AA08A093AB08B093AC081092AD08109245
:1063D000AE081092AF081092B00806C080ED97E0AA
:1063E0009093890080938800E0917F08F091800865
:1063F000309709F45FC580A18093B10880FF3FC04A
:106400008FEF8093290280912D028823D9F18CB1DE
:106410008695869586958095282F217080FF2CC0C3
:106420008091B208882341F180819181A281B3815A
:10643000181619061A061B06FCF480918D08909117
:106440008E08A0918F08B091900880938108909356
:106450008208A0938308B093840881E08093B308F6
:1064600080899189A289B3898093AD089093AE0801
:10647000A093AF08B093B0082093B20803C081E0A6
:10648000809329028091B10881FF3AC08FEF8093F9
:106490002A0280912D028823B1F123B1217031E0CD
:1064A000232759F18091B408882339F1848195819B
:1064B000A681B781181619061A061B06F4F48091F6
:1064C000910890919208A0919308B09194088093BC
:1064D000850890938608A0938708B0938808309326
:1064E000B50880899189A289B3898093AD0890937A
:1064F000AE08A093AF08B093B0082093B40803C0CF
:1065000081E080932A0220813181428153818481FC
:106510009581A681B781281739074A075B0744F0A0
:106520008091B10880FD02C0119A0FC011980AC075
:10653000281739074A075B074CF48091B10881FDA1
:1065400003C0119A139802C01198139A8091B10850
:1065500082FF3FC0159A8FEF80932B0280912D020E
:106560008823D9F18CB182958F708095282F217066
:1065700080FF2CC08091B608882341F180859185E9
:10658000A285B385181619061A061B06FCF480911D
:10659000950890919608A0919708B09198088093DB
:1065A000890890938A08A0938B08B0938C0881E0A7
:1065B0008093B70880899189A289B3898093AD08B7
:1065C0009093AE08A093AF08B093B0082093B6089C
:1065D00004C0159881E080932B028091B10883FF5D
:1065E00003C017988FEF02C0179A81E080932C02A6
:1065F00060E043C220919D0830919E0840919F0821
:106600005091A00880819181A281B381280F391F08
:106610004A1F5B1F20939D0830939E0840939F085C
:106620005093A008E480F580068117818091A1082D
:106630009091A208A091A308B091A408E80EF91EB9
:106640000A1F1B1FE092A108F092A2080093A30862
:106650001093A4081216130614061506A4F51E14AA
:106660001F04100611067CF1109A129A80899189F4
:10667000A289B389281B390B4A0B5B0B20939D0819
:1066800030939E0840939F085093A008109812984A
:1066900020918D0830918E0840918F08509190087C
:1066A00080912902992787FD9095A92FB92F820FF4
:1066B000931FA41FB51F80938D0890938E08A093FD
:1066C0008F08B093900880919D0890919E08A091AA
:1066D0009F08B091A008181619061A061B06E4F1C7
:1066E0002091A1083091A2084091A3085091A408DC
:1066F00012161306140615067CF5109A129A808954
:106700009189A289B389281B390B4A0B5B0B209313
:10671000A1083093A2084093A3085093A4081098AE
:1067200012982091910830919208409193085091CD
:10673000940880912A02992787FD9095A92FB92F57
:10674000820F931FA41FB51F809391089093920806
:10675000A0939308B093940820919D0830919E08CF
:1067600040919F085091A0081216130614061506B2
:106770000CF0CAC0E090A108F090A2080091A30814
:106780001091A4081E141F04100611060CF0BCC0C2
:106790009091B108892F8695892780FF5BC0129A56
:1067A00080899189A289B389281B390B4A0B5B0B1D
:1067B00020939D0830939E0840939F085093A00813
:1067C000129820918D0830918E0840918F08509139
:1067D000900880912902992787FD9095A92FB92FBC
:1067E000820F931FA41FB51F80938D0890938E086E
:1067F000A0938F08B093900820919108309192084F
:10680000409193085091940880912A02992787FD1E
:106810009095A92FB92F820F931FA41FB51F8093A6
:10682000910890939208A0939308B0939408129AB9
:1068300080899189A289B389E81AF90A0A0B1B0B8E
:10684000E092A108F092A2080093A3081093A40874
:1068500012985AC0109A80899189A289B389281BFD
:10686000390B4A0B5B0B20939D0830939E08409395
:106870009F085093A008109820918D0830918E08A1
:1068800040918F085091900880912902992787FDA7
:106890009095A92FB92F820F931FA41FB51F809326
:1068A0008D0890938E08A0938F08B0939008209144
:1068B00091083091920840919308509194088091EA
:1068C0002A02992787FD9095A92FB92F820F931F30
:1068D000A41FB51F8093910890939208A0939308EA
:1068E000B0939408109A80899189A289B389E81A93
:1068F000F90A0A0B1B0BE092A108F092A208009380
:10690000A3081093A40810982085318542855385EB
:106910008091A5089091A608A091A708B091A80819
:10692000280F391F4A1F5B1F2093A5083093A60824
:106930004093A7085093A8081216130614061506CC
:106940006CF5149A80899189A289B389281B390B27
:106950004A0B5B0B2093A5083093A6084093A70829
:106960005093A8081498209195083091960840916A
:1069700097085091980880912B02992787FD909550
:10698000A92FB92F820F931FA41FB51F80939508BD
:1069900090939608A0939708B0939808248535851E
:1069A000468557858091A9089091AA08A091AB08C7
:1069B000B091AC08280F391F4A1F5B1F2093A9080C
:1069C0003093AA084093AB085093AC0812161306F4
:1069D000140615066CF5169A80899189A289B389E7
:1069E000281B390B4A0B5B0B2093A9083093AA088C
:1069F0004093AB085093AC081698209199083091B9
:106A00009A0840919B0850919C0880912C029927EC
:106A100087FD9095A92FB92F820F931FA41FB51F33
:106A20008093990890939A08A0939B08B0939C0830
:106A30008091AD089091AE08A091AF08B091B008D8
:106A40000196A11DB11D8093AD089093AE08A0934F
:106A5000AF08B093B0082091AD083091AE084091D6
:106A6000AF085091B00880899189A289B38928170D
:106A700039074A075B0730F46F5F8091B8086817E1
:106A80000CF4B8CD2091AD083091AE084091AF081C
:106A90005091B00884899589A689B7898217930790
:106AA000A407B50708F4E3C0E090B908F090BA086D
:106AB0000091BB081091BC08A48CB58CC68CD78CF7
:106AC000A8019701C601B501AA27279FB12D389FBC
:106AD000E001489FD00D479FC00DD11D289FB00DEC
:106AE000C11DDA1F379FB00DC11DDA1F469FB00DC3
:106AF000C11DDA1F369FB10DCA1FDA1FB695CA1F16
:106B0000DA1F112484AD95AD8C0F9D1F9093BE08A4
:106B10008093BD0820AD31AD42AD53ADA0E0B0E0F3
:106B2000281739074A075B0720F43093BE082093E3
:106B3000BD084091BD085091BE087CE9413457071B
:106B400018F040E45CE904C08EE44132580730F0AC
:106B5000569547955695479584E007C097E2413191
:106B6000590730F05695479582E08093B80808C0E1
:106B700081E08093B8084032510510F440E250E0C3
:106B80008A0100521040E8E000301E07E8F0412F73
:106B900050E0440F551F440F551F4A5B5C4F9A014C
:106BA0002E5F3F4FF901859194919C01AA27039F85
:106BB000C001029F810D9A1F06948A1F9A1F1124FB
:106BC000FA01459154911EC0C801969587958C7F16
:106BD0008A5B984FFC0145915491FC0132962591B6
:106BE0003491802F90E087709070BC01269FC00187
:106BF000279F900D369F900D1124F3E09695879571
:106C0000FA95E1F7481B590B44365105A0F48DEA7B
:106C10009DE063E171E027DAA80160E070E08DEAB1
:106C20009DE02AE000E00E94E6708DEA9DE00E946F
:106C3000CA7044E650E050938900409388009A015E
:106C400040E050E08091B9089091BA08A091BB084B
:106C5000B091BC08820F931FA41FB51F8093B90881
:106C60009093BA08A093BB08B093BC08FEC02091D3
:106C7000AD083091AE084091AF085091B008808DBA
:106C8000918DA28DB38D82179307A407B50708F0E5
:106C9000E4C06091BF087091C0088091C1089091D4
:106CA000C208248D358D468D578DAA27639FB12D3F
:106CB000749F8001849F100D839F000D111D649FA0
:106CC000B00D011D1A1F739FB00D011D1A1F829F69
:106CD000B00D011D1A1F729FB10D0A1F1A1FB69524
:106CE0000A1F1A1F11248091BD089091BE088017B9
:106CF000910738F4E05CFF4F40815181E054F0404F
:106D000003C0AC01401B510BE05CFF4F00811181BF
:106D100022813381CA01A0E0B0E080179107A20769
:106D2000B30708F4A8017CE94134570718F040E4A0
:106D30005CE904C08EE44132580730F0569547951F
:106D40005695479584E007C097E24131590730F0E6
:106D50005695479582E08093B80808C081E08093FB
:106D6000B8084032510510F440E250E08A01005268
:106D70001040E8E000301E07E8F0412F50E0440FDB
:106D8000551F440F551F4A5B5C4F9A012E5F3F4FC2
:106D9000F901859194919C01AA27039FC001029F4C
:106DA000810D9A1F06948A1F9A1F1124FA0145919A
:106DB00054911EC0C801969587958C7F8A5B984F29
:106DC000FC0145915491FC01329625913491802F1C
:106DD00090E087709070BC01269FC001279F900DA6
:106DE000369F900D112423E0969587952A95E1F71B
:106DF000481B590B44365105A0F48DEA9DE063E130
:106E000071E031D9A80160E070E08DEA9DE02AE0F0
:106E100000E00E94E6708DEA9DE00E94CA7044E6A0
:106E200050E050938900409388009A0140E050E080
:106E30008091BF089091C008A091C108B091C2088C
:106E4000820F931FA41FB51F8093BF089093C008A3
:106E5000A093C108B093C20808C08091C308909164
:106E6000C40890938900809388002091AD083091E8
:106E7000AE084091AF085091B008E0917F08F091C2
:106E8000800880899189A289B389281739074A0720
:106E90005B0780F01092800810927F08909168083C
:106EA00080916908981731F0809169088F5F8F7021
:106EB00080936908FF91EF91DF91CF91BF91AF91DE
:106EC0009F918F917F916F915F914F913F912F9102
:106ED0001F910F91FF90EF90DF90CF90BF90AF90F8
:106EE0000F900BBE0F900FBE0F901F901895EF9252
:106EF000FF920F931F93DF93CF930F92CDB7DEB71F
:106F00008091B308882349F48091B508882329F437
:106F10008091B708882309F4E7C0E6E4FBE0849198
:106F20008F017E010894E11CF11C0CC089838DEA5D
:106F30009DE0B70141E050E00E94196F0F5F1F4FC5
:106F4000F8018491882391F7E8E5FBE084918F01B3
:106F50007E010894E11CF11C0CC089838DEA9DE040
:106F6000B70141E050E00E94196F0F5F1F4FF80119
:106F70008491882391F78091B308882391F1E4E507
:106F8000FBE084918F017E010894E11CF11C0CC090
:106F900089838DEA9DE0B70141E050E00E94196FBE
:106FA0000F5F1F4FF8018491882391F7609181084A
:106FB0007091820880918308909184080E94DE7508
:106FC00020913C0330913D0340913E0350913F039B
:106FD0000E944375AB01BC018DEA9DE022E00E9456
:106FE00082718091B508882391F1E0E5FBE08491FE
:106FF0008F017E010894E11CF11C0CC089838DEA8D
:107000009DE0B70141E050E00E94196F0F5F1F4FF4
:10701000F8018491882391F7609185087091860822
:1070200080918708909188080E94DE752091400326
:107030003091410340914203509143030E944375B4
:10704000AB01BC018DEA9DE022E00E94827180913B
:10705000B708882391F1ECE4FBE084918F017E0175
:107060000894E11CF11C0CC089838DEA9DE0B701F6
:1070700041E050E00E94196F0F5F1F4FF8018491AB
:10708000882391F76091890870918A0880918B0814
:1070900090918C080E94DE75209144033091450345
:1070A00040914603509147030E944375AB01BC01D8
:1070B0008DEA9DE022E00E9482718DEA9DE067E208
:1070C00071E00E9433308AE089838DEA9DE0BE0141
:1070D0006F5F7F4F41E050E00E94196F1092B3083C
:1070E0001092B5081092B7080F90CF91DF911F91C1
:1070F0000F91FF90EF900895CF93DF930FB6F89420
:107100008091A80D9091A90DA091AA0DB091AB0D01
:107110000FBE8093C9099093CA09A093CB09B0937D
:10712000CC09E091F209F091F309EC50F64F80811F
:10713000882399F4EFE8FBE06491EF0107C08DEA42
:107140009DE00E94E3112196FE0164916623B9F748
:107150008DEA9DE06AE00E94E311DF91CF910895EE
:107160008130910541F46F5F7F4F09F051C085EC8C
:1071700098E00C944F5C892B09F04AC06F5F7F4FF9
:1071800009F046C08AEC92E09093740980937309E9
:1071900080917909882321F086E799E00E94D454F0
:1071A0008AEC92E0909333098093320980913809F8
:1071B000882321F085E399E00E94D4548AEC92E080
:1071C000909315098093140980911A09882321F05E
:1071D00087E199E00E94D4548AEC92E09093F708FA
:1071E0008093F6088091FC08882321F089EF98E0CD
:1071F0000E94D4548AEC92E09093D7088093D608EA
:107200008091DC08882321F089ED98E00C94D45417
:10721000089580E090E06FEF7FEFA2CF81E090E0F3
:107220006FEF7FEF9DCFCF93DF93E7E6FBE06491B5
:10723000EF0107C08DEA9DE00E94E3112196FE0157
:1072400064916623B9F7EEE6FBE06491EF0107C0B5
:107250008DEA9DE00E94E3112196FE016491662370
:10726000B9F78DEA9DE06AE00E94E3110E940318DD
:10727000779A769A479A439AF894DF91CF91089536
:10728000EF92FF920F931F930FB6F8948091A80D81
:107290009091A90DA091AA0DB091AB0D0FBEE090F9
:1072A000CD09F090CE090091CF091091D00920911D
:1072B000C9093091CA094091CB095091CC09821B70
:1072C000930BA40BB50BE816F9060A071B0730F45D
:1072D000E114F1040105110509F0A5DFE090420277
:1072E000F09043020091440210914502E114F10430
:1072F0000105110531F10FB6F8948091A80D909118
:10730000A90DA091AA0DB091AB0D0FBE2091C90996
:107310003091CA094091CB095091CC09821B930B43
:10732000A40BB50BE816F9060A071B0750F4909159
:10733000680880916908981721F4779A769A479A95
:10734000439A0E94951D1F910F91FF90EF90089511
:107350006F927F928F929F92AF92BF92CF92DF9265
:10736000EF92FF920F931F93F82E6091D1097091C5
:10737000D2098091D3099091D4092091D5093091F7
:10738000D6094091D7095091D8090E9457773B01FF
:107390004C0160913E0270913F0200D000D000D0BD
:1073A0000DB71EB70F5F1F4F882777FD8095982F69
:1073B0000E94DE75209146023091470240914802BA
:1073C000509149020E941C7820E030E040E752E4EE
:1073D0000E94437520E030E048EC52E40E9443757F
:1073E0005B016C01F8016082718282829382F48277
:1073F0008091C70985838BEA99E06DED79E041EDD5
:1074000059E020E001E032E0E32E0E94750E809109
:10741000DD099091DE09A091DF09B091E009809328
:10742000AB099093AC09A093AD09B093AE098091DC
:10743000E1099091E209A091E309B091E4098093F8
:10744000AF099093B009A093B109B093B2098091AC
:10745000E5099091E609A091E709B091E8098093C8
:10746000B3099093B409A093B509B093B60980917C
:10747000E9099091EA09A091EB09B091EC09809398
:10748000B7099093B809A093B909B093BA090FB698
:10749000F8948091A80D9091A90DA091AA0DB0919A
:1074A000AB0D0FBE8093C9099093CA09A093CB0975
:1074B000B093CC098DB79EB706960FB6F8949EBFD1
:1074C0000FBE8DBF1F910F91FF90EF90DF90CF9077
:1074D000BF90AF909F908F907F906F9008958F9204
:1074E0009F92AF92BF92CF92DF92EF92FF920F9353
:1074F0001F930FB6F8948091A80D9091A90DA091BB
:10750000AA0DB091AB0D0FBE8093C9099093CA0923
:10751000A093CB09B093CC0960913E0270913F02D9
:10752000BDEDCB2EB9E0DB2EA8E0AA2EB12CAC0C21
:10753000BD1CFCE08F2E912C8C0C9D1C882777FDA8
:107540008095982F0E94DE75209146023091470267
:1075500040914802509149020E941C7820E030E09E
:1075600040E752E40E94437520E030E048EC52E4EA
:107570000E9443757B018C01C60124E030E0C20EFD
:10758000D31EB601A5019401E7ECCE2EE9E0DE2E74
:107590000E9400238091DD099091DE09A091DF090E
:1075A000B091E0098093AB099093AC09A093AD0929
:1075B000B093AE098091E1099091E209A091E309AD
:1075C000B091E4098093AF099093B009A093B109F9
:1075D000B093B2098091E5099091E609A091E7097D
:1075E000B091E8098093B3099093B409A093B509C9
:1075F000B093B6098091E9099091EA09A091EB094D
:10760000B091EC098093B7099093B809A093B90998
:10761000B093BA091F910F91FF90EF90DF90CF9038
:10762000BF90AF909F908F900895CF93DF938DEA96
:107630009DE00E94016FE2E9FBE06491EF0107C069
:107640008DEA9DE00E94E3112196FE01649166237C
:10765000B9F74091F8095091F9096091FA097091D0
:10766000FB094F5F5F4F6F4F7F4F8DEA9DE00E9498
:1076700071718DEA9DE06AE00E94E3113DDDDF91CA
:10768000CF9108954091F2095091F30920E630E03E
:10769000B901469F9001479F300D569F300D112430
:1076A000682F772767FD7095C9018A5F954F0E9403
:1076B000990B9C019093010A8093000A80E0232B90
:1076C00009F081E008950F931F93DF93CF93CDB717
:1076D000DEB7E0970FB6F894DEBF0FBECDBFDE0178
:1076E0001196E6EBF2E080E101900D928150E1F716
:1076F000DE015196E6EAF2E080E101900D928150C0
:10770000E1F7DE019196E6E9F2E080E101900D9269
:107710008150E1F789819A81AB81BC8180933C03E0
:1077200090933D03A0933E03B0933F0389899A89C8
:10773000AB89BC8980932C0390932D03A0932E03D7
:10774000B0932F0389A19AA1ABA1BCA180934C0354
:1077500090934D03A0934E03B0934F038D819E8170
:10776000AF81B8858093400390934103A093420377
:10777000B09343038D899E89AF89B88D8093300380
:1077800090933103A0933203B09333038DA19EA154
:10779000AFA1B8A58093500390935103A0935203D7
:1077A000B093530389859A85AB85BC858093440348
:1077B00090934503A0934603B0934703898D9A8D18
:1077C000AB8DBC8D8093340390933503A093360327
:1077D000B093370389A59AA5ABA5BCA580935403A4
:1077E00090935503A0935603B09357038D859E85C0
:1077F000AF85B8898093480390934903A0934A03C7
:10780000B0934B038D8D9E8DAF8DB8A180933803BF
:1078100090933903A0933A03B0933B038DA59EA5A3
:10782000AFA5B8A98093580390935903A0935A0326
:10783000B0935B0380E090E8ABE3B5E48093600332
:1078400090936103A0936203B093630380936403F6
:1078500090936503A0936603B093670320E030E044
:1078600040E050E020935C0330935D0340935E035F
:1078700050935F0380E29EE4A0E0B0E08093280391
:1078800090932903A0932A03B0932B0320937403AE
:1078900030937503409376035093770380E090E034
:1078A000A0EAB1E48093680390936903A0936A030C
:1078B000B0936B038DEC9CECACECBEE380936C035B
:1078C00090936D03A0936E03B0936F0380E090E0FC
:1078D000A0EAB0E48093700390937103A0937203C5
:1078E000B0937303EAE9FBE064918F0108C08DEA6D
:1078F0009DE00E94E3110F5F1F4FF8016491662322
:10790000B1F78DEA9DE068E271E00E9433308DEAC4
:107910009DE06AE00E94E311E0960FB6F894DEBFA6
:107920000FBECDBFCF91DF911F910F910895809130
:10793000000A9091010A019660E070E04AE050E090
:107940000C94310A8091000A9091010A019660E03E
:1079500070E00C94D408AF92BF92CF92DF92EF9276
:10796000FF920F931F93CF93DF931BEAE12E19E051
:10797000F12ECDEDD9E000E010E0F801E85AFD4F1E
:10798000808180DE882331F1DDDF5B016C01F8014D
:10799000EC55F64F8081882311F061E002C06091C0
:1079A000ED0970E0882777FD8095982F0E94DE759D
:1079B000F70120813181428153810E941C789B0113
:1079C000AC01C601B5010E946374688379838A8320
:1079D0009B8309C0F70180819181A281B381888353
:1079E0009983AA83BB830F5F1F4F84E090E0E80E6A
:1079F000F91E24960430110509F0BFCF86E442DE5B
:107A00008823D9F09FDF7B018C016093EE0970938E
:107A1000EF098093F0099093F10920E030E040E015
:107A200050E00E944A77181644F4E0924602F09221
:107A300047020093480210934902DF91CF911F91B2
:107A40000F91FF90EF90DF90CF90BF90AF9008958F
:107A500082DF89E417DE882349F074DF6093D1095F
:107A60007093D2098093D3099093D4098AE40ADEF3
:107A7000882349F067DF6093D5097093D609809316
:107A8000D7099093D80908952F923F924F925F9211
:107A90006F927F928F929F92AF92BF92CF92DF921E
:107AA000EF92FF920F931F93DF93CF93CDB7DEB783
:107AB000A1970FB6F894DEBF0FBECDBF87E4E2DD1D
:107AC000882309F4B7C43EDF0E94AB7564307105AA
:107AD00081F16530710554F46230710511F1633044
:107AE000710514F57723CCF40C949E4C6A3571051E
:107AF00009F441C46B35710534F46C31710511F032
:107B00000C949E4C6DC06B35710509F438C46C350E
:107B1000710511F00C949E4C37C41DDFE0DC0C9411
:107B2000D14C96DF81E002C093DF80E011DC0C9441
:107B3000D14C80E5A7DD882321F4EE24FF248701C2
:107B400005C000DF0E94B0757B018C0183E59ADDE2
:107B5000882359F0F7DE20E030E04AE754E40E9441
:107B60001C780E94B0757B018C010E9420300FB6FA
:107B7000F894A090A80DB090A90DC090AA0DD09037
:107B8000AB0D0FBEAE0CBF1CC01ED11E0FB6F894BD
:107B90008091A80D9091A90DA091AA0DB091AB0D67
:107BA0000FBE8093C9099093CA09A093CB09B093E3
:107BB000CC0904C00E94881581E062DB0FB6F894FE
:107BC0008091A80D9091A90DA091AA0DB091AB0D37
:107BD0000FBE8A159B05AC05BD0560F30C949E4C49
:107BE0008091460290914702A0914802B0914902CB
:107BF0008093FC099093FD09A093FE09B093FF09BF
:107C000080913E0290913F029093A9098093A80928
:107C100084E690E090933F0280933E020FB6F89482
:107C20008091A80D9091A90DA091AA0DB091AB0DD6
:107C30000FBE8093C9099093CA09A093CB09B09352
:107C4000CC0981E00E94502F8091AB099091AC0942
:107C5000A091AD09B091AE098093DD099093DE0942
:107C6000A093DF09B093E0098091AF099091B0092A
:107C7000A091B109B091B2098093E1099093E20912
:107C8000A093E309B093E4098091B3099091B409FA
:107C9000A091B509B091B6098093E5099093E609E2
:107CA000A093E709B093E8098091B7099091B809CA
:107CB000A091B909B091BA098093E9099093EA09B2
:107CC000A093EB09B093EC0980E090E0A0E0B0E075
:107CD0008093460290934702A0934802B0934902D2
:107CE00088E5D0DC882351F489E5CCDC882331F4A5
:107CF0008AE5C8DC882311F481E001C080E080932C
:107D00004A02882329F488E5BDDC882309F4DAC017
:107D10000F2EF0E08F2EF0E09F2EF0E0AF2EF0E07F
:107D2000BF2EF02D8092AB099092AC09A092AD09C4
:107D3000B092AE098BEA99E06FEA79E043EB59E043
:107D400027EB39E00E941C1E80E090ECA9E9B3EC1F
:107D50008093DD099093DE09A093DF09B093E009D9
:107D600060912E0270912F02809130029091310229
:107D700060934602709347028093480290934902B1
:107D800020E030E040E752E40E9443757B018C0123
:107D90008DED99E061EE79E045EE59E029EE39E0AC
:107DA000A7ECCA2EA9E0DA2E0E9400230E94203000
:107DB0008092AB099092AC09A092AD09B092AE0945
:107DC0008BEA99E06FEA79E043EB59E027EB39E081
:107DD0000E941C1E80E090E0A0EAB0E48093DD09E0
:107DE0009093DE09A093DF09B093E0096091460209
:107DF00070914702809148029091490220E030E062
:107E000040E752E40E9443757B018C018DED99E0BF
:107E100061EE79E045EE59E029EE39E00E94002359
:107E20000E94203080E090E0A0E2B1EC8093DD0978
:107E30009093DE09A093DF09B093E00960912E02D0
:107E400070912F02809130029091310220E030E059
:107E500040E05FE30E941C78609346027093470203
:107E6000809348029093490220E030E040E752E4DA
:107E70000E9443757B018C018DED99E061EE79E004
:107E800045EE59E029EE39E00E9400230E9420309F
:107E90008092AB099092AC09A092AD09B092AE0964
:107EA0008092DD099092DE09A092DF09B092E0098C
:107EB0008092460290924702A0924802B0924902F4
:107EC0000E94492F80914A02882329F489E5DADB50
:107ED000882309F4DAC00F2EF0E08F2EF0E09F2EF9
:107EE000F0E0AF2EF0E0BF2EF02D8092AF0990921F
:107EF000B009A092B109B092B2098BEA99E06FEA99
:107F000079E043EB59E027EB39E00E941C1E80E04A
:107F100090ECA9E9B3EC8093E1099093E209A09376
:107F2000E309B093E40960913202709133028091C9
:107F30003402909135026093460270934702809319
:107F400048029093490220E030E040E752E40E946A
:107F500043757B018C018DED99E061EE79E045EE92
:107F600059E029EE39E0F7ECCF2EF9E0DF2E0E9440
:107F700000230E9420308092AF099092B009A09215
:107F8000B109B092B2098BEA99E06FEA79E043EB6C
:107F900059E027EB39E00E941C1E80E090E0A0EA47
:107FA000B0E48093E1099093E209A093E309B093D0
:107FB000E4096091460270914702809148029091D5
:107FC000490220E030E040E752E40E9443757B0123
:107FD0008C018DED99E061EE79E045EE59E029EEF6
:107FE00039E00E9400230E94203080E090E0A0E26F
:107FF000B1EC8093E1099093E209A093E309B09377
:10800000E4096091320270913302809134029091C0
:10801000350220E030E040E05FE30E941C7860938E
:10802000460270934702809348029093490220E0F1
:1080300030E040E752E40E9443757B018C018DEDF6
:1080400099E061EE79E045EE59E029EE39E00E94D1
:1080500000230E9420308092AF099092B009A09234
:10806000B109B092B2098092E1099092E209A0921E
:10807000E309B092E4098092460290924702A092EE
:108080004802B09249020E94492F80914A028823F7
:1080900029F48AE5F7DA882309F4DAC00F2EF0E034
:1080A0008F2EF0E09F2EF0E0AF2EF0E0BF2EF02DEF
:1080B0008092B3099092B409A092B509B092B60922
:1080C0008BEA99E06FEA79E043EB59E027EB39E07E
:1080D0000E941C1E80E090E0A6E9B3EC8093E509C5
:1080E0009093E609A093E709B093E80960913602FE
:1080F0007091370280913802909139026093460264
:1081000070934702809348029093490220E030E048
:1081100040E752E40E9443757B018C018DED99E0AC
:1081200061EE79E045EE59E029EE39E0E7ECCE2E3C
:10813000E9E0DE2E0E9400230E9420308092B309E5
:108140009092B409A092B509B092B6098BEA99E071
:108150006FEA79E043EB59E027EB39E00E941C1EFF
:1081600080E090E0A0E8BFE38093E5099093E60902
:10817000A093E709B093E809609146027091470225
:10818000809148029091490220E030E040E752E4BB
:108190000E9443757B018C018DED99E061EE79E0E1
:1081A00045EE59E029EE39E00E9400230E9420307C
:1081B00080E090E0A0E0B0EC8093E5099093E609C0
:1081C000A093E709B093E8096091360270913702F5
:1081D000809138029091390220E030E040E05FE386
:1081E0000E941C7860934602709347028093480275
:1081F0009093490220E030E040E752E40E9443754A
:108200007B018C018DED99E061EE79E045EE59E05E
:1082100029EE39E00E9400230E9420308092B309A9
:108220009092B409A092B509B092B6098092E5097E
:108230009092E609A092E709B092E809809246027E
:1082400090924702A0924802B09249020E94492FA0
:1082500088E518DA8823C9F06ADB611571058105A4
:10826000910599F06FDB2091BB093091BC094091D9
:10827000BD095091BE090E9463746093AB0970936D
:10828000AC098093AD099093AE0989E5FBD98823A9
:10829000C9F04DDB611571058105910599F052DB3F
:1082A0002091BF093091C0094091C1095091C20984
:1082B0000E9463746093AF097093B0098093B10911
:1082C0009093B2098AE5DED98823C9F030DB6115C5
:1082D00071058105910599F035DB2091C309309135
:1082E000C4094091C5095091C6090E946374609306
:1082F000B3097093B4098093B5099093B6098BEADA
:1083000099E06FEA79E043EB59E027EB39E00E940E
:108310001C1E80E00E94502F8091FC099091FD0965
:10832000A091FE09B091FF09809346029093470205
:10833000A0934802B09349028091A8099091A9099D
:1083400090933F0280933E020FB6F8948091A80D5F
:108350009091A90DA091AA0DB091AB0D0FBE809385
:10836000C9099093CA09A093CB09B093CC090E9484
:10837000492F0C949E4C1092ED090C949E4C81E078
:108380008093ED090C949E4C85E47CD9882311F4EC
:108390000E9420307BEAE72E79E0F72E6BEBC62EA9
:1083A00069E0D62E00E010E0F801E85AFD4F808128
:1083B00069D9882389F1C6DAF601208131814281A9
:1083C00053810E946374F701608371838283938376
:1083D000033059F4B7DAF7016083718382839383A2
:1083E00087EB99E00E94FF1D17C0ACDAF6012081EF
:1083F0003181428153810E946374F70160837183EC
:10840000828393838BEA99E06FEA79E043EB59E04A
:1084100027EB39E00E941C1E0F5F1F4F44E050E025
:10842000E40EF51EC40ED51E0430110509F0BCCFB4
:108430000C949E4C8DE426D9882311F40C94034CA3
:1084400081DA0E94AB756936710509F422C36A3678
:1084500071050CF070C06B31710509F47AC16C3193
:10846000710584F56631710509F418C1673171052C
:10847000BCF46231710509F427C66331710534F427
:108480006131710511F00C949E4CD3C064317105BB
:1084900009F4D5C06531710511F00C949E4CF8C0FB
:1084A0006831710509F418C1683171050CF4FCC01C
:1084B0006931710509F429C16A31710511F00C9413
:1084C0009E4C29C16235710509F4F7C56335710504
:1084D000BCF46E31710509F47EC16F31710534F45D
:1084E0006C31710511F00C949E4C39C16F317105DE
:1084F00009F4B6C16A32710511F00C949E4C2BC27E
:108500006535710509F429C66635710554F463357E
:10851000710509F4D5C56435710511F00C949E4CB4
:10852000D3C56C35710509F42EC66836710511F096
:108530000C949E4C4FC26C3C710509F4D2C76D3C43
:108540007105A4F56337710509F43BC664377105FD
:1085500094F46B36710509F4ADC56B3671050CF4F6
:1085600081C56D36710509F420C36237710511F0BC
:108570000C949E4C36C66E3B710509F4BFC46F3B2C
:10858000710554F46737710509F404C76C38710537
:1085900011F00C949E4C6AC2693C710509F449C7FC
:1085A0006B3C710511F00C949E4C7DC751E06D320F
:1085B000750711F40C942E4B81E06E327807ACF401
:1085C0006E3C710511F40C94EF4A6E3C71050CF48D
:1085D000A8C76C3D710511F40C940D4B6D3D7105F0
:1085E00011F00C949E4C0C941F4B91E0603979076C
:1085F00011F40C94FA4BE1E061397E076CF4F1E080
:108600006E327F0711F40C94E74B6F52714011F0FA
:108610000C949E4C0C94EB4B41E0653F740711F4B5
:108620000C94FD4B665F714011F00C949E4C0C94C1
:10863000FF4B77987698479843980C949E4CE2EBC2
:10864000FCE064918F0108C08DEA9DE00E94E31177
:108650000F5F1F4FF80164916623B1F78DEA9DE02B
:108660006AE00E94E31185EC98E00E948564E4EAE8
:10867000FCE064918F0108C08DEA9DE00E94E31147
:108680000F5F1F4FF80164916623B1F70C94994C6A
:1086900085EC98E00E94D5600C949E4C85EC98E0A7
:1086A0000E94A95C0C949E4C8091000A9091010A52
:1086B00004966AE270E00E94990BFC01009711F0A9
:1086C000319710826091000A7091010A6C5F7F4FB0
:1086D00085EC98E041E07BC085EC98E00E94AD5CC1
:1086E0000FB6F8948091A80D9091A90DA091AA0DB4
:1086F000B091AB0D0FBE8093020A9093030AA09332
:10870000040AB093050A0C949E4C85EC98E00E94F4
:10871000B45C0C949E4C8091C708882311F40C948F
:108720009E4C83E50E94423B882311F40C949E4C9E
:10873000FED8AB01BC014093990950939A098093EC
:108740009B0970939C0986E799E00E94BD530C94A5
:108750009E4C85EC98E00E94605D0C949E4C80914C
:10876000000A9091010A04966AE270E00E94990B57
:108770008C01009719F12091F2093091F30980E6FC
:1087800090E0AC01249FC001259F900D349F900D77
:1087900011248A5F954F6EE470E00E94990B60E2AD
:1087A00070E00E94990B9C012F5F3F4F3093010AAC
:1087B0002093000A01501040F80110826091000AD5
:1087C0007091010A6C5F7F4F85EC98E040E00E9459
:1087D000C35D0C949E4C8091C708882311F40C94BF
:1087E0009E4C85EC98E00E94D55C8091000A9091A7
:1087F000010A04966AE270E00E94990B8C010097CE
:1088000019F12091F2093091F30980E690E0AC0172
:10881000249FC001259F900D349F900D11248A5FE5
:10882000954F6EE470E00E94990B60E270E00E9448
:10883000990B9C012F5F3F4F3093010A2093000A50
:1088400001501040F80110826091000A7091010AF5
:108850006C5F7F4F85EC98E00E949E5F0C949E4C6D
:108860000FB6F8946091A80D7091A90D8091AA0D92
:108870009091AB0D0FBE6093860B7093870B809326
:10888000880B9093890B2091020A3091030A409142
:10889000040A5091050A621B730B840B950B28EE9A
:1088A00033E040E050E00E942079F22EE32ED42EF7
:1088B000C52E4DB75EB7485050400FB6F8945EBF16
:1088C0000FBE4DBF0DB71EB70F5F1F4FCE010196F4
:1088D000EDB7FEB79283818380E491E0F801938342
:1088E00082836F2D7E2D8D2D9C2D2CE330E040E07A
:1088F00050E00E942079F801358324836F2D7E2D6E
:108900008D2D9C2D2CE330E040E050E00E9420793A
:10891000F801778366830E94E20BEAE9FBE0649149
:108920008F014DB75EB7485F5F4F0FB6F8945EBFDB
:108930000FBE4DBF08C08DEA9DE00E94E3110F5F9E
:108940001F4FF80164916623B1F78DEA9DE0BE01E7
:108950006F5F7F4F8AC783E50E94423B882309F4FB
:10896000EDC70E94A23C7B018C0180E50E94423B46
:10897000882309F4E3C7C801B7010E94AB756B01F6
:1089800077FF01C0DBC76F3F710511F00CF0D6C750
:108990000E94A23C0E94AB757B01ECE5F2E0808175
:1089A00091818E159F0509F4C9C7329622E0E03DFA
:1089B000F207A9F7F7FE01C0C1C78E2D0E943A6CDD
:1089C000EE2DF0E00C2C0E944B6C8E2DB6010E9417
:1089D000F56DB4C78091C70980938A0B84E50E9426
:1089E000423B8823E1F00E94A23C0E94B075609354
:1089F0008A0B6623A1F0EAE9FBE064918F0108C0CD
:108A00008DEA9DE00E94E3110F5F1F4FF801649112
:108A10006623B1F78DEA9DE06FE471E0EAC083E57B
:108A20000E94423B8823F9F00E94A23C6B017C012A
:108A3000B0908A0B0B2D10E00E94AB75DC01CB01CE
:108A40006B2D0E943E17000F111FF801E252FD4FDF
:108A500091838083000F111F0A511D4FF801C082BE
:108A6000D182E282F3820E942C1368C783E50E94C0
:108A7000423B882309F462C70E94A23C0E94AB7566
:108A8000DC01CB010E9418129093E1028093E00276
:108A900055C78091C70980938A0B84E50E94423BA9
:108AA0008823E1F00E94A23C0E94B07560938A0B7B
:108AB0006623A1F0EAE9FBE064918F0108C08DEA2A
:108AC0009DE00E94E3110F5F1F4FF8016491662340
:108AD000B1F78DEA9DE066E671E08BC0EEE9FCE05F
:108AE00064918F0108C08DEA9DE00E94E3110F5F41
:108AF0001F4FF80164916623B1F760918A0BE62F4E
:108B0000F0E0EE0FFF1FEE51FD4F808191810E943A
:108B10006714AB01BC018DEA9DE022E00E948271E6
:108B2000EAE9FCE064918F0108C08DEA9DE00E94B3
:108B3000E3110F5F1F4FF80164916623B1F7809135
:108B4000E4029091E5020E947912AB01BC018DEA2A
:108B50009DE022E00E948271E6E9FCE064918F01D1
:108B600008C08DEA9DE00E94E3110F5F1F4FF801DE
:108B700064916623B1F780918A0B90E00E941212F3
:108B8000AC01662757FD6095762F8DEA9DE00E9427
:108B900071718DEA9DE06DE771E00E9433308DEADE
:108BA0009DE06AE00E94E311FCC68091C7098093B2
:108BB0008A0B84E50E94423B882349F10E94A23C33
:108BC0000E94B07560938A0B662309F1EAE9FBE025
:108BD00064918F0108C08DEA9DE00E94E3110F5F50
:108BE0001F4FF80164916623B1F78DEA9DE06EE7AF
:108BF00071E00E94333040918A0B50E060E070E0F9
:108C00008DEA9DE02AE000E00E94E67092C683E5CE
:108C10000E94423B8823F9F00E94A23C6B017C0138
:108C2000B0908A0B0B2D10E00E94AB75DC01CB01DC
:108C30006B2D0E943E17000F111FF801E252FD4FED
:108C400091838083000F111F0A511D4FF801C082CC
:108C5000D182E282F3820E942C130FB6F8946090C6
:108C6000A80D7090A90D8090AA0D9090AB0D0FBE2D
:108C7000E0918A0BF0E0EE0FFF1FDF01A252BD4F23
:108C80002D903C90EE51FD4F40805180AA24AA9433
:108C9000BA2C6501E3E9FCE024912F8FEFE8FCE0BA
:108CA000449148A3EBE8FCE0549159A311C16F8DA6
:108CB00003E91CE008C08DEA9DE00E94E3110F5F0C
:108CC0001F4FF80164916623B1F760918A0BE62F7C
:108CD000F0E0EE0FFF1FEE51FD4F808191810E9469
:108CE0006714AB01BC018DEA9DE022E00E94827115
:108CF00068A10FE81CE008C08DEA9DE00E94E31126
:108D00000F5F1F4FF80164916623B1F740918A0B02
:108D100050E0662757FD6095762F8DEA9DE00E9412
:108D2000717169A10BE81CE008C08DEA9DE00E940A
:108D3000E3110F5F1F4FF80164916623B1F7D7FC71
:108D400024C00FB6F8942091A80D3091A90D409140
:108D5000AA0D5091AB0D0FBEC601B501605F784DF5
:108D60008F4F9F4F621B730B840B950B28EE33E0E4
:108D700040E050E00E9420798DEA9DE0BA01A9010F
:108D80002AE000E00E94E67006C08DEA9DE065E9F9
:108D900071E00E9433308DEA9DE06AE00E94E311A9
:108DA0000FB6F8946090A80D7090A90D8090AA0D50
:108DB0009090AB0D0FBE0E94881581E00E94403953
:108DC000FFEFAF16FFEFBF06FFEFCF06FFEFDF06A7
:108DD00031F5E0918A0B421453048CF4F0E0EE0F6D
:108DE000FF1FDF01AE51BD4FE252FD4F20813181A7
:108DF0008D919C91821793070CF043C04DC0F0E019
:108E0000EE0FFF1FDF01AE51BD4FE252FD4F20813B
:108E100031818D919C91281739079CF53DC0D7FC75
:108E20003BC060918A0BE62FF0E0EE0FFF1FEE5182
:108E3000FD4F808191810E9467147B018C016091BC
:108E40008A0BE62FF0E0EE0FFF1FE252FD4F80810C
:108E500091810E9467149B01AC01C801B7010E9477
:108E600062740E94AB7597FF07C0909580957095CE
:108E700061957F4F8F4F9F4F64307105810591053C
:108E80005CF00FB6F894A090A80DB090A90DC0901A
:108E9000AA0DD090AB0D0FBE2FEFA2162FEFB2068A
:108EA0002FEFC2062FEFD20699F0D7FC4AC50FB6B6
:108EB000F8948091A80D9091A90DA091AA0DB09160
:108EC000AB0D0FBE8A199B098051974208F039C536
:108ED0000FB6F8948091A80D9091A90DA091AA0DBC
:108EE000B091AB0D0FBE86199709A809B909895E23
:108EF0009340A040B04008F0DACE5DCF83E50E94F9
:108F0000423B882361F00E94A23C0E94AB75DC01C9
:108F1000CB010E9418129093E1028093E0020FB6F9
:108F2000F894E090A80DF090A90D0091AA0D109171
:108F3000AB0D0FBEE8E8FCE09490E4E8FCE0A49000
:108F4000E0E8FCE0B49081C00FB6F8948091A80DE1
:108F50009091A90DA091AA0DB091AB0D0FBE8E19E5
:108F60009F09A00BB10B895E9340A040B04008F46C
:108F700067C06091C709E62FF0E0EE0FFF1FEE51CA
:108F8000FD4F808191810E9467146B017C01692DE6
:108F900008E81CE008C08DEA9DE00E94E3110F5F25
:108FA0001F4FF80164916623B1F78DEA9DE0B70188
:108FB000A60122E00E9482716A2D04E81CE008C02C
:108FC0008DEA9DE00E94E3110F5F1F4FF80164914D
:108FD0006623B1F74091C70950E0662757FD6095B9
:108FE000762F8DEA9DE00E9471716B2D00E81CE0E8
:108FF00008C08DEA9DE00E94E3110F5F1F4FF8014A
:1090000064916623B1F78091E4029091E5020E9499
:109010007912AB01BC018DEA9DE022E00E948271D1
:109020008DEA9DE06AE00E94E3110FB6F894E090AB
:10903000A80DF090A90D0091AA0D1091AB0D0FBED7
:109040000E94881581E00E9440392091E002309111
:10905000E1028091E4029091E502821793070CF4FB
:1090600073CF82C483E50E94423B8823F9F00E94BB
:10907000A23C20E030E040E050E00E943C758823B4
:1090800014F460E010C00E94A23C20E030E04FE702
:1090900053E40E944A77181614F46FEF04C00E943C
:1090A000A23C0E94B0756093C80948C48FEF8093BA
:1090B000C80944C41092C80941C41092A7093EC40B
:1090C00081E08093A7093AC483E50E94423B88234C
:1090D00099F00E94A23C20E030E04AE754E40E946C
:1090E0001C780E94B0756093420270934302809393
:1090F00044029093450222C488E50E94423B8823A3
:1091000009F046C489E50E94423B882309F040C427
:109110008AE50E94423B882309F03AC485E40E9414
:10912000423B882309F034C40E942030439A0E94B5
:109130002D3004C4779A89E50E94423B8111769ACA
:109140008AE50E94423B8111479A85E40E94423B96
:10915000882309F4F3C3439AF1C383E50E94423B99
:109160000E94A23C20E030E04AE754E40E941C78D0
:109170000E94B0756093CD097093CE098093CF099A
:109180009093D009DBC308E512E03CE3E32E33E023
:10919000F32EF80180810E94423B882339F00E941F
:1091A000A23CF70160837183828393830F5F1F4F1B
:1091B00044E050E0E40EF51E52E00C35150749F787
:1091C000BDC3E5EEFBE064918F0108C08DEA9DE030
:1091D0000E94E3110F5F1F4FF80164916623B1F7FE
:1091E000ADC3E2EEFBE064918F0108C08DEA9DE023
:1091F0000E94E3110F5F1F4FF80164916623B1F7DE
:109200004091AB095091AC096091AD097091AE09E4
:109210008DEA9DE022E00E948271EFEDFBE0649117
:109220008F0108C08DEA9DE00E94E3110F5F1F4F80
:10923000F80164916623B1F74091AF095091B009EC
:109240006091B1097091B2098DEA9DE022E00E941F
:109250008271ECEDFBE064918F0108C08DEA9DE026
:109260000E94E3110F5F1F4FF80164916623B1F76D
:109270004091B3095091B4096091B5097091B60954
:109280008DEA9DE022E00E948271E9EDFBE06491AD
:109290008F0108C08DEA9DE00E94E3110F5F1F4F10
:1092A000F80164916623B1F74091B7095091B8096C
:1092B0006091B9097091BA098DEA9DE022E00E949F
:1092C0008271EFECFBE064918F0108C08DEA9DE0B4
:1092D0000E94E3110F5F1F4FF80164916623B1F7FD
:1092E00080E00E94EB2F0E94DE7520913C033091BC
:1092F0003D0340913E0350913F030E944375AB01F3
:10930000BC018DEA9DE022E00E948271ECECFBE062
:1093100064918F0108C08DEA9DE00E94E3110F5F08
:109320001F4FF80164916623B1F781E00E94EB2F93
:109330000E94DE7520914003309141034091420329
:10934000509143030E944375AB01BC018DEA9DE03F
:1093500022E00E948271E9ECFBE064918F0108C079
:109360008DEA9DE00E94E3110F5F1F4FF8016491A9
:109370006623B1F782E00E94EB2F0E94DE752091F8
:1093800044033091450340914603509147030E94A6
:10939000437511C2E2ECFBE064918F0108C08DEAD5
:1093A0009DE00E94E3110F5F1F4FF8016491662357
:1093B000B1F7639B03C067E971E002C06AE971E03D
:1093C0008DEA9DE00E943330EBEBFBE064918F016E
:1093D00008C08DEA9DE00E94E3110F5F1F4FF80166
:1093E00064916623B1F7189B03C067E971E002C07E
:1093F0006AE971E08DEA9DE00E943330E4EBFBE026
:1094000064918F0108C08DEA9DE00E94E3110F5F17
:109410001F4FF80164916623B1F7649B03C067E9AD
:1094200071E002C06AE971E08DEA9DE00E9433308C
:10943000C9C128E5C22E22E0D22EEE24FF24F60177
:1094400080810E94423B882309F10E94A23C87014F
:10945000045B1C4F0E94B075F801608371838283A6
:1094600093830E94A23C870108581C4FF701E45CDB
:10947000FC4F20813181428153810E941C780E94DF
:10948000B075F80160837183828393830894C11C53
:10949000D11C44E050E0E40EF51E5CE5C51652E038
:1094A000D50669F64BC208E512E09CE2E92E93E08E
:1094B000F92EF80180810E94423B882339F00E94F6
:1094C000A23CF70160837183828393830F5F1F4FF8
:1094D00044E050E0E40EF51E52E00C35150749F764
:1094E0002DC283E50E94423B882351F00E94A23C9A
:1094F00060936003709361038093620390936303AE
:1095000084E50E94423B882309F418C20E94A23CD1
:10951000609364037093650380936603909367037D
:109520000DC283E50E94423B882351F00E94A23C79
:1095300060935C0370935D0380935E0390935F037D
:1095400084E50E94423B882351F00E94A23C609334
:10955000740370937503809376039093770382E48A
:109560000E94423B882361F00E94A23C0E94B07599
:10957000609328037093290380932A0390932B030D
:1095800088E50E94423B882351F00E94A23C6093F0
:1095900068037093690380936A0390936B038AE571
:1095A0000E94423B882351F00E94A23C60936C03CE
:1095B00070936D0380936E0390936F0385E40E9414
:1095C000423B882309F4BAC10E94A23C6093700315
:1095D000709371038093720390937303AFC108E596
:1095E00012E08BEBE82E89E0F82EF80180810E94D2
:1095F000423B882339F00E94A23CF70160837183CB
:10960000828393830F5F1F4F44E050E0E40EF51E0A
:1096100052E00B35150749F791C183E50E94423BA3
:10962000882309F48BC10E94A23C0E94AB75709301
:109630003F0260933E0281E08093AA097FC183E5E7
:109640000E94423B882309F479C10E94A23C0E94F7
:10965000AB75709341026093400270C180E50E9437
:10966000423B882351F00E94A23C60931402709305
:109670001502809316029093170289E40E94423BE0
:10968000882381F00E94A23C2DEB37E346E05EE3A5
:109690000E941C78609318027093190280931A023A
:1096A00090931B0284E40E94423B882381F00E9435
:1096B000A23C2DEB37E346E05EE30E9443756093E6
:1096C0001C0270931D0280931E0290931F0283E47C
:1096D0000E94423B882351F00E94A23C60932002EA
:1096E0007093210280932202909323020E94FB1127
:1096F0008DEA9DE06DE971E00E9433308DEA9DE0D6
:1097000060EA71E00E9433304091140250911502DA
:1097100060911602709117028DEA9DE022E00E948E
:1097200082718DEA9DE064EA71E00E9433306091BD
:1097300018027091190280911A0290911B022DEB70
:1097400037E346E05EE30E944375AB01BC018DEA5E
:109750009DE022E00E9482718DEA9DE068EA71E05E
:109760000E94333060911C0270911D0280911E0294
:1097700090911F022DEB37E346E05EE30E941C78D8
:10978000AB01BC018DEA9DE022E00E9482718DEA6E
:109790009DE06CEA71E00E9433306091200270918C
:1097A000210280912202909123022DEB37E346E0C3
:1097B0005EE30E941C78AB01BC018DEA9DE022E0D3
:1097C0000E9482718DEA9DE06DE771E04EC081E0FC
:1097D0000E94FC1DB3C083E50E94423B882329F40C
:1097E00060E070E086E193E402C00E94A23C0E9427
:1097F0008C18A4C00E942030A1C080E001C081E08C
:109800000E94633B9BC084E50E94423B882309F48D
:1098100050C00E94A23C0E94B07560938A0BEAE996
:10982000FBE0662329F164918F0108C08DEA9DE079
:109830000E94E3110F5F1F4FF80164916623B1F797
:109840008DEA9DE060EB71E00E94333040918A0B1D
:1098500050E060E070E08DEA9DE02AE000E00E94C8
:10986000E6708DEA9DE062EB71E00E94333061C0EA
:109870001092C70964918F0108C08DEA9DE00E9493
:10988000E3110F5F1F4FF80164916623B1F78DEA72
:109890009DE063EC71E00E9433304091C70950E0D5
:1098A000662757FD6095762F8DEA9DE00E947171C5
:1098B00040C0EAE9FBE064918F0108C08DEA9DE0B9
:1098C0000E94E3110F5F1F4FF80164916623B1F707
:1098D000E2EAFBE064918F0108C08DEA9DE00E94FE
:1098E000E3110F5F1F4FF80164916623B1F72091D8
:1098F000F2093091F30980E690E0289FB001299F9A
:10990000700D389F700D11246A5F754F8DEA9DE0D0
:109910000E943330E0EAFBE064918F0108C08DEAD9
:109920009DE00E94E3110F5F1F4FF80164916623D1
:10993000B1F78DEA9DE06AE00E94E3110E947C3855
:1099400030C00FB6F8948091A80D9091A90DA09108
:10995000AA0DB091AB0D0FBE8093020A9093030A3B
:10996000A093040AB093050A0FB6F8948091A80D4D
:109970009091A90DA091AA0DB091AB0D0FBE80934F
:10998000C9099093CA09A093CB09B093CC09D6CF4B
:109990000E94203088E50E94423B882309F0CACB10
:1099A000CACBA1960FB6F894DEBF0FBECDBFCF9144
:1099B000DF911F910F91FF90EF90DF90CF90BF90BC
:1099C000AF909F908F907F906F905F904F903F905F
:1099D0002F9008953F924F925F926F927F928F9255
:1099E0009F92AF92BF92CF92DF92EF92FF920F932E
:1099F0001F93DF93CF93CDB7DEB76E970FB6F89472
:109A0000DEBF0FBECDBF20E6C22ED12CE5EDFCE0BF
:109A1000B490AA24A394FAC12D3051F02A3341F016
:109A200080918C0B90918D0B8F3591050CF4CAC1F0
:109A3000E0918C0BF0918D0B309709F4D1C2A0917D
:109A40008F0BB091900BAC9D7001AD9DF00CBC9D47
:109A5000F00C1124EE0DFF1DEA5FF54F108280918E
:109A60008E0B882309F0A9C110928E0BAC50B64F13
:109A70001C9287010A5F154FC8016EE470E00E94D6
:109A8000990B9C01009709F4FEC09093010A809302
:109A9000000A2F5F3F4F201B310B2E0D3F1DC901C8
:109AA0008A5F954F60E070E04AE050E00E94310A22
:109AB0006093910B7093920B8093930B9093940B04
:109AC0002091F8093091F9094091FA095091FB0968
:109AD0002F5F3F4F4F4F5F4F621773078407950704
:109AE00009F435C080918F0B9091900B9C012C9DB7
:109AF000C0012D9D900D3C9D900D11248A5F954FC6
:109B000065ED71E00E94C80B009709F5E7E6FBE000
:109B100064917F0109C08DEA9DE00E94E3110894E1
:109B2000E11CF11CF70164916623A9F7E8E4FDE06C
:109B300064917F0109C08DEA9DE00E94E3110894C1
:109B4000E11CF11CF70164916623A9F777C08091AD
:109B50008F0B9091900B8C9D80018D9D100D9C9D85
:109B6000100D1124C8018A5F954F6AE270E00E94CF
:109B7000990B9C01009709F441C0FF2440E0C80103
:109B800002C0FE264F5FFC01E40FF11DEA5FF54FB6
:109B9000E081EA32B1F73093010A2093000AC9014B
:109BA000019660E070E00E94D4080E94AB752F2DF2
:109BB00030E02617370709F455C0E7E6FBE064916B
:109BC0007F0109C08DEA9DE00E94E3110894E11C29
:109BD000F11CF70164916623A9F7EAE2FDE06491C4
:109BE0007F0109C08DEA9DE00E94E3110894E11C09
:109BF000F11CF70164916623A9F720C0E7E6FBE0BA
:109C000064917F0109C08DEA9DE00E94E3110894F0
:109C1000E11CF11CF70164916623A9F7E1E0FDE086
:109C200064917F0109C08DEA9DE00E94E3110894D0
:109C3000E11CF11CF70164916623A9F74091F80932
:109C40005091F9096091FA097091FB098DEA9DE044
:109C50000E9471718DEA9DE06AE00E94E3110E940A
:109C6000153B4AC08091910B9091920BA091930B60
:109C7000B091940B8093F8099093F909A093FA0995
:109C8000B093FB093EC0C8016AE270E00E94990BE4
:109C9000009709F436C0E7E6FBE064917F0109C054
:109CA0008DEA9DE00E94E3110894E11CF11CF7018C
:109CB00064916623A9F7E8EDFCE064917F0109C097
:109CC0008DEA9DE00E94E3110894E11CF11CF7016C
:109CD00064916623A9F74091F8095091F9096091C0
:109CE000FA097091FB098DEA9DE00E9471718DEA7D
:109CF0009DE06AE00E94E31110928D0B10928C0B94
:109D000013C280918F0B9091900B8C9D70018D9D53
:109D1000F00C9C9DF00C112487010A5F154FC801BF
:109D200067E470E00E94990B9C01009781F1909389
:109D3000010A8093000A2F5F3F4F201B310B2E0D2D
:109D40003F1DC9018A5F954F60E070E00E94D40812
:109D50000E94AB7564307105D0F48091C5088823EA
:109D6000B1F46B2D95EDE92E9CE0F92E09C08DEA3A
:109D70009DE00E94E3110894E11CF11CF70164913D
:109D80006623A9F78DEA9DE06AE00E94E3118091C5
:109D90008F0B9091900B019664E070E00E940D791A
:109DA0009093900B80938F0B8091950B9091960BD5
:109DB00001969093960B8093950B10928D0B1092B9
:109DC0008C0B24C02B3311F4A0928E0B80918E0B40
:109DD0008823E1F420918C0B30918D0B80918F0BB7
:109DE0009091900B8C9DF0018D9DF00D9C9DF00D40
:109DF0001124E20FF31FEA5FF54F80918B0B8083F4
:109E00002F5F3F4F30938D0B20938C0B8DEA9DE09D
:109E10000E94996E181619060CF081C18091950B5D
:109E20009091960B04970CF07AC18DEA9DE00E9408
:109E3000D26E282F80938B0B8A3009F0EDCDF8CDB0
:109E400080918C0B90918D0B892B09F41FC16CC1F3
:109E50004D3069F04A3359F080918C0B90918D0B05
:109E60008F35910524F42F5F3F4F09F0EAC0209110
:109E7000990930919A0940919B0950919C098091D0
:109E8000910990919209A0919309B0919409281792
:109E900039074A075B0708F49CC0662D82ECE82E60
:109EA0008CE0F82E09C08DEA9DE00E94E311089431
:109EB000E11CF11CF70164916623A9F78DEA9DE08E
:109EC0006AE00E94E3110FB6F8946091A80D7091BA
:109ED000A90D8091AA0D9091AB0D0FBE6093860BDA
:109EE0007093870B8093880B9093890B2091020AC3
:109EF0003091030A4091040A5091050A621B730BCA
:109F0000840B950B28EE33E040E050E00E9420796E
:109F1000F22EE32ED42EC52E2DB73EB7285030405A
:109F20000FB6F8943EBF0FBE2DBF0DB71EB70F5F23
:109F30001F4FEDB7FEB7B282A182F8015382428271
:109F40006F2D7E2D842F952F2CE330E040E050E0E4
:109F50000E942079F801358324836F2D7E2D8D2D6D
:109F60009C2D2CE330E040E050E00E942079F80185
:109F7000778366830E94E20B672D0AE9E02E0BE0EF
:109F8000F02E2DB73EB7285F3F4F0FB6F8943EBF77
:109F90000FBE2DBF09C08DEA9DE00E94E311089419
:109FA000E11CF11CF70164916623A9F78DEA9DE09D
:109FB000B5010E9433308DEA9DE06AE00E94E31112
:109FC00085EC98E00E94B95C85EC98E061E00E9425
:109FD000AA6120918C0B30918D0B2115310519F45C
:109FE00010928E0BA1C080918F0B9091900B889D49
:109FF000F001899DF00D989DF00D1124E20FF31FE3
:10A00000EA5FF54F1082FC01EC50F64F3082209150
:10A01000950B3091960B2F5F3F4F3093960B20930B
:10A02000950B019664E070E00E940D799093900B7F
:10A0300080938F0B10928E0B10928D0B10928C0BC5
:10A0400038C04B3311F430928E0B80918E0B8823E5
:10A0500081F520918C0B30918D0B80918F0B90911D
:10A06000900B889DF001899DF00D989DF00D1124B5
:10A07000E20FF31FEA5FF54F80918B0B80832F5F18
:10A080003F4F30938D0B20938C0B13C010E6812E25
:10A09000912C33243394E2ECFCE064905E0108944C
:10A0A000A11CB11CB0E44B2EB1E05B2EEAE9FBE051
:10A0B00074902091990930919A0940919B0950918F
:10A0C0009C098091910990919209A0919309B09176
:10A0D0009409281739074A075B0730F58091950BDB
:10A0E0009091960B049704F580917E0990917F09D9
:10A0F000A0918009B09181098093990990939A0960
:10A10000A0939B09B0939C0986E799E07BD69C01BC
:10A11000482F80938B0B8A3009F09ACEA8CE80917D
:10A12000C608882309F08CCE6E960FB6F894DEBF71
:10A130000FBECDBFCF91DF911F910F91FF90EF9098
:10A14000DF90CF90BF90AF909F908F907F906F9057
:10A150005F904F903F900895CF93DF938091950B40
:10A160009091960B03970CF435DC85EC98E060E059
:10A170000E94AA618091950B9091960B892B09F40E
:10A180005FC08091C508882309F442C02091F2097C
:10A190003091F30980E690E0289FE001299FD00DDF
:10A1A000389FD00D1124CA5FD54FCE016AED71E002
:10A1B0000E94C80B0097A1F485EC98E0BE010E94B4
:10A1C000EA5CECE8FDE06491EF0107C08DEA9DE0F8
:10A1D0000E94E3112196FE0164916623B9F712C033
:10A1E00085EC98E00E94D55CEAE7FDE06491EF0120
:10A1F00007C08DEA9DE00E94E3112196FE01649163
:10A200006623B9F78DEA9DE06AE00E94E31102C07F
:10A210000E94443D8091950B9091960B01979093ED
:10A22000960B8093950B8091F2099091F30901961A
:10A2300064E070E00E940D799093F3098093F20935
:10A240000E94881581E00E9440390E947737DF9193
:10A25000CF910895CF92DF92EF92FF920F931F93C9
:10A26000DF93CF9300D0CDB7DEB78DEA9DE040E914
:10A2700050ED63E070E00E944E70EDE3FEE064910B
:10A280008F0108C08DEA9DE00E94E3110F5F1F4F10
:10A29000F80164916623B1F78DEA9DE06AE00E94BF
:10A2A000E3113AE9C32E3BE0D32EF6016491860117
:10A2B00008C08DEA9DE00E94E3110F5F1F4FF80177
:10A2C00064916623B1F784B7F82E80FF14C0E5E3EC
:10A2D000FEE064918F0108C08DEA9DE00E94E311C9
:10A2E0000F5F1F4FF80164916623B1F78DEA9DE07F
:10A2F0006AE00E94E311F1FE14C0E5E2FEE0649121
:10A300008F0108C08DEA9DE00E94E3110F5F1F4F8F
:10A31000F80164916623B1F78DEA9DE06AE00E943E
:10A32000E311F2FE14C0E4E1FEE064918F0108C085
:10A330008DEA9DE00E94E3110F5F1F4FF8016491C9
:10A340006623B1F78DEA9DE06AE00E94E311F3FE17
:10A3500014C0E4E0FEE064918F0108C08DEA9DE046
:10A360000E94E3110F5F1F4FF80164916623B1F75C
:10A370008DEA9DE06AE00E94E311F5FE14C0E4EF6F
:10A38000FDE064918F0108C08DEA9DE00E94E31119
:10A390000F5F1F4FF80164916623B1F78DEA9DE0CE
:10A3A0006AE00E94E31114BEEBEEFDE064918F01C0
:10A3B00008C08DEA9DE00E94E3110F5F1F4FF80176
:10A3C00064916623B1F7E1EEFDE064918F0108C06E
:10A3D0008DEA9DE00E94E3110F5F1F4FF801649129
:10A3E0006623B1F78DEA9DE06AE00E94E311F60171
:10A3F00064910AE91BE008C08DEA9DE00E94E31128
:10A400000F5F1F4FF80164916623B1F7E1EDFDE0A6
:10A4100064918F0108C08DEA9DE00E94E3110F5FF7
:10A420001F4FF80164916623B1F7E6ECFDE06491FB
:10A430008F0108C08DEA9DE00E94E3110F5F1F4F5E
:10A44000F80164916623B1F7EAEBFDE064918F01B6
:10A4500008C08DEA9DE00E94E3110F5F1F4FF801D5
:10A4600064916623B1F7E5EBFDE064918F0108C0CC
:10A470008DEA9DE00E94E3110F5F1F4FF801649188
:10A480006623B1F78DEA9DE06AE00E94E311F601D0
:10A4900064910AE91BE008C08DEA9DE00E94E31187
:10A4A0000F5F1F4FF80164916623B1F7E6EAFDE004
:10A4B00064918F0108C08DEA9DE00E94E3110F5F57
:10A4C0001F4FF80164916623B1F720914B02309140
:10A4D0004C02CE0101962115310519F48D5B9D408A
:10A4E00002C0821B930B9A83898349815A81662714
:10A4F00057FD6095762F8DEA9DE00E947171EFE81F
:10A50000FDE064918F0108C08DEA9DE00E94E31197
:10A510000F5F1F4FF80164916623B1F78DEA9DE04C
:10A5200040ED54E060E070E00E9471718DEA9DE0C2
:10A530006AE00E94E3111092F4091092F50910925A
:10A54000F6091092F70980E00E94633BEE24FF2495
:10A55000870108581C4FF701E45BFC4F6081718153
:10A56000828193810E94DC75F701E45CFC4F2081BD
:10A570003181428153810E941C780E94B075F8019C
:10A58000608371838283938384E090E0E80EF91EF8
:10A5900090E1E916F104E1F60E942F180E943D2097
:10A5A0000E94592F0F900F90CF91DF911F910F9123
:10A5B000FF90EF90DF90CF900895CF93DF93BC0191
:10A5C0008091950B9091960B04970CF06AC02091A6
:10A5D0008F0B3091900B80E690E0AC01249FC0017E
:10A5E000259F900D349F900D11248A5F954F0E94F6
:10A5F000A40BEAE9FBE06491EF0107C08DEA9DE05E
:10A600000E94E3112196FE0164916623B9F7E5E407
:10A61000FEE06491EF0107C08DEA9DE00E94E31126
:10A620002196FE0164916623B9F720918F0B30913A
:10A63000900B80E690E0289FB001299F700D389F15
:10A64000700D11246A5F754F8DEA9DE00E943330D2
:10A65000E3E4FEE06491EF0107C08DEA9DE00E9413
:10A66000E3112196FE0164916623B9F78DEA9DE01E
:10A670006AE00E94E31180918F0B9091900B0196FC
:10A6800064E070E00E940D799093900B80938F0BA3
:10A690008091950B9091960B01969093960B8093D9
:10A6A000950BDF91CF910895DB010D900020E9F724
:10A6B0001197A61BB70B0396AD01F7C4DF93CF9399
:10A6C0000F92CDB7DEB769830396BE016F5F7F4FF0
:10A6D00041E050E0EAD40F90CF91DF9108950F93BD
:10A6E0001F93CF93DF93DC01EB018A0180E090E0C0
:10A6F00020E2FE01E80FF91F208301968B309105BF
:10A70000C1F757E040E024C0622F2E3219F080E5F7
:10A710009EE007C05A3051F15AE048E018C03217A5
:10A7200029F1FC01019634913323C9F75417F0F055
:10A730002132E0F02F37D0F4822F81568A3110F485
:10A74000622F6052FE01E40FF11D60834F5F11968E
:10A750002C91222311F02F32B9F6F801B183A08396
:10A7600090E08881803219F091E001C090E0892F5B
:10A77000DF91CF911F910F9108956F927F928F92E9
:10A780009F92AF92BF92CF92DF92EF92FF920F9380
:10A790001F93CF93DF93EC017A018B012B8122234E
:10A7A00009F480C089899A89AB89BC898417950787
:10A7B000A607B70708F476C085C0E114F1040105C7
:10A7C000110551F41C821D821E821F821886198673
:10A7D0001A861B8681E067C0288539854A855B8596
:10A7E000E98DFA8D858590E00996215030404040F2
:10A7F000504039014A01082E04C0969487947794FA
:10A8000067940A94D2F72F5F3F4F4F4F5F4F0894E2
:10A81000E108F108010911095701680104C0D69443
:10A82000C794B794A7948A95D2F70894E11CF11CB9
:10A83000011D111DA614B704C804D90428F0211560
:10A8400031054105510549F48D899E89AF89B88D3F
:10A850008C839D83AE83BF8316C0A618B708C80833
:10A86000D90811C04C815D816E817F81898D9A8D5F
:10A8700094010E942D670894A108B108C108D1086D
:10A88000882331F40FC084E0882E912C8C0E9D1EFD
:10A89000A114B104C104D10429F7E886F9860A8716
:10A8A0001B8798CF80E0DF91CF911F910F91FF9090
:10A8B000EF90DF90CF90BF90AF909F908F907F9060
:10A8C0006F900895223009F078CFE7CFCF93DF93D0
:10A8D000EC018C859D85AE85BF8540E0611141E02E
:10A8E000BC01CD010E940865882319F420E030E006
:10A8F0000AC08889282F30E095E0220F331F9A95EF
:10A90000E1F72356344FC901DF91CF9108950F939A
:10A910001F93CF93DF938C01FC0183818823D9F1AE
:10A92000818187FF35C0C80161E0D0DFEC0100976D
:10A9300091F18881853E79F1F8018381823040F47C
:10A9400081899289A389B4898C8F9D8FAE8FBF8FA7
:10A95000F80185899689A789B08D9B8F8A8FCD0153
:10A96000AA27BB279D8B8C8BE091970BF091980BBE
:10A97000309751F0BE016A5E7F4FCE01489609952F
:10A98000888D998D9B8B8A8BF80181818F7781834C
:10A990000E94CF6404C081E0F801808380E0DF91F1
:10A9A000CF911F910F9108950F931F938C01AFDFEB
:10A9B000F80113821F910F910895FC018381882370
:10A9C00011F0CF01F1CF08956F927F928F929F92F5
:10A9D000AF92BF92CF92DF92EF92FF920F931F93AD
:10A9E000DF93CF9300D000D0CDB7DEB77C015A0102
:10A9F0006B01DC0113968C911397813009F08EC0A6
:10AA000011968C9181FF8AC09DC00097A105B10568
:10AA100011F481E084C0F70160847184828493849E
:10AA2000C701B601A501A9DE882309F477C0D701C3
:10AA300059968D919C915A97A114B104C104D104E7
:10AA400089F455964D915D916D917C9158970E9436
:10AA5000A267882309F462C0F701158A168A178A4B
:10AA6000108E44C0D70114964D915D916D917C91EB
:10AA700017979E012F5F3F4F0E942D67882309F48F
:10AA80004DC0D7015996ED91FC915A9749815A8151
:10AA90006B817C818789803149F4483FBFEF5B0738
:10AAA000B0E06B07B0E07B0748F020C0483F8FEF75
:10AAB00058078FEF68078FE07807C0F4CF010E9436
:10AAC000A267882359F1D70114964D915D916D913C
:10AAD0007C91179759968D919C915A970FEF1FEF84
:10AAE0002FEF3FE00E94A7668823C1F0F701A18AFB
:10AAF000B28AC38AD48A818180688183C70107DFD3
:10AB0000882361F0B601A5016A147B048C049D04BE
:10AB100010F4B401A301C70130DE01C080E00F9042
:10AB20000F900F900F90CF91DF911F910F91FF9099
:10AB3000EF90DF90CF90BF90AF909F908F907F90DD
:10AB40006F900895F70181899289A389B489841748
:10AB50009507A607B70708F058CFE0CFCF93DF934C
:10AB6000EC0140E050E060E070E02EDF882361F00F
:10AB7000CE0161E0ABDEFC01009731F085EE808311
:10AB80001B820E94CF6401C080E0DF91CF910895C5
:10AB90002F923F924F925F926F927F928F929F92ED
:10ABA000AF92BF92CF92DF92EF92FF920F931F93DB
:10ABB000CF93DF93EC012A018B81882309F4B6C07F
:10ABC000898180FFB3C0C8C025014E185F083B01D2
:10ABD00074E0272E312C2C0E3D1E4201A1C0288589
:10ABE00039854A855B856FEFA62E61E0B62EA222DD
:10ABF000B3228B8179018A0199E016950795F79424
:10AC0000E7949A95D1F7E98DFA8D823049F4428D17
:10AC1000538D648D758D4E0D5F1D601F711F3FC07C
:10AC2000D480DA94DE20A114B104D9F4DD20C9F473
:10AC3000211531054105510549F48D899E89AF895A
:10AC4000B88D8C839D83AE83BF830BC04C815D81A7
:10AC50006E817F81CF0191010E942D67882309F4C5
:10AC600065C0E98DFA8D4C815D816E817F81425096
:10AC7000504060407040058404C0440F551F661F5B
:10AC8000771F0A94D2F786859785A089B189480FE6
:10AC9000591F6A1F7B1F4D0D511D611D711D80E0E5
:10ACA00092E08A199B0984018815990508F48C01A2
:10ACB00082E00030180709F067C08091990B9091ED
:10ACC0009A0BA0919B0BB0919C0B481759076A07F0
:10ACD0007B0709F459C080919D0D90919E0D9301C1
:10ACE0000E94356B882349F421C095012356344FC7
:10ACF000C301B901A8010E94850B600E711E980165
:10AD000040E050E088859985AA85BB85820F931F16
:10AD1000A41FB51F88879987AA87BB87801A910AC5
:10AD20008114910409F05BCFA20102C04FEF5FEFE5
:10AD3000CA01DF91CF911F910F91FF90EF90DF90AB
:10AD4000CF90BF90AF909F908F907F906F905F90CB
:10AD50004F903F902F900895A988BA88CB88DC88BF
:10AD6000E884F9840A851B859A0140E050E0D60109
:10AD7000C5018E199F09A00BB10B281739074A0787
:10AD80005B0708F021CF23CFCB01BA0140E00E943E
:10AD90000865882309F0A9CFC9CF0F931F93CF93DC
:10ADA000DF938C01EB01FC018381823018F18085F7
:10ADB0009185A285B3858F719070A070B070009757
:10ADC000A105B105B9F4C801BE0140E250E0E0DEE2
:10ADD0008032910519F0892B69F40EC0888188238F
:10ADE00059F0853E81F38E3271F38B8583FDEBCF75
:10ADF00080E203C08FEF01C080E0DF91CF911F910F
:10AE00000F910895DF93CF930F92CDB7DEB7BE01B8
:10AE10006F5F7F4F41E050E0BBDE019719F02FEFED
:10AE20003FEF03C08981282F30E0C9010F90CF91F7
:10AE3000DF910895EF92FF920F931F93CF93DF93CB
:10AE4000EC018B81823030F1E884F9840A851B851E
:10AE5000CE01D8DF97FD1EC088859985AA85BB8560
:10AE60004F96A11DB11D88879987AA87BB87F5E0FA
:10AE700016950795F794E794FA95D1F72E2D30E0C3
:10AE80002F703070E5E0220F331FEA95E1F723566B
:10AE9000344F02C020E030E0C901DF91CF911F9113
:10AEA0000F91FF90EF9008950F931F93CF93DF932F
:10AEB000EC018B018B81882309F040C0FB0187895D
:10AEC000803109F041C082E08B831D8A1E8A1F8A6F
:10AED000188E808D918DA0E0B0E025E0880F991F3D
:10AEE000AA1FBB1F2A95D1F7898B9A8BAB8BBC8B82
:10AEF00013C083E08B83F801428D538D648D758D73
:10AF00004D8B5E8B6F8B788F9E012F5E3F4FC801FC
:10AF10000E94FE67882391F01A8F098F81E0898350
:10AF20001C821D821E821F82188619861A861B8625
:10AF30001C861D861E861F86188A01C080E0DF9150
:10AF4000CF911F910F9108958032C1F7D2CF1F93F7
:10AF5000CF93DF93EC01142F262F30E0F90155E059
:10AF6000EE0FFF1F5A95E1F7E356F44F8385817189
:10AF700021F0842F827109F067C08091990B909124
:10AF80009A0BA0919B0BB0919C0B8C879D87AE87F1
:10AF9000BF87688BF90145E0EE0FFF1F4A95E1F787
:10AFA000E356F44F84899589A0E0B0E0DC0199274D
:10AFB00088278D8B9E8BAF8BB88F228D338DA90107
:10AFC00060E070E0482B592B6A2B7B2B4D8B5E8BFE
:10AFD0006F8B788F838590E088719070009751F423
:10AFE000848D958DA68DB78D898B9A8BAB8BBC8B01
:10AFF00081E00CC0409741F59E012F5E3F4F898D47
:10B000009A8D0E94FE678823F9F084E08B83812F5C
:10B010008F7089831C821D821E821F82188619866A
:10B020001A861B8614FF16C0CE0140E050E060E097
:10B0300070E0CADC882371F409C049895A896B8998
:10B040007C89CE019ADB02C01B8280E0DF91CF9128
:10B050001F91089515FDF1CF81E0F8CFCF93DF93D5
:10B06000EC019C012C5F3F4F898D9A8D41E050E0AF
:10B0700060E070E00E9469688823A1F08D899E8954
:10B08000AF89B88D0097A105B10559F48C819D81D8
:10B09000AE81BF818D8B9E8BAF8BB88F898180688D
:10B0A000898381E0DF91CF9108952F923F924F9253
:10B0B0005F927F928F929F92AF92BF92CF92DF92D8
:10B0C000EF92FF920F931F93DF93CF9300D000D0A6
:10B0D00000D0CDB7DEB76C01162F072F5E834D83EE
:10B0E000DC0113968C911397813009F06CC1119695
:10B0F0008C9181FF68C185C1F601418952896389BC
:10B10000748980859185A285B38584179507A607E4
:10B11000B70729F0C60131DB882309F454C1812F18
:10B12000902F9C0119014D805E8012C1D601599665
:10B13000ED91FC915A97DA01C90149E0B695A795BE
:10B14000979587954A95D1F774807A9478228FEFF6
:10B15000882E81E0982E82229322772009F052C017
:10B160008114910409F04EC0D60114964D915D9161
:10B170006D917C911797411551056105710581F419
:10B1800055968D919D910D90BC91A02D0097A10594
:10B19000B10561F1F60184839583A683B78332C03C
:10B1A000CF019E012F5F3F4F0E942D67882309F436
:10B1B0000AC129813A814B815C81D6015996ED9172
:10B1C000FC915A978789803149F4283FBFEF3B07AC
:10B1D000B0E04B07B0E05B0770F008C0283FEFEF2E
:10B1E0003E07EFEF4E07EFE05E0728F0C60136DFBF
:10B1F000882341F4E8C0D60114962D933D934D93D6
:10B200005C93179780E092E08819990952018415A0
:10B21000950508F45C01D6015996ED91FC915A9779
:10B220001496ED90FD900D911C9117978EEF9FEF66
:10B23000AFEFBFEFE80EF91E0A1F1B1F058404C005
:10B24000EE0CFF1C001F111F0A94D2F7868597850C
:10B25000A089B189E80EF91E0A1F1B1FE70CF11C1B
:10B26000011D111D90E0A91692E0B90639F58091F3
:10B27000990B90919A0BA0919B0BB0919C0B8E1502
:10B280009F05A007B10771F410929F0D8FEF9FEFFC
:10B29000AFEFBFEF8093990B90939A0BA0939B0B0A
:10B2A000B0939C0B80919D0D90919E0DB801A701CC
:10B2B00091010E94606A8823B9F585C081149104C8
:10B2C00019F5D60118962D913D914D915C911B97E2
:10B2D00051968D919D910D90BC91A02D2817390705
:10B2E0004A075B0788F00E94CF64882309F46BC08B
:10B2F00081E080939F0DE092990BF0929A0B00935E
:10B300009B0B10939C0B08C0C801B70141E00E9441
:10B310000865882309F457C094012356344FC901A6
:10B32000B101A5010E94850B950140E050E0F601B6
:10B3300080859185A285B385820F931FA41FB51FB9
:10B3400080879187A287B3872A0C3B1C4A185B0829
:10B35000D60118962D913D914D915C911B9741140A
:10B36000510409F0E3CE51968D919D910D90BC91C1
:10B37000A02D82179307A407B50748F4F601218B87
:10B38000328B438B548B81818068818311C0809183
:10B39000970B9091980B892B59F08D819E81892B69
:10B3A00039F0D60111968C911197806811968C9383
:10B3B000F601818183FF04C0C601A9DA882319F050
:10B3C0004D815E8105C081E0D6018C934FEF5FEF28
:10B3D000CA0126960FB6F894DEBF0FBECDBFCF913F
:10B3E000DF911F910F91FF90EF90DF90CF90BF9072
:10B3F000AF909F908F907F905F904F903F902F9055
:10B40000089582FD79CE8BCEDF92EF92FF920F935B
:10B410001F93CF93DF93EC0189899A89AB89BC890B
:10B42000805E9F4FAF41B04008F070C0CE0116DE85
:10B43000882309F46BC00E94CF64882309F466C096
:10B44000E98DFA8DEC80FD800E811F818EEF9FEFDC
:10B45000AFEFBFEFE80EF91E0A1F1B1F058404C0E3
:10B46000EE0CFF1C001F111F0A94D2F786859785EA
:10B47000A089B189E80EF91E0A1F1B1F81E0809385
:10B480009F0DE092990BF0929A0B00939B0B1093F7
:10B490009C0B80E092E0EDE9FBE0DF019C011D9256
:10B4A00021503040E1F7DD24D39411C0B801A70149
:10B4B0004D0D511D611D711D80919D0D90919E0D31
:10B4C0002DE93BE00E94606A882301F1D394E98D65
:10B4D000FA8D8481D81650F320E032E040E050E04D
:10B4E000058404C0220F331F441F551F0A94D2F74E
:10B4F00089899A89AB89BC89820F931FA41FB51FC4
:10B50000898B9A8BAB8BBC8B81E001C080E0DF9193
:10B51000CF911F910F91FF90EF90DF9008958F9240
:10B520009F92AF92BF92CF92DF92EF92FF920F93D2
:10B530001F93CF93DF936C01EB01942E852EA22EE7
:10B54000898D9A8DD6015A969C938E935997CB01EB
:10B5500040E050E060E070E010D9BB2437C0CE017D
:10B5600069DCFC01009709F490C055E01695079539
:10B57000F794E7945A95D1F71E2D1F708081882388
:10B5800011F0853EC9F4BB2099F42091990B3091BC
:10B590009A0B40919B0B50919C0BD6011C962D93BE
:10B5A0003D934D935C931F9750961C93BB24B3948B
:10B5B0008081882359F418C0892D982DBF014BE054
:10B5C00050E00E94780B009709F46DC0E884F9847C
:10B5D0000A851B8589899A89AB89BC89E816F90691
:10B5E0000A071B0708F4BBCFA6FE4FC0A1FE4DC043
:10B5F000BB2049F0F6011089C60161E067D9EC0172
:10B60000009761F442C08B81823009F43EC0CE01C4
:10B61000FBDE8823D1F110E0CDE9DBE080E2DE0142
:10B620001D928A95E9F7DE01292D382DC901FC010B
:10B630008BE001900D928150E1F7E091970BF09132
:10B64000980B309739F0BE01625F7F4FCE01409674
:10B65000099508C081E298E2998B888B80E098E098
:10B660009F878E87888999899B8B8A8B998F888FF2
:10B670008E859F859F8B8E8B0E94CF64882329F0B7
:10B68000C601612F4A2D63DC01C080E0DF91CF91BC
:10B690001F910F91FF90EF90DF90CF90BF90AF90F0
:10B6A0009F908F900895A7FEEBCFEFCF2F923F9200
:10B6B0004F925F926F927F928F929F92AF92BF92C2
:10B6C000CF92DF92EF92FF920F931F93DF93CF936E
:10B6D000CDB7DEB7C654D0400FB6F894DEBF0FBE6C
:10B6E000CDBF3C016B01DE01AE5BBF4F11965C9399
:10B6F0004E9325962FAF25971C861F861FA21AA64C
:10B700006115710509F47CC0FC018381882309F06F
:10B7100077C0FA0180818F32F1F08601ECE0EE2EE5
:10B72000F12CEC0EFD1E72E4A72EB12CAC0EBD1E4A
:10B730004E010894811C911C2796FFAEEEAE279710
:10B7400067E2262E312C2C0E3D1E270123C01196B8
:10B75000B183A08301C0FD01A081B1818C918F32A2
:10B76000B1F3D60113968C91139782508230A8F2D0
:10B770008E01095D1F4F59966D917C915A97C801B2
:10B7800093DB882359F63CC0342D252D8701832F68
:10B79000922F7C01F50180819181B401A5010E9465
:10B7A0006F53882329F42CC03196D501ED93FC9377
:10B7B000D501ED91FC9180818F32B1F38823B9F0EE
:10B7C000C701B801A40121E0AADE8823C9F00C1545
:10B7D0001D0511F0C801E8D82796EEADFFAD2797FB
:10B7E000EE16FF0689F6C101322D292FCFCFC301F6
:10B7F000B801A40125962FAD259791DE182F01C021
:10B8000010E0CE018796D9D8CE010C96D6D8812FDC
:10B81000CA5BDF4F0FB6F894DEBF0FBECDBFCF912E
:10B82000DF911F910F91FF90EF90DF90CF90BF902D
:10B83000AF909F908F907F906F905F904F903F90D0
:10B840002F9008950F931F93DF93CF93CDB7DEB75B
:10B850006B970FB6F894DEBF0FBECDBF9C01AB0156
:10B8600019821C828E010F5F1F4FC801B90122E0AF
:10B870001DDF882311F410E003C0C8016FD9182F11
:10B88000CE0101969AD8812F6B960FB6F894DEBF41
:10B890000FBECDBFCF91DF911F910F910895FC0195
:10B8A000148A178A138A2AEC32E0328B218B14AA6D
:10B8B00017AA13AA32AB21ABEE5AFF4F1082339670
:10B8C00010823497108232932293B196108233966D
:10B8D000108234971082329322937F9689E180837D
:10B8E00033961082789610823A96108233961082A0
:10B8F00034971082329322937E96108211821282A4
:10B90000138238961082118212821382E45DF04015
:10B91000118212821082E852FF4F81E08083E85D3D
:10B92000F040108A17860FB6F8948091A80D909178
:10B93000A90DA091AA0DB091AB0D0FBEE053FF4F22
:10B9400088579C4EAF4FBF4F80839183A283B383B0
:10B950000895FC01118212820895FC0182818823DE
:10B9600011F081E081830895FC01818181111182B0
:10B9700008950F931F938C010E9420300E94FD2F89
:10B98000F80111828EED91E00E94DD521F910F911E
:10B990000895FC018AEC92E091838083868188235C
:10B9A00019F0CF01039600C80895EF92FF920F930C
:10B9B0001F937C018C010F541F4FC8010E948754B4
:10B9C000C8010E94D454F70110821F910F91FF907B
:10B9D000EF900895CF92DF92EF92FF920F931F9313
:10B9E000CF93DF937C016B01DB010D900020E9F721
:10B9F0008D0101501040061B170BE1EBF0E0EE0E3D
:10BA0000FF1ED7011C92EFE4FFEFEE0EFF1ECB01ED
:10BA10006EE470E00E94990BEC01009731F4F8019C
:10BA20003197EC0DFD1D86010EC060E270E00E94B2
:10BA3000990B8C010F5F1F4FCE016AE270E00E94EC
:10BA4000990BFC0131978DE081838AE08283138218
:10BA5000C70182559F4FB8010E94545381EB90E07B
:10BA6000E80EF91ED7018C91882309F1EBE7FEE07F
:10BA70006491EF0107C08DEA9DE00E94E3112196D9
:10BA8000FE0164916623B9F7E2E8FEE06491EF01FC
:10BA900007C08DEA9DE00E94E3112196FE016491AA
:10BAA0006623B9F78DEA9DE06AE00E94E311DF9119
:10BAB000CF911F910F91FF90EF90DF90CF9008955D
:10BAC000EF92FF920F93CF93DF937C01FC01828171
:10BAD000882309F43FC0EAEAFEE06491EF0107C061
:10BAE0008DEA9DE00E94E3112196FE016491662398
:10BAF000B9F784ED90E0E80EF91EF701408151811D
:10BB0000628173818CE29FEFE80EF91E8DEA9DE061
:10BB10002AE000E00E94E670E8EAFEE06491EF01AE
:10BB200007C08DEA9DE00E94E3112196FE01649119
:10BB30006623B9F78CEC90E0E80EF91EF70140811E
:10BB40005181628173818DEA9DE02AE000E00E94CC
:10BB5000E6700EC0E8E9FEE06491EF0107C08DEAEF
:10BB60009DE00E94E3112196FE0164916623B9F7DE
:10BB70008DEA9DE06AE00E94E311DF91CF910F9181
:10BB8000FF90EF9008952F923F924F925F926F92A5
:10BB90007F928F929F92AF92BF92CF92DF92EF925D
:10BBA000FF920F931F93DF93CF93CDB7DEB7AC9780
:10BBB0000FB6F894DEBF0FBECDBF5C014B014CA7A2
:10BBC000FC018281882309F4A0C131EB432E512C62
:10BBD0004A0C5B1CC2010E94D454F5011182198ADF
:10BBE0001C8A188A8AEC92E09F878E87C50141964D
:10BBF00090AB87A7F40180818F3209F07FC0C40128
:10BC00006FE270E00E94990B7C010894E11CF11C2A
:10BC10003E010894611C711C21E1222E312C2C0E56
:10BC20003D1E67C0C7016FE270E00E94990B6C0176
:10BC3000009709F46BC0E816F90608F067C08C019C
:10BC40000E191F09C301B701A8010E94B90B060D07
:10BC5000171DF80110828DEA9DE0B3010E94333078
:10BC60008DEA9DE06AE00E94E311F50167A570A9E5
:10BC70006115710519F460E070E002C06D5F7F4FDF
:10BC8000C101A30121E012DD882341F5ECE5FFE0CD
:10BC900064917F0109C08DEA9DE00E94E311089440
:10BCA000E11CF11CF70164916623A9F78DEA9DE080
:10BCB000BE016F5F7F4F0E943330EAE5FFE0649181
:10BCC0007F0109C08DEA9DE00E94E3110894E11C08
:10BCD000F11CF70164916623A9F70FC12EE030E053
:10BCE0002C0F3D1FF50130AB27A776010894E11C0E
:10BCF000F11CE114F10409F095CF05C0C501C1960E
:10BD0000F50190AB87A7082DD92C02C00E2DDF2C92
:10BD1000F50167A570A9FCA5FF2309F4A0C0611572
:10BD2000710519F460E070E002C06D5F7F4FC201E1
:10BD3000402F5D2D21E0BADC882309F469C0A501FC
:10BD400044535F4F22EC30E0A20EB31EF501808118
:10BD50009181A281B3812EE33FEFA20EB31EFA01BF
:10BD600080839183A283B383EDE4FFE064917F013C
:10BD700009C08DEA9DE00E94E3110894E11CF11CCA
:10BD8000F70164916623A9F78DEA9DE0602F7D2D70
:10BD90000E943330E6E4FFE064917F0109C08DEA40
:10BDA0009DE00E94E3110894E11CF11CF7016491ED
:10BDB0006623A9F72CEC30E0A20EB31EF5014081FA
:10BDC0005181628173818DEA9DE02AE000E00E944A
:10BDD000E6708DEA9DE06AE00E94E31128E030E021
:10BDE000A20EB31EF5011082118212821382E8E3C3
:10BDF000FFE064917F0109C08DEA9DE00E94E3119C
:10BE00000894E11CF11CF70164916623A9F775C041
:10BE1000E4E2FFE064917F0109C08DEA9DE00E94A9
:10BE2000E3110894E11CF11CF70164916623A9F762
:10BE30008DEA9DE0602F7D2D0E943330E2E2FFE02D
:10BE400064917F0109C08DEA9DE00E94E31108948E
:10BE5000E11CF11CF70164916623A9F74EC061153E
:10BE6000710519F460E070E002C06D5F7F4FC201A0
:10BE7000402F5D2D26E51ADC882339F5EEE0FFE042
:10BE800064917F0109C08DEA9DE00E94E31108944E
:10BE9000E11CF11CF70164916623A9F78DEA9DE08E
:10BEA000602F7D2D0E943330ECE0FFE064917F0134
:10BEB00009C08DEA9DE00E94E3110894E11CF11C89
:10BEC000F70164916623A9F718C081E0F50180832A
:10BED000EAEFFEE064917F0109C08DEA9DE00E94D7
:10BEE000E3110894E11CF11CF70164916623A9F7A2
:10BEF0008DEA9DE0B4010E9433308DEA9DE06AE056
:10BF00000E94E311CE010E9644DDAC960FB6F89474
:10BF1000DEBF0FBECDBFCF91DF911F910F91FF907C
:10BF2000EF90DF90CF90BF90AF909F908F907F90D9
:10BF30006F905F904F903F902F9008952F923F9277
:10BF40004F925F926F927F928F929F92AF92BF9229
:10BF5000CF92DF92EF92FF920F931F93DF93CF93D5
:10BF6000CDB7DEB7AB970FB6F894DEBF0FBECDBF2F
:10BF70005C014B01FC018281882309F4FDC0C501ED
:10BF80008F549F4F0E94D454F5011182198A1C8A44
:10BF9000188A8AEC92E09F878E87C501419690AB04
:10BFA00087A7F40180818F3209F080C0C4016FE25D
:10BFB00070E00E94990B7C010894E11CF11C3E0189
:10BFC0000894611C711C5EE0252E312C2C0E3D1E48
:10BFD00041E1442E512C4C0E5D1E63C0C7016FE23F
:10BFE00070E00E94990B6C01009709F467C0E81695
:10BFF000F90608F063C08C010E191F09C301B701CF
:10C00000A8010E94B90B060D171DF80110828DEAD8
:10C010009DE0B3010E9433308DEA9DE06AE00E940A
:10C02000E311F50167A570A96115710519F460E0C8
:10C0300070E002C06D5F7F4FC201A30121E036DBDB
:10C04000882341F5E6EEFEE064917F0109C08DEAA8
:10C050009DE00E94E3110894E11CF11CF70164913A
:10C060006623A9F78DEA9DE0BE016F5F7F4F0E94B6
:10C070003330E4EEFEE064917F0109C08DEA9DE07B
:10C080000E94E3110894E11CF11CF70164916623FE
:10C09000A9F76AC0F50130AA27A676010894E11C29
:10C0A000F11CE114F10409F099CF05C0C501C19656
:10C0B000F50190AB87A7D82C092D02C0DE2C0F2DDF
:10C0C000F50187A590A9009719F480E090E001C0E0
:10C0D00003966D2D702FB6DB882301F1E6EDFEE0AF
:10C0E00064917F0109C08DEA9DE00E94E3110894EC
:10C0F000E11CF11CF70164916623A9F78DEA9DE02C
:10C100006D2D702F0E94333084ED90E0A80EB91E83
:10C11000F50110821182128213822BC0EEEBFEE039
:10C1200064917F0109C08DEA9DE00E94E3110894AB
:10C13000E11CF11CF70164916623A9F78DEA9DE0EB
:10C140006D2D702F0E943330ECEBFEE064917F0187
:10C1500009C08DEA9DE00E94E3110894E11CF11CE6
:10C16000F70164916623A9F78DEA9DE06AE00E94D9
:10C17000E311CE010E960DDCAB960FB6F894DEBF40
:10C180000FBECDBFCF91DF911F910F91FF90EF9028
:10C19000DF90CF90BF90AF909F908F907F906F90E7
:10C1A0005F904F903F902F900895EF92FF920F93E2
:10C1B0001F93CF93DF937C01FC0112828789882330
:10C1C00021F0C70144960E94D454870105571F4FA0
:10C1D000C80160E04AE10E94666B8823E9F4E0E66A
:10C1E000FEE06491EF0107C08DEA9DE00E94E3113B
:10C1F0002196FE0164916623B9F7E6ECFFE06491B5
:10C20000EF0107C08DEA9DE00E94E3112196FE0137
:10C2100064916623B9F76FC0E701C057DF4FCE01C5
:10C22000B80141E02FD4882319F5CE01B80140E0D0
:10C2300029D48823E9F4EBE7FEE06491EF0107C01D
:10C240008DEA9DE00E94E3112196FE016491662330
:10C25000B9F7E3EBFFE06491EF0107C08DEA9DE0E1
:10C260000E94E3112196FE0164916623B9F743C051
:10C27000C7014496BE010E9454578823E9F4EBE7B6
:10C28000FEE06491EF0107C08DEA9DE00E94E3119A
:10C290002196FE0164916623B9F7E3EAFFE0649119
:10C2A000EF0107C08DEA9DE00E94E3112196FE0197
:10C2B00064916623B9F71FC081E0F7018283E0E64D
:10C2C000FEE06491EF0107C08DEA9DE00E94E3115A
:10C2D0002196FE0164916623B9F7E8E9FFE06491D5
:10C2E000EF0107C08DEA9DE00E94E3112196FE0157
:10C2F00064916623B9F78DEA9DE06AE00E94E3113C
:10C30000C7014196F70190AB87A7C701C49620E902
:10C3100030E0E20EF31EB7010E945457882399F4CF
:10C32000E4E8FFE06491EF0107C08DEA9DE00E9420
:10C33000E3112196FE0164916623B9F78DEA9DE031
:10C340006AE00E94E311DF91CF911F910F91FF905E
:10C35000EF9008952F923F924F925F927F928F922B
:10C360009F92AF92BF92CF92DF92EF92FF920F9384
:10C370001F93DF93CF93CDB7DEB7CC55D0400FB628
:10C38000F894DEBF0FBECDBF7C01662359F528EDC2
:10C3900030E0E20EF31ED7018C91E8E2FFEFEE0EE3
:10C3A000FF1E882309F4F2C00FB6F8942091A80D5F
:10C3B0003091A90D4091AA0D5091AB0D0FBE60EDCB
:10C3C00070E0E60EF71EF70180819181A281B381B2
:10C3D00060E37FEFE60EF71E82179307A407B50709
:10C3E00008F4D4C088ED90E0E80EF91ED7011C9245
:10C3F000E8E2FFEFEE0EFF1ED70112968C91882324
:10C4000039F4C701D2DEF7018281882309F4BEC066
:10C4100000D000D000D0EDB7FEB731968E010F5F8F
:10C420001F4FADB7BEB712961C930E9311978AEEAD
:10C4300091E093838283D7011F968D919C915097B1
:10C44000958384830E94E20BCC24DD24EDB7FEB7F4
:10C4500036960FB6F894FEBF0FBEEDBF58010AC066
:10C46000D8018C91992787FD90950E947F79F801DA
:10C4700081938F01C601F50101900020E9F7319702
:10C48000EA19FB090894C11CD11C8E179F0744F3BD
:10C49000E4E18E2E912C8E0C9F1CC40140E050E0F4
:10C4A00060E070E00E94BD5377247DE3A72EB12C9D
:10C4B000AC0EBD1E1E010894211C311C6FE1462EDE
:10C4C000512C4C0E5D1E48C0D6018C9190E00E940C
:10C4D0007F79F60181936F01C801F5010190002079
:10C4E000E9F73197EA19FB090F5F1F4F8E179F0776
:10C4F0005CF327968FAD27978E3771F1C501B10197
:10C5000045E050E00E94AB0B009731F500D000D021
:10C5100000D0EDB7FEB73196ADB7BEB712965C92BC
:10C520004E92119723EF31E03383228335822482A8
:10C530000E94E20B6DB77EB76A5F7F4F0FB6F8942B
:10C540007EBF0FBE6DBFC2010E94DD528AEF91E037
:10C550000E94DD5277247394C401B5010E94CD5628
:10C56000181624F4650100E010E0B6CF772041F4FE
:10C570008FEF9FEFD70150969C938E931F9706C025
:10C58000F701878590890196908B8787C45ADF4F82
:10C590000FB6F894DEBF0FBECDBFCF91DF911F91D4
:10C5A0000F91FF90EF90DF90CF90BF90AF909F9052
:10C5B0008F907F905F904F903F902F9008952F9293
:10C5C0003F924F925F926F927F928F929F92AF9223
:10C5D000BF92CF92DF92EF92FF920F931F93DF9360
:10C5E000CF93CDB7DEB7CB58D0400FB6F894DEBFAF
:10C5F0000FBECDBF6C012B015A0183E090E0A80E65
:10C60000B91EF6013396CC57DF4FF983E883C4583F
:10C61000D040CA57DF4F1882C658D04014E6E12EEA
:10C62000F12CEC0EFD1EC7010B96C957DF4F998305
:10C630008883C758D040B9ED6B2E712C6C0C7D1CD3
:10C64000ABED8A2E912C8C0C9D1CF6E42F2E312CF8
:10C650002C0E3D1EF1013396C757DF4FF983E88357
:10C66000C958D040E0E6FEE08491C557DF4F88838B
:10C67000CB58D04023C1F7018385482F50E0BA0141
:10C68000687170706031710509F020C1F30120817B
:10C6900031812130310509F419C12230310509F405
:10C6A00015C1F701DE0111969081903239F08E2F7D
:10C6B0008E19883011F48EE28D939D933196C9576F
:10C6C000DF4F88819981C758D040E817F90761F793
:10C6D0001C921E86F2018081882331F4CE010E96D1
:10C6E0006EEF71E00E948E0BCE010E96B2010E9499
:10C6F0008E0BCE010E96BE016F5F7F4F0E948E0B98
:10C70000CE010E966EEF71E00E948E0B1BA61EA648
:10C710001AA68AEC92E099A788A7CE018B96B5015C
:10C72000AE014F5F5F4F21E00E94565B882371F599
:10C73000F30180819181892B49F5C557DF4F6881CD
:10C74000CB58D04000E61EE008C08DEA9DE00E9474
:10C75000E3110F5F1F4FF80164916623B1F78DEA73
:10C760009DE060E072E00E9433308DEA9DE06AE077
:10C770000E94E3118DEA9DE0BE016F5F7F4F0E9432
:10C7800033308DEA9DE06AE00E94E311C757DF4F26
:10C79000A881B981C958D040FE01BB968BE10190B8
:10C7A0000D928150E1F78AA5F10182838AEC92E033
:10C7B00091838083C601BE01625F7F4FA101FFDECE
:10C7C000C101E7D8CE018896E4D878C0953E09F437
:10C7D00075C09E3209F472C09F3509F46FC043FDE5
:10C7E0006DC080E06031710509F481E0F601868753
:10C7F000882349F4F7018085873409F05FC081857B
:10C800008E3709F45BC0CC57DF4FA881B981C4587B
:10C81000D040F7018081803241F08E2F8E19883010
:10C8200011F48EE28D9380818D933196C957DF4F3D
:10C8300088819981C758D040E817F90759F71C92A9
:10C84000F301808191810097A9F48DEA9DE0B20106
:10C850000E9433308DEA9DE0CC57DF4F68817981AB
:10C86000C458D0400E9433308DEA9DE06AE00E94B7
:10C87000E31124C08130910539F4F4018081918164
:10C880000196918380831AC00297C1F4CA57DF4F83
:10C89000F881C658D0402F2F30E0F401808191817B
:10C8A00028173907C1F0CA57DF4FF881C658D04062
:10C8B000FF5FCA57DF4FF883C658D040C501B701A4
:10C8C0000E94CD5618160CF4D6CE05C0F701908103
:10C8D000992309F07BCFC557DF4F0FB6F894DEBF21
:10C8E0000FBECDBFCF91DF911F910F91FF90EF90C1
:10C8F000DF90CF90BF90AF909F908F907F906F9080
:10C900005F904F903F902F900895EF92FF920F937A
:10C910001F93DF93CF93CDB7DEB76E970FB6F89422
:10C92000DEBF0FBECDBF7C0189ED90E0E80EF91EA1
:10C93000F7011182108287E29FEFE80EF91E87014E
:10C940000C5E1F4FC80140E050E060E070E00E94C4
:10C95000BD53DE011496F8018BE101900D928150D8
:10C96000E1F7F70183898B838AEC92E09A838983CC
:10C97000C70163E172E08E010F5F1F4FA8011FDE48
:10C98000C80107D86E960FB6F894DEBF0FBECDBFB4
:10C99000CF91DF911F910F91FF90EF9008958091BB
:10C9A0009F0D882389F14091990B50919A0B6091CA
:10C9B0009B0B70919C0B80919D0D90919E0D2DE98C
:10C9C0003BE07ED5882311F14091A00D5091A10D3F
:10C9D0006091A20D7091A30D41155105610571057E
:10C9E00089F080919D0D90919E0D2DE93BE068D5D9
:10C9F000882361F01092A00D1092A10D1092A20D4B
:10CA00001092A30D10929F0D81E0089580E008958B
:10CA1000DF92EF92FF920F931F937B018C01D42E34
:10CA20008091990B90919A0BA0919B0BB0919C0BCC
:10CA30008E159F05A007B107B1F0B1DF8823D9F0AB
:10CA400080919D0D90919E0DB801A7012DE93BE0CD
:10CA50000CD6882381F0E092990BF0929A0B009308
:10CA60009B0B10939C0BDD2011F481E005C081E04D
:10CA700080939F0D01C080E01F910F91FF90EF9078
:10CA8000DF9008958F929F92AF92BF92CF92DF92E4
:10CA9000EF92FF920F931F93CF93DF936C01142FAC
:10CAA00070939E0D60939D0DFC01178A82E090E0CB
:10CAB000A0E0B0E080839183A283B38310929F0DA6
:10CAC0001092A00D1092A10D1092A20D1092A30D24
:10CAD0008FEF9FEFAFEFBFEF8093990B90939A0B7F
:10CAE000A0939B0BB0939C0B442321F4882499249E
:10CAF00054013FC0453008F01CC160E070E080E0A8
:10CB000090E040E085DF882309F413C1C12FD0E015
:10CB10002197FE0174E0EE0FFF1F7A95E1F7E356CF
:10CB2000F44FE254FE4F8081EE5BF14090E08F774E
:10CB30009070892B09F0FDC0E653FE4F80819181F2
:10CB4000A281B38184369105A105B10508F4F1C035
:10CB500064E0CC0FDD1F6A95E1F7CD59D24F888094
:10CB60009980AA80BB8081149104A104B10409F4C6
:10CB7000E0C0C501B40140E04BDF882309F4D9C00F
:10CB80008091A80B9091A90B8050924009F0D1C0E0
:10CB90002091AD0B222309F4CCC08091AB0B909176
:10CBA000AC0B892B09F4C5C08091AA0B882309F42A
:10CBB000C0C0F601228B8091AA0B8483158661E0A8
:10CBC00070E007C04F5FF60145874150483008F0DC
:10CBD000B0C0F6014585848190E09B01042E02C01F
:10CBE000220F331F0A94E2F78217930759F7209117
:10CBF000B30B3091B40B2115310519F040E050E032
:10CC000008C02091C10B3091C20B4091C30B5091D1
:10CC1000C40BF6012583368347835087E090AB0B26
:10CC2000F090AC0B00E010E0E80CF91C0A1D1B1D95
:10CC3000E38AF48A058B168B8091AE0B9091AF0B33
:10CC4000918F808F6091AD0B70E080E090E00E944A
:10CC5000EE786E0D7F1D801F911FF601628F738F1E
:10CC6000848F958F2091AE0B3091AF0B55E0220F42
:10CC7000331F5A95E1F721503E4F232F3327269536
:10CC800040E050E0260F371F481F591F268737877F
:10CC9000408B518B8091B00B9091B10B009719F0A4
:10CCA000A0E0B0E008C08091BD0B9091BE0BA091B8
:10CCB000BF0BB091C00B85017401E21AF30A040B9B
:10CCC000150BA8019701280F391F4A1F5B1FF6019A
:10CCD000058404C056954795379527950A94D2F751
:10CCE0002187328743875487253FFFE03F07F0E0E5
:10CCF0004F07F0E05F0720F48CE0F601878B19C046
:10CD0000255F3F4F4040504018F480E1F6010EC0CF
:10CD10008091C90B9091CA0BA091CB0BB091CC0B19
:10CD2000F601828F938FA48FB58F80E2878B81E08D
:10CD300001C080E0DF91CF911F910F91FF90EF90A4
:10CD4000DF90CF90BF90AF909F908F9008956F929B
:10CD50007F928F929F92AF92BF92CF92DF92EF928B
:10CD6000FF920F931F93CF93DF93EC015A016B0156
:10CD700038014901423051056105710508F45DC073
:10CD800089859A85AB85BC850196A11DB11D841747
:10CD90009507A607B70708F450C08F89803129F49A
:10CDA000E52EF62E072F11270CC0803209F045C062
:10CDB0007A018B0187E016950795F794E7948A9599
:10CDC000D1F78B899C89AD89BE89E80EF91E0A1FAF
:10CDD0001B1FC801B70141E01BDE882371F18F8959
:10CDE000803149F4F501F070EE0FFF1FE356F44F68
:10CDF000718260820DC0F501EF77F070EE0FFF1FBA
:10CE0000EE0FFF1FE356F44F60827182828293829D
:10CE10008A89823080F08D819E81AF81B885E80E4D
:10CE2000F91E0A1F1B1FE092A00DF092A10D0093A6
:10CE3000A20D1093A30D81E001C080E0DF91CF919E
:10CE40001F910F91FF90EF90DF90CF90BF90AF9028
:10CE50009F908F907F906F900895CF92DF92EF9286
:10CE6000FF920F931F93CF93DF93EC017A018B0115
:10CE7000690189859A85AB85BC850196A11DB11D87
:10CE800084179507A607B70708F452C08F89803129
:10CE900029F45527412F302F2F2D0CC0803209F057
:10CEA00047C09A01AB0167E056954795379527959E
:10CEB0006A95D1F78B899C89AD89BE89280F391F66
:10CEC0004A1F5B1F8091990B90919A0BA0919B0B2D
:10CED000B0919C0B281739074A075B0731F0CA014C
:10CEE000B90140E095DD882319F18F89803159F42B
:10CEF000F701F070EE0FFF1FE356F44F8081918130
:10CF0000A0E0B0E00EC0F701EF77F070EE0FFF1F6A
:10CF1000EE0FFF1FE356F44F80819181A281B38110
:10CF2000BF70F60180839183A283B38381E001C047
:10CF300080E0DF91CF911F910F91FF90EF90DF90F4
:10CF4000CF900895AF92BF92CF92DF92EF92FF926F
:10CF50000F931F93DF93CF9300D000D0CDB7DEB7F0
:10CF60006C017A018B0182E090E0A0E0B0E0F60174
:10CF700080839183A283B3835E010894A11CB11CBA
:10CF8000C601B801A701950168DF882339F1C60100
:10CF9000B801A70100E010E020E030E0D8DE8823EF
:10CFA000E9F0E980FA800B811C81F60187898031E4
:10CFB00051F4F8EFEF16FFEFFF06F0E00F07F0E097
:10CFC0001F07F0F209C088EFE8168FEFF8068FEF21
:10CFD00008078FE01807A0F281E001C080E00F9001
:10CFE0000F900F900F90CF91DF911F910F91FF90B5
:10CFF000EF90DF90CF90BF90AF9008954F925F92E7
:10D000006F927F928F929F92AF92BF92CF92DF9258
:10D01000EF92FF920F931F93DF93CF9300D000D036
:10D02000CDB7DEB76C0149835A836B837C833901AA
:10D03000EE24FF2487012E010894411C511C812CF1
:10D04000E2E09E2EA12CB12C49815A816B817C811A
:10D05000C601920102DF882339F1D501C401F6012E
:10D06000058404C0880F991FAA1FBB1F0A94D2F71A
:10D07000E80EF91E0A1F1B1F29813A814B815C8132
:10D080008789803131F4285F3F4F40405040E0F2C3
:10D0900005C0285F3F4F4F4F5F40B0F2F301E08281
:10D0A000F1820283138381E00F900F900F900F9015
:10D0B000CF91DF911F910F91FF90EF90DF90CF9074
:10D0C000BF90AF909F908F907F906F905F904F90A8
:10D0D00008952F923F924F925F926F927F928F921C
:10D0E0009F92AF92BF92CF92DF92EF92FF920F93F7
:10D0F0001F93DF93CF93CDB7DEB72F970FB6F8947A
:10D10000DEBF0FBECDBF1C014A875B876C877D8762
:10D110003F872E87DC0119968D919D910D90BC91D2
:10D12000A02D0196A11DB11D8E839F83A887B9876D
:10D13000F901008111812281338101151105210539
:10D14000310549F0480159010894811C911CA11C2A
:10D15000B11C1D8210C0D1018D909D90AD90BC90EE
:10D160001D828A859B85AC85BD850197A105B1058A
:10D1700011F491E09D83750164014424552432012A
:10D180008E010F5F1F4FF10181859285A385B485C4
:10D19000481659066A067B0608F08CC08E819F816E
:10D1A000A885B9858C159D05AE05BF0550F4A2E094
:10D1B0008A2E912CA12CB12CF2E0CF2ED12CE12C77
:10D1C000F12CC101B701A601980147DE882309F4BB
:10D1D00071C089819A81AB81BC81A70196012F5FC3
:10D1E0003F4F4F4F5F4F0097A105B10519F049011F
:10D1F0005A010DC0281939094A095B098A859B859E
:10D20000AC85BD85281739074A075B0759F0089494
:10D21000411C511C611C711C0894C11CD11CE11CD7
:10D22000F11CB1CFC101A601B7010FEF1FEF2FEF26
:10D230003FE08DDD882391F43DC02601370108943D
:10D240004108510861087108C101B301A2019701A9
:10D2500086017DDD882371F1730162018C149D04C8
:10D26000AE04BF0450F3AE85BF854D915D916D91C5
:10D270007C91411551056105710531F0C1019501A0
:10D28000840165DD8823B1F0EE85FF85808291827F
:10D29000A282B382FD81FF2359F00894811C911C66
:10D2A000A11CB11CD1018D929D92AD92BC9213979D
:10D2B00081E001C080E02F960FB6F894DEBF0FBE6C
:10D2C000CDBFCF91DF911F910F91FF90EF90DF9035
:10D2D000CF90BF90AF909F908F907F906F905F9016
:10D2E0004F903F902F900895FC014281242F30E011
:10D2F000C9019595879580658CBD40FF02C080E08F
:10D3000004C080E0463009F081E08DBD8081E82FC7
:10D31000F0E0CAC2DF92EF92FF920F931F93CF9378
:10D32000DF93EC01D62E79018A01DEDF0FB6F89487
:10D330008091A80D9091A90DA091AA0DB091AB0D6F
:10D340000FBE9C014FEF10C00FB6F8948091A80D4E
:10D350009091A90DA091AA0DB091AB0D0FBE821BAB
:10D36000930B8C52914038F44EBD0DB407FEFDCFA7
:10D370008EB58F3F49F78D2D80648EBD0DB407FEAD
:10D38000FDCF28E130E0D801C701022E04C0B695D8
:10D39000A795979587950A94D2F78EBD0DB407FE91
:10D3A000FDCF285030408FEF283F380761F7DD2050
:10D3B00011F485E906C058E0D51611F487E801C0DC
:10D3C0008FEF8EBD0DB407FEFDCF8CE0D81631F483
:10D3D0008FEF8EBD0DB407FEFDCF8EB59FEF2FEF03
:10D3E0002EBD0DB407FEFDCF8EB587FF04C0992377
:10D3F00011F09150F5CF8B83DF91CF911F910F9159
:10D40000FF90EF90DF900895BF92CF92DF92EF925E
:10D41000FF920F931F938C01B62E69017A0167E387
:10D4200020E030E040E050E075DFC8016B2DA7013F
:10D43000960170DF1F910F91FF90EF90DF90CF90DA
:10D44000BF900895FC018081E82FF0E027C2DC0145
:10D450006EBDFA0120E030E00DB407FEFDCF808103
:10D460008EBD0DB407FEFDCF81818EBD2E5F3F4F77
:10D47000329682E02030380779F70DB407FEFDCFF1
:10D480008FEF8EBD0DB407FEFDCF8FEF8EBD0DB4B7
:10D4900007FEFDCF8FEF8EBD0DB407FEFDCF8EB51D
:10D4A00013968C9313978F71853011F481E0089552
:10D4B00083E111968C931197CD01C4DF80E008952C
:10D4C000CF92DF92EF92FF920F931F93CF93DF9350
:10D4D000EC017A018B0169018C81833039F059E0CC
:10D4E000EE0CFF1C001F111F5A95D1F7CE0168E109
:10D4F000A80197010FDF882311F086E036C0CE0126
:10D500006EEFA601A4DF882389F10FB6F89480910D
:10D51000A80D9091A90DA091AA0DB091AB0D0FBED1
:10D520009C014FEF10C00FB6F8948091A80D909118
:10D53000A90DA091AA0DB091AB0D0FBE821B930B4C
:10D540008855924040F44EBD0DB407FEFDCF1EB588
:10D550001F3F49F717C087E108C01EBD0DB407FE85
:10D56000FDCF8EB58823C1F086E18983CE016ADFC5
:10D5700080E0DF91CF911F910F91FF90EF90DF90AE
:10D58000CF900895CE016DE020E030E040E050E023
:10D59000C1DE882349F7E1CFCE0154DF81E0E9CF36
:10D5A000CF93DF93EC010FB6F8948091A80D909182
:10D5B000A90DA091AA0DB091AB0D0FBEFC013FEFDC
:10D5C00013C00FB6F8948091A80D9091A90DA09169
:10D5D000AA0DB091AB0D0FBE8E1B9F0B8D529140CB
:10D5E00018F02B8381E10BC03EBD0DB407FEFDCFCB
:10D5F0002EB52F3F31F32B832E3F31F08FE08983FF
:10D60000CE0120DF80E02EC0DA011197452BD9F042
:10D610008FEF8EBD20E030E09FEF0BC00DB407FE12
:10D62000FDCF8EB5FB01E20FF31F80839EBD2F5F00
:10D630003F4F2A173B0790F30DB407FEFDCF8EB581
:10D64000A60FB71F8C938FEF8EBD0DB407FEFDCFD5
:10D650008EB58FEF8EBD0DB407FEFDCF8EB5CE011A
:10D66000F1DE81E0DF91CF910895CF92DF92EF92CA
:10D67000FF920F931F93CF93DF93EC017A018B01FD
:10D6800069018C81833039F0A9E0EE0CFF1C001F8A
:10D69000111FAA95D1F7CE0161E1A80197013ADEE9
:10D6A000882331F084E08983CE01CCDE80E005C0A0
:10D6B000CE01B60140E052E073DFDF91CF911F91C0
:10D6C0000F91FF90EF90DF90CF900895BF92CF928F
:10D6D000DF92EF92FF920F931F93CF93DF93EC01B2
:10D6E000B62E842F1C82198248830FB6F89420919D
:10D6F000A80D3091A90D4091AA0D5091AB0D0FBE10
:10D700006901B8D0CE019EDE23982B98229A219AE7
:10D71000269A2E9A809180008F7D8093800085E0EC
:10D720008A8382E58CBD1DBC80E09FEF9EBD0DB459
:10D7300007FEFDCF8F5F8A30C9F712C00FB6F8948D
:10D740008091A80D9091A90DA091AA0DB091AB0D5B
:10D750000FBE8C199D09815D974010F081E05BC080
:10D76000CE0160E020E030E040E050E0D3DD182F53
:10D770008B83813019F7CE0168E02AEA31E040E07E
:10D7800050E0C8DD82FF02C01C8311C080E02FEF93
:10D790002EBD0DB407FEFDCF9EB58F5F8430C1F75F
:10D7A0009B839A3A11F082E036C082E08C838C81B0
:10D7B000823021F0EE24FF24870118C0E12CF12CE7
:10D7C000012D00E4102F12C00FB6F8948091A80D1F
:10D7D0009091A90DA091AA0DB091AB0D0FBE8C191F
:10D7E0009D09815D974010F08AE015C0CE0169E285
:10D7F000A801970109DE8B83882331F78C81823061
:10D8000019F5CE016AE320E030E040E050E082DD2F
:10D81000882329F088E08983CE0114DE20C08FEFB1
:10D820008EBD0DB407FEFDCF8EB5807C803C11F41B
:10D8300083E08C8380E09FEF9EBD0DB407FEFDCF9B
:10D840002EB58F5F8330C1F7CE01FCDD86E08B15EE
:10D8500018F488E1898303C0BA8281E001C080E0C6
:10D86000DF91CF911F910F91FF90EF90DF90CF90BC
:10D87000BF9008958E3270F4E3EDFFE0880FE80F5B
:10D88000F11D9591E491F0E02FB7F8948181892BF7
:10D8900081832FBF0895002039F000C0EE3250F48C
:10D8A000EE0FE55AF3490994EE3220F4EE0FE954F5
:10D8B000F34909940895589AB6C0599AD0C05A9A13
:10D8C00008955B9A08955C9A08955D9A08955E9A0A
:10D8D00008955F9A0895709A0895719A0895409AEC
:10D8E0000895419A0895429A0895439A0895449A52
:10D8F000C8C0459AC0C0469AB8C0479A0895769A5B
:10D900000895779A0895289A0895299A08952A9A49
:10D9100008952B9A08952C9A9CC02D9A88C02E9A0F
:10D920008CC02F9A90C0109A0895119A0895129A57
:10D930000895139A0895149A0895159A0895169AB9
:10D940000895179A0895749A0895759A0895889A73
:10D950000895899A08958A9A08958B9A08958C9AC1
:10D9600008958D9A08958E9A08958F9A08955898DB
:10D970005AC0599874C05A9808955B9808955C9855
:10D9800008955D9808955E9808955F980895709839
:10D99000089571980895409808954198089542987F
:10D9A00008954398089544986CC0459864C046987B
:10D9B0005CC04798089576980895779808952898B8
:10D9C0000895299808952A9808952B9808952C98D9
:10D9D00040C02D982CC02E9830C02F9834C010987D
:10D9E0000895119808951298089513980895149819
:10D9F000089515980895169808951798089574989D
:10DA000008957598089588980895899808958A9832
:10DA100008958B9808958C9808958D9808958E9800
:10DA200008958F980895E4B5EF7DE4BD0895E091E1
:10DA30008000EF77E09380000895E0918000EF7D13
:10DA4000E09380000895E0918000E77FE0938000FC
:10DA50000895E091B000EF77E093B0000895E09171
:10DA6000B000EF7DE093B0000895E0919000EF7773
:10DA7000E09390000895E0919000EF7DE093900096
:10DA80000895E0919000E77FE093900008951DBA1B
:10DA9000109268001CBC10BE1FBA10927A0010923F
:10DAA0006E0010926F001092700010927100109230
:10DAB000C9001092BC0011B814B817B81AB81DB834
:10DAC00010BA12B815B818B81BB81EB811BA089514
:10DAD000F89480E29EE40197F1F781E08093E00002
:10DAE00080E28093D80080E69AEE0197F1F7CFDFCD
:10DAF0000C9400FEFFCFF894CADF80E69AEE0197FF
:10DB0000F1F70C940000FFCF8F938FB78F93809124
:10DB1000AC0D8D5F8D37D0F48093AC0D8091A80D46
:10DB20008F5F8093A80DD8F08091A90D8F4F8093BF
:10DB3000A90DA8F08091AA0D8F4F8093AA0D78F0BF
:10DB40008091AB0D8F4F8093AB0D09C08D578093A3
:10DB5000AC0D8091A80D8E5F8093A80D28F7809161
:10DB6000A40D8C5F8093A40D58F08091A50D8F4F6C
:10DB70008093A50D28F08091A60D8F4F8093A60D60
:10DB80008F918FBF8F9118959B01AC0114D0FB0131
:10DB90000CC011D06E1B7F0B685E7340D0F3215018
:10DBA000304040405040E851FC4F211531054105BF
:10DBB000510579F708950FB6F89466B515B27091CE
:10DBC000A40D8091A50D9091A60D0FBE10FE05C06D
:10DBD0006F3F19F07C5F8F4F9F4F11240024660F19
:10DBE000001C660F001C702908951F93CF93DF93CC
:10DBF000182FEB013FDE103109F44FC0113160F4F2
:10DC0000113009F442C01130A8F01E3009F455C09B
:10DC10001F3009F05CC049C01931B9F01A3120F445
:10DC2000183109F054C02BC01A31B9F01B3109F07A
:10DC30004EC01DC0209721F4589884B58F7D03C035
:10DC4000C8BD84B5806284BD4AC0D0938900C093AA
:10DC5000880080918000806807C0D0938B00C093BB
:10DC60008A008091800080628093800038C0D093C9
:10DC70008D00C0938C00809180008860F5CFC093A8
:10DC8000B3008091B000806805C0C093B40080915B
:10DC9000B00080628093B00022C0D0939900C093FE
:10DCA00098008091900080680FC0D0939B00C09333
:10DCB0009A0080919000806207C0D0939D00C0932D
:10DCC0009C008091900088608093900008C0E12FB4
:10DCD000F0E0C038D10514F4E7DD01C0DFDDDF91ED
:10DCE000CF911F910895F894E1E6F0E020E82083B9
:10DCF000108283E084BD85BDEEE6F0E08081816026
:10DD0000808391E09093800082E0809381009093E3
:10DD1000B0008093B100909390008093910086E8CA
:10DD200080937A0020937B0010927E00A5D3789494
:10DD30000895FC019FB7F8948091BD0D882311F4DC
:10DD400020E010C083E08093E9002091F2002223BC
:10DD500049F48091E80082FF05C085FD03C08BE691
:10DD60008093E8009FBF8085918597FD03C02F3F7A
:10DD700009F02F5F822F90E00895CF93DF93EC019D
:10DD80008885998597FF09C0E881F9810680F78128
:10DD9000E02DCE0109959987888788859985DF913F
:10DDA000CF910895FC012085318537FD05C08FEFA7
:10DDB0009FEF9187808722C02FB7F8948091BD0D87
:10DDC000882369F083E08093E9009BE68091E80076
:10DDD00085FD09C082FF03C09093E800F7CF2FBFF5
:10DDE0002FEF3FEF0CC09091F1008091E80085FD8E
:10DDF00003C08BE68093E8002FBF292F30E0C901D4
:10DE00000895FC018091BD0D882371F09FB7F894AF
:10DE100083E08093E9002BE602C02093E800809124
:10DE2000E80085FDFACF9FBF8FEF9FEF9187808736
:10DE300008956F927F928F929F92AF92BF92CF92EE
:10DE4000DF92EF92FF920F931F93CF93DF933C01EA
:10DE50008B018091BD0D882329F481E0D3011296B6
:10DE60008C9311C03FB7F89484E08093E9008091CF
:10DE7000B90D882369F08091E80085FD07C03FBF98
:10DE800081E0E3018A8388249924DAC01092B90DD5
:10DE90008824992474E0A72E60E4B62E21EFE22EA8
:10DEA000F12C9AE3C92E83E0D82EC5C09091E400EE
:10DEB000915F8091E80085FD19C03FBF8091E4002B
:10DEC000891731F481E08093B90DF3018283B8C0E2
:10DED0008091BD0D882329F481E0D30112968C93A3
:10DEE000AFC03FB7F894A092E900E3CF8091F20071
:10DEF0002B2D281B822F90E04817590708F4242F58
:10DF0000622F70E0E801D701E0E4E21BE03428F47E
:10DF1000EE0FFF27E257F049099480C089918C9356
:10DF200089918C9389918C9389918C9389918C930D
:10DF300089918C9389918C9389918C9389918C93FD
:10DF400089918C9389918C9389918C9389918C93ED
:10DF500089918C9389918C9389918C9389918C93DD
:10DF600089918C9389918C9389918C9389918C93CD
:10DF700089918C9389918C9389918C9389918C93BD
:10DF800089918C9389918C9389918C9389918C93AD
:10DF900089918C9389918C9389918C9389918C939D
:10DFA00089918C9389918C9389918C9389918C938D
:10DFB00089918C9389918C9389918C9389918C937D
:10DFC00089918C9389918C9389918C9389918C936D
:10DFD00089918C9389918C9389918C9389918C935D
:10DFE00089918C9389918C9389918C9389918C934D
:10DFF00089918C9389918C9389918C9389918C933D
:10E0000089918C9389918C9389918C9389918C932C
:10E0100089918C9389918C9389918C938E018091B5
:10E02000E80085FD02C0C092E800461B570B860E33
:10E03000971ED092B70D4115510509F037CF3FBF5C
:10E04000C401DF91CF911F910F91FF90EF90DF906E
:10E05000CF90BF90AF909F908F907F906F900895DA
:10E06000EDEAFDE08AE0DF011D928A95E9F7109262
:10E07000AF0D88EE93E0A0E0B0E08093B00D9093F8
:10E08000B10DA093B20DB093B30D1092B40D82ED0B
:10E0900092E09093AE0D8093AD0D08952FEF3FEF7A
:10E0A000FC0131872087E8D10FB6F8948091A80D44
:10E0B0009091A90DA091AA0DB091AB0D0FBEAC012E
:10E0C0008091BD0D882329F068EC70E080E090E03D
:10E0D0005BCD8091BE0D882309F10FB6F894809135
:10E0E000A80D9091A90DA091AA0DB091AB0D0FBEF6
:10E0F0009C0110C00FB6F8948091A80D9091A90DC5
:10E10000A091AA0DB091AB0D0FBE821B930B8B3F5C
:10E110009105A8F48091BE0D882361F70FB6F8949D
:10E120008091A80D9091A90DA091AA0DB091AB0D71
:10E130000FBE841B950B855C994008F4C1CF0895F0
:10E14000CF92DF92EF92FF920F931F93CF93DF93C3
:10E150007C016B018A01C0E0D0E00FC0D6016D9157
:10E160006D01D701ED91FC910190F081E02DC70187
:10E170000995C80FD91F015010400115110571F7FD
:10E18000CE01DF91CF911F910F91FF90EF90DF9023
:10E19000CF900895DF93CF9300D0CDB7DEB7DC01E9
:10E1A0008DE089838AE08A83ED91FC91119702804A
:10E1B000F381E02DCD01BE016F5F7F4F42E050E063
:10E1C00009950F900F90CF91DF9108954F925F9234
:10E1D0006F927F928F929F92AF92BF92CF92DF9277
:10E1E000EF92FF920F931F93DF93CF93CDB7DEB7DC
:10E1F000A1970FB6F894DEBF0FBECDBF3C016A01F8
:10E200007B01222349F4DC01ED91FC910190F08126
:10E21000E02D642F09954EC0213009F42AE0C11485
:10E22000D104E104F10421F480E389A310E227C0C2
:10E2300010E2822E9924AA24BB242E010894411CAA
:10E24000511CC701B601A5019401FAD76A3010F438
:10E25000605D01C0695CF201E10FF11D6083C701DF
:10E26000B601A5019401ECD7C901DA016C017D0169
:10E27000C114D104E104F10411F01150E2CF0023E4
:10E2800031F01150FE01E10FF11D8DE28183812FEC
:10E2900090E0D301ED91FC91BE016F5F7F4F680F5D
:10E2A000791F41E250E0481B590B0280F381E02DB9
:10E2B000C3010995A1960FB6F894DEBF0FBECDBF7E
:10E2C000CF91DF911F910F91FF90EF90DF90CF9052
:10E2D000BF90AF909F908F907F906F905F904F9086
:10E2E00008950F9377FD02C000E008C07095609517
:10E2F000509541955F4F6F4F7F4F0DE22AE066DFEB
:10E300000F9108953F924F925F926F927F928F92FA
:10E310009F92AF92BF92CF92DF92EF92FF920F93B4
:10E320001F93DF93CF93CDB7DEB728970FB6F8943E
:10E33000DEBF0FBECDBF3C017A018B01522ECB0157
:10E34000BA0120E030E040E050E096D387FD02C003
:10E35000442406C017FB109517F9109544244394E4
:10E3600020E030E040E05FE3DD240AC0CA01B901EB
:10E370002DEC3CEC4CEC5DE35FD69B01AC01D394FF
:10E38000D514A0F3C801B7019ED24B015C01E8D3BC
:10E390006B017C01C301B701A6012AE0042D16DF41
:10E3A000482E392E552009F447C0C701B60104D4C0
:10E3B0009B01AC01C501B40185D29B01AC018EE289
:10E3C0008983D52C87E0851510F487E0D82EBD2CE5
:10E3D000CC24C3944E010894811C911C1FC0CA0117
:10E3E000B90120E030E040E251E426D67B018C0107
:10E3F000B7D3F401EC0DF11D605D60836053C394ED
:10E4000070E0882777FD8095982FD8D39B01AC01C9
:10E41000C801B70157D29B01AC01BA94BB20F9F6F1
:10E42000D301ED91FC91D3940280F381E02DC301DF
:10E43000B4014D2D50E00995842D932D28960FB6EB
:10E44000F894DEBF0FBECDBFCF91DF911F910F912A
:10E45000FF90EF90DF90CF90BF90AF909F908F9004
:10E460007F906F905F904F903F9008953CDC0E94AA
:10E470002A510E94AC50FDCF8091D80087FF02C086
:10E4800085FF1BC081E88093D70080EA8093D80085
:10E4900086E189BD09B400FEFDCF80E98093D800F4
:10E4A0001092E0001092BD0D1092BE0D1092BA0DA8
:10E4B0001092E1008DE08093E20008951F920F9288
:10E4C0000FB60F920BB60F9211242F933F934F93D9
:10E4D0005F936F937F938F939F93AF93BF93EF93CC
:10E4E000FF931092E9008091E80083FF57C12091CB
:10E4F000F1009091F1004091F1005091F100609194
:10E50000F1007091F100A091F100B091F10082EF63
:10E510008093E800963009F044C0EFE3F0E120E09A
:10E52000859195918417950711F0359617C08591BF
:10E5300095918617970711F0339610C02591359164
:10E540004491CD01AF3FB10519F010F08FEF90E08D
:10E55000841708F4482FF9015EEF04C02F5F2630BE
:10E56000F9F61CC18091E800282F30E0C9018570C0
:10E570009070892BB9F322FD14C1242F413208F089
:10E5800020E2922F04C085918093F100915099234D
:10E59000D1F7421B5093E800442321F7203211F3B6
:10E5A00000C1953061F48EEF8093E8008091E8001F
:10E5B00080FFFCCF842F80688093E300F2C0993005
:10E5C00009F5222309F0EAC04093BD0D1092BA0D5F
:10E5D0001092B70D8EEF8093E800E9E6F0E191E04C
:10E5E0009093E90085918093EB00882331F0859129
:10E5F0008093EC0085918093ED009F5F953081F7CB
:10E600008EE1C7C0983061F4203809F0C7C080910E
:10E61000E80080FFFCCF8091BD0D8093F10096C093
:10E620009132A9F4213A09F0B9C08091E80080FF45
:10E63000FCCF20E030E0F901E35BFD4F8081809367
:10E64000F1002F5F3F4F27303105A9F77FC090328F
:10E6500009F04BC0213209F0A1C08091E80082FF8F
:10E66000FCCF20E030E0F901E35BFD4F8091F10049
:10E6700080832F5F3F4F27303105A9F78BEF8093C1
:10E68000E8008EEF8093E80080914D0290914E0259
:10E69000A0914F02B091500286389105A105B105B5
:10E6A00019F48FE08093B80D80914D0290914E0245
:10E6B000A0914F02B091500286399105A105B10594
:10E6C00009F06FC084E08093E9002FEF06C020932B
:10E6D000E8008091E80082FDFCCF8091EE0090E0A0
:10E6E00083709070892B99F706DA923251F42132B7
:10E6F00009F054C04093BA0D8091E80080FFFCCF30
:10E7000025C0933241F4213209F048C08091E800DD
:10E7100080FFFCCF1BC09923E9F48091E80080FFC3
:10E72000FCCF223811F080E00DC06093E9008091A9
:10E73000EB0090E025E0969587952A95E1F78170AA
:10E740001092E9008093F1001092F1008EEF809317
:10E75000E80027C0913011F0933001F52230F1F438
:10E76000452BE1F4262F2F77822F81508630B0F48D
:10E770008EEF8093E8002093E900933079F089E1EF
:10E780008093EB0081E090E002C0880F991F2A95EA
:10E79000E2F78093EA001092EA0003C081E28093DE
:10E7A000EB00FF91EF91BF91AF919F918F917F917E
:10E7B0006F915F914F913F912F910F900BBE0F90F2
:10E7C0000FBE0F901F9018951F920F920FB60F92C9
:10E7D0000BB60F9211242F933F934F935F936F9338
:10E7E0007F938F939F93AF93BF93EF93FF9380910A
:10E7F000E1001092E100982F83FF11C01092E90010
:10E8000081E08093EB001092EC0082E28093ED00B7
:10E8100088E08093F0001092BD0D1092BA0D92FF27
:10E820001DC08091BD0D8823C9F08091B70D88234C
:10E8300059F081508093B70D882331F484E08093A0
:10E84000E9008AE38093E8008091B80D882331F0D5
:10E8500081508093B80D882309F43AD990FF0CC0F9
:10E8600080E18093E2001092BD0D81E08093BE0DA7
:10E8700080EA8093D80019BC8091BE0D882379F07E
:10E8800094FF0DC086E189BD09B400FEFDCF80E98B
:10E890008093D8008DE08093E2001092BE0DFF912E
:10E8A000EF91BF91AF919F918F917F916F915F9108
:10E8B0004F913F912F910F900BBE0F900FBE0F9075
:10E8C0001F9018955058BB27AA270ED081C241D25D
:10E8D00030F046D220F031F49F3F11F41EF411C203
:10E8E0000EF4E095E7FBDCC1E92F94D280F3BA1770
:10E8F000620773078407950718F071F49EF5C3C289
:10E900000EF4E0950B2EBA2FA02D0B01B90190014A
:10E910000C01CA01A0011124FF27591B99F0593F8E
:10E9200050F4503E68F11A16F040A22F232F342FD6
:10E930004427585FF3CF469537952795A795F04024
:10E940005395C9F77EF41F16BA0B620B730B840B39
:10E95000BAF09150A1F0FF0FBB1F661F771F881FF1
:10E96000C2F70EC0BA0F621F731F841F48F4879549
:10E9700077956795B795F7959E3F08F0B3CF939538
:10E98000880F08F09927EE0F979587950895E1D1A4
:10E9900058F080E891E009F49EEFE2D128F040E8D9
:10E9A00051E059F45EEF09C0ACC16DC2E92FE078C7
:10E9B00031D268F3092E052AC1F326173707480715
:10E9C000590738F00E2E07F8E02569F0E025E064DD
:10E9D0000AC0EF6307F8009407FADB01B9019D0153
:10E9E000DC01CA01AD01EF935DD0F2D10AD05F9195
:10E9F000552331F02BED3FE049E450FD49EC63CF66
:10EA00000895DF93DD27B92FBF7740E85FE316163F
:10EA1000170648075B0710F4D92FA1D29F938F9355
:10EA20007F936F93C0D3E8E9F0E06ED1D1D12F91FD
:10EA30003F914F915F910CD3DD2349F09058A2EAAA
:10EA40002AED3FE049EC5FE3D0785D274DDFDF91B1
:10EA5000BFC102D280F09F3740F491110EF414C26E
:10EA600060E070E080E89FE3089526F01B16611DCA
:10EA7000711D811D1BC135C1EFD008F481E00895DF
:10EA800077D1E395B6C10CD0A3C16AD140F061D172
:10EA900030F021F45F3F19F003C15111F5C131C1CC
:10EAA000B9D198F39923C9F35523B1F3951B550BAD
:10EAB000BB27AA2762177307840738F09F5F5F4F51
:10EAC000220F331F441FAA1FA9F333D00E2E3AF092
:10EAD000E0E830D091505040E695001CCAF729D0AC
:10EAE000FE2F27D0660F771F881FBB1F26173707FB
:10EAF0004807AB07B0E809F0BB0B802DBF01FF272B
:10EB000093585F4F2AF09E3F510568F0C9C0BCC1C1
:10EB10005F3FECF3983EDCF3869577956795B79564
:10EB2000F7959F5FC9F7880F911D9695879597F97F
:10EB30000895E1E0660F771F881FBB1F62177307F8
:10EB40008407BA0720F0621B730B840BBA0BEE1F0D
:10EB500088F7E095089504D06894B11195C108959F
:10EB600061D188F09F5790F0B92F9927B751A0F045
:10EB7000D1F0660F771F881F991F1AF0BA95C9F751
:10EB800012C0B13081F07FD1B1E008957CC1672F10
:10EB9000782F8827B85F39F0B93FCCF38695779501
:10EBA0006795B395D9F73EF49095809570956195EA
:10EBB0007F4F8F4F9F4F0895E89409C097FB3EF415
:10EBC00090958095709561957F4F8F4F9F4F9923BA
:10EBD000A9F0F92F96E9BB279395F6958795779538
:10EBE0006795B795F111F8CFFAF4BB0F11F460FFF8
:10EBF0001BC06F5F7F4F8F4F9F4F16C0882311F050
:10EC000096E911C0772321F09EE8872F762F05C063
:10EC1000662371F096E8862F70E060E02AF09A95FE
:10EC2000660F771F881FDAF7880F9695879597F9F3
:10EC3000089512D180F09F3740F491110EF024C155
:10EC400060E070E080E89FEB089526F41B16611DDC
:10EC5000711D811D2BC045C0990F0008550FAA0BCF
:10EC6000E0E8FEEF16161706E807F907C0F01216DF
:10EC70001306E407F50798F0621B730B840B950BE2
:10EC800039F40A2661F0232B242B252B21F4089537
:10EC90000A2609F4A140A6958FEF811D811D0895D4
:10ECA00097F99F6780E870E060E00895882371F429
:10ECB000772321F09850872B762F07C0662311F415
:10ECC00099270DC09051862B70E060E02AF09A954C
:10ECD000660F771F881FDAF7880F9695879597F943
:10ECE00008959F3F49F0915028F486957795679550
:10ECF000B7959F5F80389F4F880F9695879597F9B6
:10ED000008959FEF80EC0895DF93CF931F930F93A7
:10ED1000FF92EF92DF927B018C01689405C0DA2E9E
:10ED2000EF0196D1FE01E894A59125913591459189
:10ED30005591AEF3EF01D8DDFE019701A801DA94F9
:10ED400079F7DF90EF90FF900F911F91CF91DF91B6
:10ED5000089500240A941616170618060906089541
:10ED600000240A9412161306140605060895C9CF46
:10ED700059D0E8F3E894EFEFBB273FE048EC5FE7BA
:10ED80006B3D73078407950708F1FF279F57B25A19
:10ED90006A4D7F40894CF04032F4BE556542704F59
:10EDA0008643FF4F0894EE1F915030F0BB0F661F53
:10EDB000771F881FFF1FEBCF9EE7882332F0BB0F22
:10EDC000661F771F881F9A95C1F79395E09589CFA5
:10EDD000092E0394000C11F4882352F0BB0F40F469
:10EDE000BF2B11F460FF04C06F5F7F4F8F4F9F4FA9
:10EDF0000895EF93E0FF06C0A2EA2AED3FE049EC58
:10EE00005FEB72DDE5DF0F90039401FC9058E5ECB9
:10EE1000F0E0D3C157FD9058440F551F59F05F3FA4
:10EE200071F04795880F97FB991F61F09F3F79F02C
:10EE300087950895121613061406551FF2CF4695AE
:10EE4000F1DF08C0161617061806991FF1CF869530
:10EE50007105610508940895E5DFA0F0BEE7B917D4
:10EE600088F4BB279F3860F41616B11D672F782FE2
:10EE70008827985FF7CF869577956795B11D93950D
:10EE80009639C8F30895E894BB2766277727CB0106
:10EE900097F90895E1DE08F48FEF08955ADF19F02D
:10EEA0005FDF09F02ECFFCCEB901CA011ACF9F77E0
:10EEB0005F77B0DF98F39923B9F35523B9F3FF27B0
:10EEC000951758F4E52FE91BED3070F75E3B10F015
:10EED000F1E41CC09034E0F40AC0E92FE51BED30EA
:10EEE00028F79E3B10F0F1E411C0503488F4F9EAA1
:10EEF00088232AF09A95660F771F881FDAF7442334
:10EF00002AF05A95220F331F441FDAF79F1B5F1B0D
:10EF1000FF931F930F93FF92EF9279018A01BB2712
:10EF2000AB2F9B01AC0196D09701A801BF937B0149
:10EF30008C01AA27BA2FB901CA018CD0AF919701D1
:10EF4000A801EF90FF900F911F91CEDC41DFE1D03F
:10EF50004F9140FF0895552747FD509509C09B01EB
:10EF6000AC0160E070E080E89FE38DCD99CEB9CE32
:10EF700059DFE8F39923D9F3940F511DBBF3915056
:10EF8000504094F059F0882332F0660F771F881FA5
:10EF900091505040C1F79E3F510544F7880F911D95
:10EFA0009695879597F908955F3FACF0983E9CF051
:10EFB000BB27869577956795B79508F4B1609395CB
:10EFC000C1F7BB0F58F711F460FFE8CF6F5F7F4FB9
:10EFD0008F4F9F4FE3CF58CF25DF58F19E5758F101
:10EFE0009851A0F0E9F0983020F5092E9927660F86
:10EFF000771F881F991F0A94D1F712C0062E672F1A
:10F00000782F8827985F11F4000C07C0993FB4F35C
:10F010008695779567959395D9F7611D711D811D2B
:10F020003EF490958095709561957F4F8F4F9F4FDF
:10F030000895689429CF27CF0BD0CACE8ADE28F056
:10F040008FDE18F0952309F02BCE5BCE11241CCF58
:10F05000E1DEA0F3959FD1F3950F50E0551F629F1D
:10F06000F001729FBB27F00DB11D639FAA27F00D21
:10F07000B11DAA1F649F6627B00DA11D661F829F48
:10F080002227B00DA11D621F739FB00DA11D621F2D
:10F09000839FA00D611D221F749F3327A00D611D4A
:10F0A000231F849F600D211D822F762F6A2F11242C
:10F0B0009F5750408AF0E1F088234AF0EE0FFF1F7F
:10F0C000BB1F661F771F881F91505040A9F79E3FB6
:10F0D000510570F0E5CDD8CE5F3FECF3983EDCF300
:10F0E000869577956795B795F795E7959F5FC1F7F3
:10F0F000FE2B880F911D9695879597F908959F93FC
:10F1000037DE0F9007FCEE5F74CE11F40EF4F9CDEC
:10F11000E8CD88DED0F39923D9F3CEF39F57550B72
:10F1200087FF44D056959795B0E020F4660F771F7F
:10F13000881FBB1F1F930F9300249001A001800123
:10F14000F001A0E80E0F1F1F0A1E511D601B710B5E
:10F150008009B50B48F4600F711F801DB51F0E1B91
:10F160001F0B0A0A510907C02E0F3F1F4A1F0E0F1F
:10F170001F1F0A1E511D660F771F881FBB1FA695F4
:10F18000F795E795F8F60617170708065B07211DA0
:10F19000311D411D0F911F91B901842F9158880F86
:10F1A0009695879508959B01AC0146CF91505040AC
:10F1B000660F771F881FD2F708959F938F937F93D1
:10F1C0006F93FF93EF939B01AC0136DFEF91FF91BB
:10F1D0009BDD2F913F914F915F912ECF629FD00188
:10F1E000739FF001829FE00DF11D649FE00DF11D02
:10F1F000929FF00D839FF00D749FF00D659FF00DB1
:10F200009927729FB00DE11DF91F639FB00DE11D9D
:10F21000F91FBD01CF011124089597FB092E072680
:10F220000AD077FD04D049D006D000201AF470959A
:10F2300061957F4F0895F6F7909581959F4F0895BA
:10F24000A1E21A2EAA1BBB1BFD010DC0AA1FBB1FEA
:10F25000EE1FFF1FA217B307E407F50720F0A21B5C
:10F26000B30BE40BF50B661F771F881F991F1A94C9
:10F2700069F760957095809590959B01AC01BD01F3
:10F28000CF01089597FB092E05260ED057FD04D017
:10F29000D7DF0AD0001C38F4509540953095219561
:10F2A0003F4F4F4F5F4F0895F6F7909580957095BB
:10F2B00061957F4F8F4F9F4F0895AA1BBB1B51E154
:10F2C00007C0AA1FBB1FA617B70710F0A61BB70BD6
:10F2D000881F991F5A95A9F780959095BC01CD017B
:10F2E0000895EE0FFF1F0590F491E02D0994911100
:10F2F0000EC0803219F089508550D0F708959111D1
:10F30000089581548A5108F4805E855A089599279A
:10F31000882708952F923F924F925F926F927F922B
:10F320008F929F92AF92BF92CF92DF92EF92FF9215
:10F330000F931F93CF93DF93CDB7DEB7CA1BDB0BC1
:10F340000FB6F894DEBF0FBECDBF09942A88398866
:10F3500048885F846E847D848C849B84AA84B9846D
:10F36000C884DF80EE80FD800C811B81AA81B98179
:10F37000CE0FD11D0FB6F894DEBF0FBECDBFED018D
:10F38000089511E1CCE4D1E103C0FE01ACDF229687
:0AF39000CE34D107D1F7F894FFCF77
:10F39A00504944204175746F74756E6520737461A9
:10F3AA00727400537465707261746520746F20689A
:10F3BA00696768203A2000005573696E67204465C2
:10F3CA006661756C742073657474696E67733A004C
:10F3DA002569206D696E2C20256920736563004DAF
:10F3EA0031303420496E76616C69642065787472B4
:10F3FA007564657220004D31303520496E76616C36
:10F40A0069642065787472756465722000004D31F4
:10F41A00303920496E76616C69642065787472753A
:10F42A0064657220003F004C20004820006F6B008A
:10F43A0020703A0020693A0020643A0020633A00BA
:10F44A005400496E76616C696420657874727564DB
:10F45A0065720041637469766520457874727564D3
:10F46A0065723A20004D313130004D3239004D3845
:10F47A003420582059205A2045006175746F256937
:10F48A002E67004D3233202573004D3234002F0091
:10F49A0043616E6E6F74206F70656E20737562645F
:10F4AA00697200000000F04185F4103E1070594462
:10F4BA000000803FFF3FFF3F010101010101008081
:10F4CA003B4500803B45000070430000000064009B
:10F4DA00640060EA00000080BB4401BF0D00E10047
:10F4EA00000000080000000058595A4500000100B9
:10F4FA001C001D0013002F00FFFF1E001F0012003A
:10F50A001400FFFF2000210011002400FFFFFFFF6D
:10F51A00FFFF0E001000220023000D000F00010063
:10F52A00FFFFFFFF000028230000282300006400DB
:10F53A000000102700000000FA430000FA43000010
:10F54A00A04000003442B89E2F43B89E2F43E17A70
:10F55A009D449A99BC42000000005E53A0700000CE
:0EF56A000000E311196F996ED26EBD6E016F35
:00000001FF
